:020000040800F2
:10000000E094072489030008356C00909F2D009030
:10001000950300080B0700909784009000000000F3
:10002000000000000000000000000000FF7B0090C6
:100030009908009000000000376C0090017C00904F
:10004000A3030008A3030008A3030008A3030008F8
:10005000A3030008A3030008A3030008A3030008E8
:10006000A3030008A3030008A3030008A3030008D8
:10007000A3030008A3030008A3030008A3030008C8
:10008000A3030008A3030008A3030008A3030008B8
:10009000A3030008A3030008A3030008A3030008A8
:1000A000A3030008A3030008A3030008A303000898
:1000B000A3030008A3030008057C0090A303000825
:1000C000A3030008A3030008A3030008A303000878
:1000D000A3030008D9150008A3030008A303000820
:1000E000A3030008A303000800000000A303000806
:1000F000A3030008A3030008A3030008A303000848
:10010000A3030008A3030008A3030008A303000837
:10011000A3030008A3030008A3030008A303000827
:10012000A3030008A3030008A3030008A303000817
:10013000A3030008A3030008A3030008A303000807
:1001400000000000000000000000000000000000AF
:10015000A3030008A3030008A3030008A3030008E7
:10016000A3030008A3030008A3030008A3030008D7
:10017000A3030008A3030008A3030008A3030008C7
:10018000A3030008A3030008A3030008A3030008B7
:10019000A3030008A3030008A3030008A3030008A7
:1001A000A3030008A3030008A3030008A303000897
:1001B000A3030008A3030008A3030008A303000887
:1001C000A3030008A3030008A3030008A303000877
:1001D000A3030008A3030008A3030008A303000867
:1001E000A3030008A3030008A3030008A303000857
:1001F000A3030008A3030008A3030008A303000847
:10020000A3030008A3030008A3030008A303000836
:10021000A3030008A3030008A3030008A303000826
:10022000A3030008A3030008A303000800000000C4
:10023000A3030008A303000800000000A3030008B4
:10024000A3030008A3030008A3030008A3030008F6
:10025000A3030008A3030008A3030008A3030008E6
:10026000A3030008A3030008A3030008A3030008D6
:10027000A3030008A3030008A30300080000000074
:10028000A303000800000000A30300080000000012
:1002900000000000A303000800F002F800F05CF882
:1002A0000AA090E8000C82448344AAF10107DA45D1
:1002B00001D100F051F8AFF2090EBAE80F0013F0C7
:1002C000010F18BFFB1A43F001031847781800000C
:1002D000981800000A444FF0000C10F8013B13F08E
:1002E000070408BF10F8014B1D1108BF10F8015B8F
:1002F000641E05D010F8016B641E01F8016BF9D182
:1003000013F0080F1EBF10F8014BAD1C0C1B09D1D8
:100310006D1E58BF01F801CBFAD505E014F8016B4A
:1003200001F8016B6D1EF9D59142D6D370470000DC
:100330000023002400250026103A28BF78C1FBD8EE
:10034000520728BF30C148BF0B6070471FB501F08E
:10035000EBFB1FBD10B510BD00F0B0F81146FFF764
:10036000F5FF01F0A9F900F0CEF803B4FFF7F2FFB2
:1003700003BC01F063F9000030BF72B6704762B68B
:10038000704780F30888704709488047094800474C
:10039000FEE7FEE7FEE7FEE7FEE7FEE7FEE7FEE735
:1003A000FEE7FEE704480549054A064B7047000092
:1003B0005515000899020008E0880724E0940724F6
:1003C000E08A0724E08A072453EA020C00F06980DF
:1003D0002DE9F04B4FF00006002B1FBFB3FA83F559
:1003E00003FA05F424FA05F65E4012BF1643B2FA8A
:1003F00082F502FA05F4C5F120051EBF22FA05FCBC
:1004000044EA0C04203556EA044C4FEA144418BF61
:10041000641C4FF000084FF00009904271EB030C90
:1004200039D3002919BFB1FA81F701FA07F6B0FAFA
:1004300080F700FA07F6C7F120071EBF20FA07FC75
:1004400046EA0C062037B6FBF4FCA7EB0507103F85
:1004500007F01F0BCBF120060CFA0BFB2CFA06F66B
:1004600044BFB3460026202FA4BF5E464FF0000BCA
:100470005BEA060C08BF4FF0010B19EB0B09ABFB55
:10048000027C48EB0608C01B06FB02CC0BFB03CC2E
:1004900071EB0C01C1E70B46024641464846BDE8F8
:1004A000F08B13B54FF000004FF00001AFF3008068
:1004B000BDE81C407047704770477047754600F0B4
:1004C0002BF8AE4605006946534620F007008546E6
:1004D00018B020B5FFF766FFBDE820404FF00006DA
:1004E0004FF000074FF000084FF0000B21F007011C
:1004F000AC46ACE8C009ACE8C009ACE8C009ACE85F
:10050000C0098D46704710B50446AFF30080204601
:10051000BDE81040FFF729BF0048704780880724D6
:1005200041F2997CC9F2000C604742F60D3CC9F2D9
:10053000000C604742F6013CC9F2000C604742F6ED
:10054000F74CC9F2000C604745F6492CC9F2000C83
:10055000604742F6156CC9F2000C604746F6197CFC
:10056000C9F2000C604743F22D1CC9F2000C604731
:1005700048F2FD4CC9F2000C60474AF2397CC9F2DE
:10058000000C604745F69F1CC9F2000C604747F21B
:10059000592CC9F2000C604740F6457CC9F2000CAA
:1005A000604748F6ED7CC9F2000C604749F6A14C63
:1005B000C9F2000C604749F2651CC9F2000C6047A3
:1005C00049F6E94CC9F2000C604743F2CD0CC9F280
:1005D000000C604748F6BD7CC9F2000C604745F648
:1005E000291CC9F2000C604742F68D4CC9F2000C80
:1005F00060470000F0B5BFF34F8FBFF36F8F1D4909
:1006000000200860BFF34F8FBFF36F8F1A4C216833
:1006100041F400312160BFF34F8FBFF36F8F164954
:1006200070310860BFF34F8F081F006843F6FF75F5
:10063000104E1036C0F34E31C0F3C90305EA411223
:10064000184642EA80773760401EFAD2491EF5D23A
:10065000BFF34F8F206840F480302060BFF34F8F8E
:10066000BFF36F8F03484C30016841F00401016013
:10067000F0BD000050EF00E014ED00E0024801681A
:1006800041F0010101607047200400582DE9F84F46
:100690006C4C00224FF0B04A4FF0010B4FF0030EAC
:1006A0004FF00F090B680BFA02F73B40BB4270D1C9
:1006B0004D68022D01D0122D12D1D50800EB850C0A
:1006C000DCF820605507ED0E09FA05F826EA080661
:1006D000D1F8108008FA05F848EA0608CCF820801E
:1006E000D0F80080560091F804C00EFA06F50CF020
:1006F000030C28EA05080CFA06FC4CEA080CC0F8C2
:1007000000C0D1F804C0BCF1010F08D0BCF1020F49
:1007100005D0BCF1110F02D0BCF1120F16D1D0F8E8
:1007200008C0D1F80C802CEA050C08FA06F848EA53
:100730000C08C0F80880D0F804C02CEA070C0F7928
:10074000C7F30017974047EA0C074760C768AF43F5
:100750008D68B5403D43C5604D68ED006BD53A4DA1
:100760002E6846F002062E602D6822F0030606F180
:10077000B04605F002050095D6F808C495072F0F7E
:1007800009FA07F52CEA050C304DA84202D10025E4
:100790002EE050E02E4DA84201D1012528E02D4D3C
:1007A000A84201D1022523E02B4DA84201D1032507
:1007B0001EE02A4DA84201D1042519E0284DA84287
:1007C00001D1052514E0274DA84201D106250FE0EF
:1007D000254DA84201D107250AE0244DA84201D1A8
:1007E000082505E0224DA84201D1092500E00A258F
:1007F000BD4045EA0C05C6F8085425684E689D437F
:10080000F60300D51D43256065684E689D43B60319
:1008100000D51D436560DAF8005056464F689D4389
:10082000FF0200D51D43356075684F689D43BF02C8
:1008300000D51D437560521C102AFFF433AFBDE88C
:10084000F88F000080000058F4440258000002585D
:100850000004025800080258000C02580010025808
:100860000014025800180258001C025800200258B8
:10087000002402580069084000D0012070474269F6
:100880004A40426170470AB1018370474183704713
:100890000148806870470000140000240248816805
:1008A000027811448160704714000024032010B5C1
:1008B00000F0A2F80F2000F007F808B1012010BDE9
:1008C00000F06CF8002010BD70B50D4D04464FF4DB
:1008D0007A712878B1FBF0F00A490968B1FBF0F0B1
:1008E00000F0A4FC48B9102C07D200222146501E6B
:1008F00000F062F800206C6070BD012070BD000047
:100900001400002400000024134A41781160111DD6
:1009100003780A1DE3B143680B60017BC37A0907C2
:1009200041EA0361837A41EAC341437B41EA83415F
:10093000837B41EA4341C37B41EA0341437A41EA75
:100940000321037A007841EA4301014311607047B3
:10095000002008601060704798ED00E0BFF35F8FE3
:100960000448016821F4803101600249002070319F
:100970000860704724ED00E0074940F0010008607E
:1009800005487038016841F480310160BFF34F8F32
:10099000BFF36F8F7047000094ED00E070470028B0
:1009A00009DB012100F01F0291404009800000F1A5
:1009B000E020C0F8001170470E4BF0B41B68C3F381
:1009C0000223C3F10704042C00D904241D1D072DA4
:1009D00001D2002300E0DB1E012606FA04F56D1E9D
:1009E0000D409D409E40761E164045EA0601F0BC33
:1009F00000F014BE0CED00E0064A00F0070110689C
:100A00004FF6FF03184040EA0120034908431060F5
:100A1000704700000CED00E00000FA052DE9F047FA
:100A2000DFF8BC9104460E46D9F8000000F007003C
:100A3000B0420CD2D9F8001021F007013143C9F8B7
:100A40000010D9F8000000F00700B0427ED12078F5
:100A5000DFF89081800707D5D8F80010E26821F010
:100A60000F011143C8F800102078C00762D0D8F8F1
:100A70000010A26821F470611143C8F800105949B0
:100A80006068183902281CD003281DD00968012885
:100A90001DD04907002960DA524F083F396821F01C
:100AA000070101433960FFF7F3FE0546606841F234
:100AB0008831022813D003281ED001288A4627D067
:100AC00034E009688903E5E709688901E2E7C905B7
:100AD000E0E7FFF7DDFE411B514501D923E08A46DF
:100AE0003868C0F3C2000228F3D123E0FFF7D0FE3C
:100AF000411B514501D916E08A463868C0F3C2004F
:100B00000328F3D116E0FFF7C3FE411B51450AD875
:100B10003868C0F3C2000128F5D10BE0FFF7B8FE3A
:100B2000411B514502D90320BDE8F087386810F019
:100B3000380FF3D1D9F80010484601F00701B1424F
:100B40000DD9016821F00701314300E005E00160A3
:100B5000006800F00700B04201D00120E4E72078EF
:100B6000400707D5D8F80010226921F07001114321
:100B7000C8F80010207801071B4805D50168626994
:100B800021F07001114301602178C90605D5016883
:100B9000A26921F4E061114301602078800607D545
:100BA0001149091D0868E26920F0700010430860CF
:100BB00000F066F8D8F800104FF4807292FAA2F2B2
:100BC00001F47061B2FA82F2D140084A515CC84027
:100BD000074908600F20FFF777FE0020A4E7000018
:100BE00000200052184402581C440258321B0008CE
:100BF0000000002410B5FFF793FC084909680122A2
:100C000092FAA2F201F00F01B2FA82F2D140044A44
:100C1000515CC8400349086010BD000018440258E8
:100C2000321B00080400002410B5FFF7E3FF07495A
:100C30000968102292FAA2F201F07001B2FA82F26F
:100C4000D140034A515CC84010BD00001C4402580A
:100C5000321B000810B5FFF7CDFF074909684FF4B4
:100C6000807292FAA2F201F4E061B2FA82F2D1400B
:100C7000024A515CC84010BD1C440258321B000897
:100C80003548F0B50068364D10F03801334809D0CA
:100C90000411082904D0334E10290BD018290BD089
:100CA0002046F0BD29688906FBD52968C1F3C1013A
:100CB000C840F0BD3046F0BD274918310A680968C0
:100CC00012F00302284BC1F305111B68274F03F0F4
:100CD00001033F68DFED260AB7EE001AC7F3CC0721
:100CE00017FB03F300EE103A224BB8EE400A06D091
:100CF000012A01D0022A2BD0B4FBF1F008E02A68C7
:100D0000920603D52A68C2F3C102D040B0FBF1F0CD
:100D100001EE900A1868B8EE612AC0F3080001EEEF
:100D2000900A1868F8EE611A40EE201A31EE810A36
:100D300022EE000AC0F34620401C00EE900AF8EEB6
:100D4000600A80EE201ABCEEC10A10EE100AF0BD57
:100D5000B6FBF1F0DCE70000104402580090D0032D
:100D60000044025840787D012C4402583444025813
:100D700000000039304402582DE9F05F0446007845
:100D8000DFF8FC8341F28839DFF8F8A3FE4DC00795
:100D90004ED0D8F800104046C1F3C20102291AD043
:100DA0000068C0F3C200032805D1DAF8000000F0A3
:100DB000030002280FD06068B0F5803F12D010B158
:100DC000B0F5A02F19D0286820F48030286028685A
:100DD00020F4802009E02868800329D56068002875
:100DE00074D025E0286840F480302860606890B1B5
:100DF000FFF74EFD06464F4609E0286840F4802084
:100E00002860EFE7FFF744FD801BB8427DD82868D3
:100E10008003F7D50CE0FFF73BFD06464F4604E0A4
:100E2000FFF736FD801BB842F0D828688003F7D45E
:100E30002078D64F80075AD5D8F8001040464FF496
:100E40007C3B11F0380F13D00068C0F3C2000328B8
:100E500003D1DAF8000080070AD0E068A8B3296857
:100E600021F0190101432960FFF712FD06461DE03C
:100E70002868400702D5E0680028B1D02868E168FA
:100E800020F0190008432860FFF702FD064604E041
:100E9000FFF7FEFC801B0228B8D828684007F7D56A
:100EA00007E0FFF7F5FC801B0228AFD82868400751
:100EB000F7D538689BFAABF220F47C312069B2FA9E
:100EC00082F290400143396011E000E0AEE0286812
:100ED00020F001002860FFF7DBFC064604E0FFF786
:100EE000D7FC801B022891D828684007F7D42078C7
:100EF000C00655D5D8F8001040464FF0F84BC1F366
:100F0000C201012917D0006800E0EDE0C0F3C20083
:100F1000032805D1DAF8000000F0030001280AD008
:100F2000E069002828682CD040F080002860FFF796
:100F3000AFFC064616E02868C00502D5E0698028A7
:100F400074D138689BFAABF220F0F841206AB2FA0B
:100F500082F290400143396022E0FFF799FC801B48
:100F6000022899D82868C005F7D538689BFAABF2F3
:100F7000216AB2FA82F220F0F840914008433860CA
:100F80000EE020F080002860FFF782FC064604E0B7
:100F9000FFF77EFC801B022887D82868C005F7D49D
:100FA0002078000724D5774F60694C3700283868CF
:100FB0000FD040F001003860FFF76AFC064604E0FD
:100FC000FFF766FC801B02288DD838688007F7D5AC
:100FD0000EE020F001003860FFF75AFC064604E0FE
:100FE000FFF756FC801B02287ED838688007F7D4AC
:100FF0002078800623D5A069002828680FD040F407
:1010000080502860FFF744FC064604E0FFF740FCF0
:10101000801B022868D828688004F7D50FE020F4E8
:1010200080502860FFF734FC064605E0D6E0FFF765
:101030002FFC801B022857D828688004F7D420781A
:10104000400744D5524F386840F480703860FFF74D
:101050001FFC064604E0FFF71BFC801B642843D8F6
:101060003868C005F7D5474FA068483701280AD02F
:1010700008B1052811D0386820F0010038603868C0
:1010800020F0040002E0386840F001003860A068F9
:1010900088B1FFF7FDFB064609E0386840F0040020
:1010A0003860F0E7FFF7F4FB811B49451CD838682E
:1010B0008007F7D50BE0FFF7EBFB064604E0FFF7F0
:1010C000E7FB811B49450FD838688007F7D4606A71
:1010D000F0B3D8F80010C1F3C20103297ED0022872
:1010E000286820F0807000E079E0286003D0FFF7E6
:1010F000CFFB044687E0FFF7CBFB064604E0FFF793
:10110000C7FB801B02287BD828688001F7D4DAF857
:10111000001040F2F3329143E26A41EA0211A26AFE
:101120001143CAF8001094F834004FF4FE02218EE7
:101130004002491EA0F5007080B2C1F308010843C7
:10114000218F491E02EA0141084394F83C1000E057
:101150005CE0491E120202EA0161084309490831B4
:1011600008600B1D19684FF6F872A06C914392FA53
:10117000A2F2B2FA82F2904001431960014809E0FC
:1011800010440258284402580044025804440258AB
:1011900000480258001D0168226C21F00C01114327
:1011A00001600168626C21F0020111430160016875
:1011B00041F480310160016841F40031016001684F
:1011C00041F480210160016841F00101016028685B
:1011D00040F080702860FFF75BFB01E018E00FE053
:1011E000044604E0FFF754FB001B022808D82868D7
:1011F0008001F7D50AE0FFF74BFB001B022802D95C
:101200000320BDE8F09F28688001F4D40020F8E7AF
:101210000120F6E74FF0E0210428086903D020F010
:1012200004000861704740F00400FAE7401EB0F186
:10123000807F10B501D3012010BD4FF0E024606124
:101240000F21601700F0EAF90020A061072020615B
:10125000002010BD10B5006886B01B49884230D10F
:101260001A48016841F001010160006800F00100C6
:10127000059016481030016841F0100101600068C7
:101280000121134C00F0100005904FF40070009005
:101290000220CDE901010390072069460490204611
:1012A000FFF7F4F94FF48061204600916946FFF79B
:1012B000EDF92520FFF773FB032225201146FFF7E8
:1012C0007BFB06B010BD000000100140E044025856
:1012D0000000025830B50068114988420CD1114A0B
:1012E0005088010408D411464FF0000344040978E3
:1012F00006D50A2901D0538030BD40F400400DE0EE
:101300000D2909D0084DC0F30D04401C80B2C72838
:1013100029555080EFD830BD40F48040508030BD1A
:10132000001001400C000024C001002454482DE9A5
:10133000F041524C86B0016841F002010160016841
:1013400041F0200101604E480C38016841F48041B1
:10135000016040200090022001900320DFF82481EA
:10136000002569460A270497CDE902504046FFF759
:101370008DF9042069460926049600904046FFF73F
:1013800085F90496C020404E694600903046FFF72C
:101390007DF94FF440706946049700903046FFF79E
:1013A00075F937486438016841F48041016001688B
:1013B00021F4804101603148203881688906FCD4DD
:1013C0003249016032494160016841F00101016028
:1013D00081688906FCD44FF49C714161816889075A
:1013E000FCD5C16841F00201C16081688906FCD466
:1013F0004FF48371416181688907FCD5C16841F070
:101400000201C16081688906FCD4224941610561FD
:1014100081684907FCD530212170016841F0040141
:10142000016081688907FCD5C16841F00201C16093
:1014300081688906FCD481688906FCD4C561164997
:1014400041611648016821F480310160134970310F
:101450000A6822F001020A600A1D156082060F4B1D
:1014600078331A601B1D0E4A1A6005220A60016853
:1014700041F48031016006B0BDE8F0812050005297
:10148000E0440258000402580014025810030001FE
:1014900001041600C0030003EBEF180F24ED00E079
:1014A0002D00030370B5294C9CB0256825F0040578
:1014B0002560264C00260C34256845F440452560FF
:1014C000256805F440451B952568AD04FCD501242D
:1014D00000940CAD03962404019402240994CDE9F0
:1014E0000A410796082485E80D00CDE910466846B4
:1014F000FFF742FC98B9FFF719FF3F201390032034
:10150000CDE9140640200101CDE91640CDE91801CE
:1015100050201A90022113A8FFF780FA10B1012081
:101520001CB070BD0A48016841F0800101600848A4
:10153000F430016841F002010160006800F002002F
:101540001B90FFF79BF80020EAE700000C480258C8
:10155000004402581C48016841F4700101601B49B5
:10156000086840F001000860184A0020103210603E
:101570000A68174B1A400A60144A18321060121D8C
:101580001060121D1060114A28321060121D106088
:10159000121D1060121D1060121D1060121D1060CF
:1015A000121D1060121D10600A6822F480220A6069
:1015B00006496031086001200649C1F80801C006EB
:1015C000014980390860704788ED00E00044025806
:1015D0007FEDF6EA0080005170B50D4D00240D48F6
:1015E000FEF7A3FF02E0641CAC4204D80948FEF7F2
:1015F000A1FF2028F7D1002402E0641CAC4206D8E9
:10160000054901220348FEF79AFF0028F5D170BD75
:10161000FFFF0100880200240C0000240907090EC6
:10162000002804DB00F1E02080F80014704700F08F
:101630000F0000F1E02080F8141D70477047000093
:1016400010B504460420FFF7E5FD0148046010BD15
:101650000800002470B5002405464FF47A7603E0B4
:10166000304600F005F8641CAC42F9D370BD0000B0
:1016700070B54FF0E02500216C69094AAB6912682A
:101680005043AA699A42FCD002D2A3EB020302E0C3
:10169000A4EB02063344194413468142F1D370BDD2
:1016A000080000240349CA695206FCD5C2B20A8563
:1016B00070470000001001401FB5FEF79BFFFFF7C9
:1016C000F5F8042302220521A020FFF7EBFE4FF4DA
:1016D000C870FFF7B5FF4FF4E13000F009FA9E48FB
:1016E0004168C8208847FEF72FFFFEF732FFFEF75C
:1016F00035FFFEF738FFFEF73BFF0020FEF73DFF0A
:101700000120FEF73AFF0220FEF737FF0320FEF725
:1017100034FF0420FEF731FF0520FEF72EFFDFF82F
:101720003C828FA010244FF478412346C822C8F889
:1017300000103221CDE900401E20FEF723FF8DA0CE
:101740001023C822CDE9004046211E20FEF71AFFD3
:101750008BA01023C822CDE900405A211E20FEF79D
:1017600011FF8BA01023C822CDE900406E211E205E
:10177000FEF708FF89A01023C822CDE9004082218E
:101780001E20FEF7FFFEDFF828924FF4FA751BE0EB
:1017900088A01023C822CDE9004096211E20FEF724
:1017A000F1FE2846FFF756FF86A01023C822CDE998
:1017B000004096211E20FEF7E5FE2846FFF74AFF6F
:1017C00002214846FFF75BF8FEF7E1FE0028DFD173
:1017D000FEF7E2FEFEF7E5FE7E4D01227EA12868BF
:1017E000FEF7E4FE686801227CA1FEF7DFFE7C4F75
:1017F0000D284FF400764FF47A7A1CD179A010238B
:10180000C822CDE9004096211E20FEF7BBFE0096BF
:1018100000223B68072171A0FEF7CDFE98B178A0A9
:101820001023C822CDE9004096211E20FEF7AAFE13
:101830005046FFF70FFFA868012278A1FEF7B6FE19
:101840000D2805D021E076A0FEF7BAFE77A0E7E7E5
:101850007DA01023C822CDE9004096211E20FEF76E
:1018600091FE009600223B6807216CA0FEF7A3FEC4
:10187000B0B17BA01023C822CDE9004096211E20E4
:10188000FEF780FE5046FFF7E5FEA6234FF6FF75F4
:10189000F022009596211E20FEF797FE4E461EE090
:1018A00075A0FEF78DFE77A0E4E77CA01023C82288
:1018B000CDE9004096211E20FEF764FEC820FFF708
:1018C000C9FEA6230095F02296211E20FEF77DFE7C
:1018D000C820FFF7BFFE02213046FEF7D0FF03AA63
:1018E00002A923A0FEF776FE0028DED171A01F21F9
:1018F000C8F800101023CDE90040C82296211E2010
:10190000FEF740FE6EA01023C822CDE90040AA21B8
:101910001E20FEF737FE70A01023C822CDE900403C
:10192000BE211E20FEF72EFE02980523AA21009458
:10193000820A8E20FEF753FE03980523BE210094F1
:10194000820A8E20FEF74BFEC820FFF783FE02219D
:101950003046FEF794FFF7E77C00002420000024C7
:10196000504F4C4152495320483735302F46373578
:101970003000000046415446532054455354000063
:1019800041544F4D40414C49454E54454B00000099
:10199000323031392F352F31320000005573652038
:1019A00055534D41525420666F7220746573740014
:1019B0000004025853442043617264204572726FE0
:1019C00072210000506C6561736520436865636B2C
:1019D0002120000048180024303A0000313A00006D
:1019E0007C010024466C617368204469736B204657
:1019F0006F726D617474696E672E2E2E0000000088
:101A0000466C617368204469736B20466F726D6128
:101A100074204572726F722000000000323A00009C
:101A2000313A414C49454E54454B0000466C617378
:101A300068204469736B20466F726D61742046693B
:101A40006E697368000000004E414E442044697383
:101A50006B20466F726D617474696E672E2E2E0056
:101A60004E414E44204469736B20466F726D617421
:101A7000204572726F722000323A4E414E44444902
:101A8000534B00004E414E44204469736B20466F17
:101A9000726D61742046696E697368005344204317
:101AA000617264204661746673204572726F7221A0
:101AB000000000004641544653204F4B21000000D7
:101AC000534420546F74616C2053697A653A202026
:101AD0002020204D420000005344202046726565BE
:101AE0002053697A653A20202020204D42000000D2
:101AF0000B490A4A10B5C1E9002000208860C8607F
:101B0000086188610C2048610846FEF76DFDBDE85C
:101B10001040044901220248FEF711BD00100140A7
:101B2000880200240C0000244FF04070E1EE100AFF
:101B300070470000000001020304010203040607CD
:101B400008090000641B000800000024C001000018
:101B5000D4020008E81B0008C001002420930700FD
:101B600030030008113C90D00304B13201A2102AC6
:101B7000FF0181CB18EF191E38AE03904C041A54A4
:101B8000041A40041A5C041A3C041A440413D3A92E
:101B90001B9084081321BA1B9060081355161B086C
:101BA0009C081A71082AB42C21142479B1149025A8
:101BB000AB1B90B9041AD90C4A047F01E91339A769
:101BC0001B90ED04138018122434401FC0323032B1
:101BD0003842201C80180718133FC314C003301A62
:081BE000F0181CE0012008913F
:0200000490006A
:10000000642900F08F80752900F08C80782900F039
:10001000C580632900F0D582732900F0DA820020C0
:10002000704710B54C1084EA530404D54042C1F126
:10003000000138BF491E1B4204D55242C3F10003E0
:1000400038BF5B1E00F0F8FA14F0804F04D0404235
:10005000C1F1000138BF491E14F0004F04D05242D4
:10006000C3F1000338BF5B1E10BD00000FB404498C
:1000700010B503AA029800F0B1FA10BC5DF814FBA9
:100080001000002470B5044685690068C10601D5DA
:10009000302600E02026C00707D070BDD4E901213A
:1000A00030469047206A401C20626D1EF6D570BD18
:1000B00070B5044685690078C00707D170BDD4E9E2
:1000C000012120209047206A401C20626D1EF6D539
:1000D00070BD70B50C460546012A05D0287880060B
:1000E00000D5EA69002302E0012305E05B1C93428E
:1000F00002D2E05C0028F9D1A869E618C01AA8610C
:10010000286A184428622846FFF7BCFF04E0D5E9B6
:10011000012114F8010B9047B442F8D32846FFF7A9
:10012000C7FF70BD2DE9F04106460024106875290F
:10013000314616A510D0AFF30080002802DA404205
:1001400013A507E031688A0701D512A502E0490727
:1001500004D511A5012401E0AFF3008000210A229B
:1001600006F1240709E0B0FBF2FCB0FBF2F302FB5E
:100170001C00303078541846491C0028F3D123461F
:100180002A463046BDE8F04100F0B8B90000000052
:100190002D0000002B0000002000000070B5044678
:1001A0000D4621461068AFF300802188090502D56D
:1001B0000F4A7A4402E00E4A7A440E32002104F1DA
:1001C000240305E000F00F060009965D5E54491C0B
:1001D0000028F7D120780023000704D5702D02D025
:1001E00009B1022311322046BDE8704000F086B903
:1001F00046AC03002DE9F05F894604464FF0000A43
:10020000DFF874B1FB44C0F820A02046E1688847BD
:10021000002874D0252806D0D4E901219047206A0F
:10022000401C2062F1E700265F462046E1688847CF
:100230002028054607DB312D05D2781910F8200C4F
:1002400008B10643F1E7B00701D526F00406C4F86B
:100250001CA00027C4F818A02A2D09D0284608F0B1
:10026000E5FA38B304EB8708303DC8F8185019E0B8
:1002700059F8041B204604EB87029161E168884726
:10028000012F054618D1E069002820DA26F0200663
:100290001DE0D8F8180000EB800005EB4000303876
:1002A000C8F818002046E1688847054608F0BEFAFD
:1002B0000028EED1012F0AD02E2D08D12046E1686A
:1002C00088477F1C0546022F46F02006C4DBA06944
:1002D000002803DA404246F00106A061F00701D091
:1002E00026F010066C2D0BD0682D09D04C2D39D07E
:1002F0006A2D35D0742D35D07A2D33D016E038E004
:10030000E1682F4620468847B842054609D16C2F40
:1003100026D04FF48060E1680643204688470546B2
:1003200004E06C2F1AD04FF4807006430DB3A5F192
:100330004100192802D8203546F400664A4629466D
:10034000204626604E46FFF75BFE80B101280BD0A9
:10035000F61D26F0070000F1080956E74020E4E703
:100360008020D8E70020D6E706F104094DE72846AB
:1003700052E7206ABDE8F09F1CAC0300032A40F25C
:10038000308010F0030C00F0158011F8013BBCF137
:10039000020F624498BF11F801CB00F8013B38BF4F
:1003A00011F8013BA2F1040298BF00F801CB38BF5D
:1003B00000F8013B11F0030300F02580083AC0F07B
:1003C000088051F8043B083A51F804CBA0E8081023
:1003D000F5E7121D5CBF51F8043B40F8043BAFF356
:1003E0000080D20724BF11F8013B11F801CB48BFB0
:1003F00011F8012B24BF00F8013B00F801CB48BFE6
:1004000000F8012B704710B5203AC0F00B80B1E81E
:100410001850203AA0E81850B1E81850A0E8185039
:10042000BFF4F5AF5FEA027C24BFB1E81850A0E842
:10043000185044BF18C918C0BDE810405FEA827C5C
:1004400024BF51F8043B40F8043B08BF7047D20773
:1004500028BF31F8023B48BF11F8012B28BF20F814
:10046000023B48BF00F8012B70474FF000020429FF
:10047000C0F0128010F0030C00F01B80CCF1040CD3
:10048000BCF1020F18BF00F8012BA8BF20F8022B07
:10049000A1EB0C0100F00DB85FEAC17C24BF00F8AD
:1004A000012B00F8012B48BF00F8012B70474FF0DB
:1004B000000200B5134694469646203922BFA0E8B4
:1004C0000C50A0E80C50B1F12001BFF4F7AF0907C0
:1004D00028BFA0E80C5048BF0CC05DF804EB8900B1
:1004E00028BF40F8042B08BF704748BF20F8022BF4
:1004F00011F0804F18BF00F8012B70472DE9F0472D
:100500000D4699469246044600F124080168880683
:1005100004D5E06921F01001216000E00120A8422B
:1005200001DD471B00E00027A1697A1902EB0900F1
:10053000081AA0612078C00602D42046FFF7A2FD69
:10054000002608E0D4E901211AF806009047206A45
:10055000401C761C20624E45F4DB2078C0060AD58C
:100560002046FFF78FFD06E0D4E9012130209047B7
:10057000206A401C2062381EA7F10107F4DC07E066
:10058000D4E9012118F805009047206A401C206238
:10059000281EA5F10105F3DC2046FFF789FD207830
:1005A000000602D50220BDE8F0870120FBE710B568
:1005B000436913B1AFF3008001E0FFF78AFD01202A
:1005C00010BD127800F124010A7000224A70012245
:1005D000EDE711684FF0FF32E9E70000074B70B517
:1005E0000D467B4400F011F80446284600F020F840
:1005F00010B14FF0FF3070BD204670BDBF100078C5
:1006000001694A1C02610878704700B58FB0CDE9D6
:1006100001310021059105497944CDE903101146C6
:100620006846FFF7E7FD0FB000BD0000E5FFFFFFE4
:10063000007B00F08000704740F2C93CC0F6000C1F
:10064000604740F28D6CC0F6000C604740F6814C6C
:10065000C0F6000C604740F6F53CC0F6000C604761
:1006600040F6910CC0F6000C604741F2552CC0F6E4
:10067000000C604741F2556CC0F6000C604741F237
:10068000716CC0F6000C604740F6870CC0F6000C99
:10069000604740F65D1CC0F6000C604740F6091C40
:1006A000C0F6000C604740F6791CC0F6000C6047AD
:1006B00040F6750CC0F6000C604740F6B91CC0F659
:1006C000000C604740F69F1CC0F6000C604740F2EB
:1006D0007B3CC0F6000C604740F27F3CC0F6000C4B
:1006E000604740F69D0CC0F6000C604741F2D52CE7
:1006F000C0F6000C604740F6294CC0F6000C60477D
:1007000040F6554CC0F6000C6047FEE7084A002052
:100710004FF4803102E0536B1B0602D4491EFAD21B
:1007200000E011B103499163704703207047000056
:1007300000700052FF0FE01F0E4A10B5516B11F010
:10074000450FFBD00C4B4C0704D5042090639363FA
:10075000032010BDC90702D00120906310BD1169AC
:10076000814201D0102010BD9363506900F0080051
:1007700010BD000000700052FF0FE01F10B50F4CBD
:1007800000204FF480320BE0616B11F0450F07D071
:100790000AB14A0707D5A16B032041F004010AE022
:1007A000521EF1D2F5E7C90704D0A16B012041F038
:1007B0000101A1630249A16310BD00000070005255
:1007C000FF0FE01F0849486B10F0450FFBD04007B2
:1007D00005D5886B40F00400886303207047034808
:1007E000886300207047000000700052FF0FE01F78
:1007F00030B5174B054600205A6B12F0450FFBD061
:10080000540705D5986B40F004009863032030BD71
:10081000D20705D0986B40F001009863012030BDED
:100820001A69AA420ED10B4A9A635A6912F4604FB0
:1008300003D0910404D5132030BD120C0A8030BDC2
:10084000510401D5102030BD1104FCD50F2030BD5E
:1008500000700052FF0FE01F10B50E4C00204FF447
:1008600080320BE0616B11F0450F07D00AB14A07E7
:1008700007D5A16B032041F0040108E0521EF1D21C
:10088000F5E7490604D5A16B002041F04001A163C2
:1008900010BD0000007000527047C268D1E900230B
:1008A00042EA03220B89097B1B0443EA01610A43E4
:1008B000C260002070478268D1E9002342EA032227
:1008C0000B89097B1B0443EA01610A438260002013
:1008D0007047000030B50268094B1A40D1E9013475
:1008E0002343D1E903452C4323434C69896943EAF7
:1008F000442343EA413111430160002030BD000030
:100900008901F0FF70B5B3F5804F05D06FF07041ED
:1009100040F82210002070BD50F82230084C2340CF
:10092000D1E900458E8944EA05148D6889692D0254
:1009300045EA06452C430C431C4340F82240E9E7B6
:100940000000F0CFF0B50C6850F824501A4A15405A
:10095000D1E90123D1E903671A433E4332434E698B
:1009600032438E693243CE6932430E6A32434E6A55
:1009700032438E6A3243CE6A32430E6B32438E6B01
:1009800032434E6B32432A43082B01D142F04002DE
:1009900040F824200A6BB2F5801F05D10A684AB1DD
:1009A000026842F4801202600A681AB10268496B58
:1009B0000A4302600020F0BD8004C0FF00EB820209
:1009C000F0B553688E8903F04044D1E9003543EA1D
:1009D00005138D682D0245EA06450E8A2B430D4D01
:1009E00005EB065633430E7D6F0107EB0666334376
:1009F0008E693343234353600268D20207D54268AD
:100A0000098A22F4700205EB015111434160002074
:100A1000F0BD00000000F0FF30B5D1E901230D6802
:100A20001A43D1E9033423431A434B691A438B69B0
:100A30001A43D1E90734496A012D056807D01A43E2
:100A400022430A436FF30E052A4302600AE025F4AD
:100A5000F845234329430B43416803606FF30E01BC
:100A60000A434260002030BD426942EA41014161CF
:100A70000020704718B5D1E900236FF01F041A4316
:100A80008B68C96804EB431343EA41210A4300928F
:100A90000261002018BD0000F0B5D1E900346FF00C
:100AA0000F055B1E2E0105EB041423438C682F03F6
:100AB0004FEA054C0D8A06EB04248E8A2343CC684A
:100AC000097E4FF07F4E012A07EB05450CEB0656D9
:100AD0000EEB01610CD082683F1107EB0434234315
:100AE0002B4333430B4302F07042134383600FE008
:100AF0008768084A17402203C468A2F5805232432F
:100B00003A4382602B430B4304F070442343C36099
:100B10000020F0BDFF0F0FFF38B50A4D04464FF01F
:100B2000AA306A46009004230021A879604306F0A9
:100B300071F8A879042300216A466043401C06F03E
:100B400069F838BDA01700242DE9FC47254F002582
:100B50008946064600240DF1040810E0CDF8008017
:100B60004A46798870438B08002105F0CBFE7888CF
:100B7000BDF80410B1EB900F04D1641CA4B2B87995
:100B8000A042EBD8B879A04202D10020BDE8FC8792
:100B9000304605F08FFC20B113A02946FFF766FA16
:100BA00016E0B9F1FF3F13D000200AE07A8806FB77
:100BB000001093080022114606F000F8BDF804006A
:100BC000401CADF80400B879BDF804108842EDD897
:100BD0006D1CADB2032DBDD309A03146FFF746FA17
:100BE0000120D3E7A01700246572726F722065722E
:100BF00061736520626C6F636B3A25640D0A0000B7
:100C000062616420626C6F636B20636865636B650F
:100C1000643A25640D0A000038B5114D04460020E1
:100C20006A468DF8000001230021A879604305F091
:100C3000A1FE9DF80000FF2801D0022038BDA87950
:100C4000012300216A466043401C05F093FE9DF895
:100C50000000FF2801D0012038BD002038BD000071
:100C6000A01700242DE9F84F91462F4A8A461D46C9
:100C70009179B0FBF1F3B0FBF1F801FB130B4046A7
:100C800000F0B8F8284907464889B84202D2012046
:100C9000BDE8F88F002428E05C4516D3ADB14A8842
:100CA000A2EB0A01A94201D28EB200E0AEB24B46DD
:100CB00007FB004108FB00405246009605F068FA29
:100CC000AD1B4FF0000AB14405E007FB004108FBF3
:100CD000004005F03FFB30B13846FFF71DFF012013
:100CE00000F024F8CBE7641CA4B20F498879A04235
:100CF000D2D80D46A879A04214D1384600F028FA7F
:100D0000404605F0D7FB6A890020696908E031F8A0
:100D10001040444502D121F8107003E0401C80B21D
:100D20008242F4D80020B3E7A0170024F8B52A4D7A
:100D3000002106464FF6FF7003E06A6922F81100B1
:100D4000491C6A898A42F8D80020A88104461CE020
:100D5000A879042300216A46604305F00BFE9DF844
:100D60000000FF280CD1B6B1A879012300216A4602
:100D70006043401C05F0FEFD9DF80000FF280AD0EE
:100D800016A02146FFF772F9641C6989A142DFD8D9
:100D90006A69002016E09DF803109DF8020000EB40
:100DA00001206989814202D9696921F81040A88926
:100DB000401CA881E8E732F810308B4201D3E8816B
:100DC00002E0401C8142F6D8E889642801D2022062
:100DD000F8BD0020F8BD0000A01700246261642067
:100DE000626C6F636B20696E6465783A25640D0AE6
:100DF0000000000070B5104E104C71892268491E29
:100E0000914200D2216000F001052068294600F0DF
:100E100017F8411C0AD170892168401E884207D901
:100E20002946206000F00CF8411C01D0206070BD04
:100E30004FF0FF3070BD0000A01700243C000024DC
:100E4000F8B5401C0D4600210400009112D00C4F53
:100E5000012626EA0400A8420AD1B879611E0423BB
:100E60006A464843002105F085FD0098401C04D0E7
:100E7000641EEED14FF0FF30F8BD601EF8BD0000DB
:100E8000A0170024F8B5254E00273C46B78113E093
:100E90002046FFF7C1FE70B9204605F00BFB38B1C4
:100EA0001FA02146FFF7E2F82046FFF735FE02E0DB
:100EB000B089401CB081641C7089A042E8D8B18917
:100EC0001BA0FFF7D3F8B089642801D20120F8BD38
:100ED000C0EB40100097642100EB4000B0FBF1F53F
:100EE000002410E02046FFF797FE58B9B07902239E
:100EF0006A461946604305F08DFE0098401C00903C
:100F0000A84203D0641C7089A042EBD80120FFF7EF
:100F10000DFF0028DBD00220F8BD0000A017002440
:100F200042616420626C6F636B3A25640D0A0000B5
:100F3000676F6F645F626C6F636B6E756D3A25648B
:100F40000D0A000010B505F0E1FA00BB184C61690C
:100F500011B1002009F068FC60894100002009F00F
:100F60006FFC606161894900FFF77FFA606970B1C9
:100F70000120FFF7DBFE60B10EA0FFF777F8FFF767
:100F800081FF90B111A0FFF771F8022010BD012080
:100F900010BD618912A0FFF769F8A18916A0FFF7BB
:100FA00065F8E18919A0FFF761F8002010BD000085
:100FB000A0170024666F726D6174206E616E6420EC
:100FC000666C6173682E2E2E0D0A0000666F726DBE
:100FD0006174206661696C6564210D0A000000007F
:100FE000746F74616C20626C6F636B206E756D3A08
:100FF00025640D0A00000000676F6F6420626C6F4B
:10100000636B206E756D3A25640D0A0076616C691C
:101010006420626C6F636B206E756D3A25640D0AF7
:10102000000000000549CA89824202D24FF6FF70D3
:101030007047496931F8100070470000A01700247C
:101040002DE9FF5F00269B461546824679E03F4C1E
:101050006088B0FBF5F1A079414301988319B3FB97
:10106000F1F0FFF7DFFF6189814203D8012004B06E
:10107000BDE8F09F354C6188A479B1FBF5F262437D
:10108000B3FBF2F702FB17326A43B2FBF1F300FB4A
:101090000437B2FBF1F001FB1028A1EB0800B0FB14
:1010A000F5F084B2ABEB0600A04200D284B2524607
:1010B0001FFA88F1384604FB05F91FFA89F305F099
:1010C000FBFA032809D11FFA89F352461FFA88F167
:1010D000384605F0F1FA032804D004282ED068B36E
:1010E0000220C4E71FFA88F14B4652463846FFF704
:1010F000B9FDDFF858804FF0FF3198F80600B7FBD4
:10110000F0F0FFF721FD80B998F806000021B7FB49
:10111000F0F0FFF719FD814698F80600B7FBF0F0F4
:1011200005F0C8F9B9F1000F08D098F80600B7FB30
:10113000F0F0FFF7F1FC0120FFF7F8FD05FB04AA32
:1011400026445E4583D3002091E70000A0170024C9
:1011500008B5CC216A4601238DF80010034989792E
:101160004843194605F056FD08BD0000A0170024AD
:101170002DE9FF4F0027154685B04FF0FF3B7BE080
:10118000404C6088A179B0FBF5F048430699CB1933
:10119000B3FBF0F0FFF746FF61898046414503D875
:1011A000012009B0BDE8F08F364A50889279B0FB33
:1011B000F5F15143B3FBF1F401FB143101FB05FAE6
:1011C000BAFBF0F308FB0231BAFBF0F20291089986
:1011D000C91B03918CB200FB12A9A0EB090080B2DD
:1011E000B0FBF5F0ADF80400844200D304464FF0A4
:1011F000FF3201A8009004FB05F61FFA89F102985E
:10120000C6F38F0305F07EFB08B10220C9E7BDF8E5
:101210000400B0EB960F0FD1B3B2059A1FFA89F113
:10122000029805F01BFC38B9C345414620D008465A
:10123000FFF78EFFC346D8B11248817940884143F9
:10124000A1EB0A000399B0FBF5F08CB280B2ADF8C7
:101250000400844200D30446059A1FFA89F10298DB
:1012600004FB05F63346FFF7FDFC08B1032098E7C1
:1012700005982744304405900898874280D3002081
:101280008FE70000A0170024F0B500240E460822C6
:10129000074601212546102005F01CFE1020FFF70F
:1012A0004BFA00282ED13A040121372005F012FE16
:1012B0003720FFF741FA002824D101230322082117
:1012C000401E05F013FE00220121332005F002FE2E
:1012D0003320FFF731FA002814D1174940F22A527F
:1012E0004B6B134206D14B6B1B03F9D4D1F88040F2
:1012F000D1F880504A6B120705D5886B40F0080082
:1013000088630420F0BD4A6B920705D5886B40F0D6
:10131000020088630220F0BD4A6B920605D5886BF7
:1013200040F0200088630620F0BD044A8A6321BA99
:10133000716029BA3160F0BD00700052FF0FE01FEC
:1013400010B528B190F83510022903D080214165ED
:10135000012010BD1D4A4FF4956301688C189C4212
:1013600007D8042280F83520086820F001000860C2
:1013700029E00C6824F00E040C6001680A440A6835
:1013800022F001020A60016E0A6822F480720A608B
:1013900090F85C30012202FA03F10D4B1960D0E99C
:1013A00019134B60C16E31B10B6823F480730B606D
:1013B000D0E91C134B60002180F8341080F83520F0
:1013C000016D01B18847002010BD0000F0FFFDBF96
:1013D000045402582DE9F041044690F8A000154647
:1013E0000F4601281DD0012684F8A060022084F851
:1013F000A10005EB850000EBC500342204EB800062
:101400003830FFF700F82A463946204604F00EFE31
:101410002068466284F8A160002084F8A000BDE83E
:10142000F0810220FBE7000070B5040004D094F8BE
:10143000A100002510B106E0012070BD204684F80F
:10144000A05000F06BF8022084F8A10020688169A8
:1014500021F070418161D4E901100143D4E9030214
:1014600010430143206882691143816120688268CA
:1014700029490A408260A08A020420688368A6691C
:101480003343134383602068C2680A40C260A08B64
:1014900002042068C368266A33431343C36020688C
:1014A00002690A400261A08C020420680369A66AEE
:1014B000334313430361206842690A404261A08DAF
:1014C000010420684269236B1A430A43426194F87D
:1014D0003500020294F8360001042068C36A03F064
:1014E0007F43C3622068C36A114394F83460334376
:1014F0000B43C3622068416B41F0060141632068E1
:10150000816941F001018161C4F8A450012084F88F
:10151000A100002070BD000000F800F02B4810B5BD
:1015200086B0016841F008010160006800F0080021
:10153000059026481038016841F0100101600068EC
:1015400000F0100005902148001F016841F48071EF
:101550000160016801F480710591016841F4007136
:101560000160016801F400710591016841F4806136
:10157000016000680324694600F480600590202023
:10158000009001200190CDE902041148FFF759F8BD
:101590004FF4E04000900220019000206946CDE920
:1015A00002040E2004900B48FFF74BF848F67C60CD
:1015B000009009486946FFF744F8FF20009007486B
:1015C0006946FFF73EF806B010BD0000E44402583B
:1015D0000004025800200258002402580028025833
:1015E00070B5044690F8A0000E46012820D00125D1
:1015F00084F8A050022084F8A10003EB830000EBE4
:10160000C30004EB80018E63086E3044C1E90F0211
:10161000486E1044486438311A46204604F006FDEE
:101620002068456284F8A150002084F8A00070BDB5
:10163000022070BD70B5044690F8A0000E46012847
:1016400020D0012584F8A050022084F8A10003EBEB
:10165000830000EBC30004EB8001886B3044C86357
:10166000086C10444864C1E9186238311A462046B3
:1016700004F0DCFC2068456284F8A150002084F866
:10168000A00070BD022070BD70B5040015460E4666
:1016900003D094F8210010B107E0012070BD0020B4
:1016A00084F82000204600F01FF82068211DFFF775
:1016B00011F9D4E900023146FFF7FDF8D4E9000240
:1016C0002946FFF7EAF82068016841F0040101604B
:1016D0000448016841F000410160012084F82100C4
:1016E000002070BD00400052274870B586B00168E8
:1016F00041F480510160006800F480500590224858
:101700000C30016841F008010160016801F0080136
:101710000591016841F010010160016801F01001BC
:101720000591016841F04001016000680024032533
:10173000164E00F04000059040206946CDE90004B7
:101740000120CDE902053046FEF77BFF01A94FF4E9
:1017500000700090022081E831000C2004900C48B9
:101760006946FEF76EFF4DF633006946029400901D
:101770003046FEF766FF4FF4F0600090054869467A
:10178000FEF75FFF06B070BDD4440258000C02584B
:10179000001802580010025810B5FEF757FF08490C
:1017A00009684FF4807292FAA2F201F47061B2FA01
:1017B00082F2D140034A515CC8400349086010BD21
:1017C00018440258321B00080000002410B5FEF730
:1017D00042FF07490968102292FAA2F201F0700153
:1017E000B2FA82F2D140034A515CC84010BD0000F9
:1017F00020440258321B0008364930B50A6809688F
:1018000012F00302344BC1F305311B68334C03F073
:1018100010032468DFED320AB7EE001AC4F3CC04DB
:1018200014FB03F300EE103A2E4BB8EE400A07D03B
:101830002D4C012A01D0022A4AD0B4FBF1F10BE071
:10184000244C283C22689506284A03D52468C4F312
:10185000C104E240B2FBF1F101EE901A1968B8EE52
:10186000612AC1F3080101EE901A1968F8EE611AB5
:1018700040EE201A31EE810A22EE000AC1F3462121
:10188000491C00EE901AF8EE600A80EE201AFCEE79
:10189000C10AC0ED000A1968C1F30641491C00EEF7
:1018A000901AF8EE600A80EE201AFCEEC10AC0ED34
:1018B000010A1968C1F30661491C00EE901AF8EE9E
:1018C000600A80EE201ABCEEC10A80ED020A30BD2B
:1018D000074ABFE7284402582C4402583C440258A7
:1018E000000000393844025800093D000090D00340
:1018F00040787D01364930B50A68096812F0030264
:10190000344BC1F305511B68334C03F480732468D6
:10191000DFED320AB7EE001AC4F3CC0414FB03F374
:1019200000EE103A2E4BB8EE400A07D02D4C012A9B
:1019300001D0022A4AD0B4FBF1F10BE0244C283C40
:1019400022689506284A03D52468C4F3C104E240FE
:10195000B2FBF1F101EE901A1968B8EE612AC1F3F9
:10196000080101EE901A1968F8EE611A40EE201A8B
:1019700031EE810A22EE000AC1F34621491C00EE35
:10198000901AF8EE600A80EE201AFCEEC10AC0ED53
:10199000000A1968C1F30641491C00EE901AF8EEDE
:1019A000600A80EE201AFCEEC10AC0ED010A196837
:1019B000C1F30661491C00EE901AF8EE600A80EE51
:1019C000201ABCEEC10A80ED020A30BD074ABFE70B
:1019D000284402582C44025844440258000000395C
:1019E0004044025800093D000090D00340787D013A
:1019F0002DE9F84F0446006800252E46010104F148
:101A00002400FE4FDFF8F88300901DD5606E50B1C2
:101A1000B0F5801F0CD0B0F5001F0ED0B0F5401F00
:101A20001DD001250FE0386840F40030386016E022
:101A30000221201D05F000F903E00098022105F0C5
:101A400073F905000BD02E462088C00523D5606DA4
:101A500005281ED2DFE800F00C11161B1B00D8F879
:101A60000010626E21F440111143C8F80010EBE73A
:101A7000386840F40030386009E00021201D05F08E
:101A8000DBF803E00098002105F04EF905466DB142
:101A900000E001252E432088800528D5A06D8028F0
:101AA0001ED00CDC90B140280ED114E0D8F8001004
:101AB000626D21F007011143C8F80010EBE7C02860
:101AC00013D0B0F5807F10D001250FE0386840F4C6
:101AD0000030386009E00021201D05F0ADF803E07A
:101AE0000098002105F020F9054685B12E43208895
:101AF000DFF8109340052CD5D4F8A400B0F5800F82
:101B000020D00DDCA0B1B0F5001F0FD115E0D8F842
:101B10000010A26D21F4E0711143C8F80010E6E74F
:101B2000B0F5C00F13D0B0F5000F10D001250FE0B5
:101B3000386840F40030386009E00021201D05F0CD
:101B40007BF803E00098002105F0EEF8054675B13A
:101B50002E43208800052DD5D4F8A800B0F1007FD1
:101B600021D00EDCA8B1B0F1807F10D116E0D9F8F9
:101B70000010D4F8A42021F460011143C9F800102A
:101B8000E7E7B0F1407F13D0B0F1806F10D00125AE
:101B90000FE0386840F40030386009E00021201D73
:101BA00005F04AF803E00098002105F0BDF805466D
:101BB0006DB12E43206880011FD5A06CD8B11028CC
:101BC0000FD0202812D0302815D0012514E0D9F8E4
:101BD0000010D4F8A82021F0E0611143C9F80010EA
:101BE000E8E7386840F40030386004E00221201D46
:101BF00005F022F805466DB12E432088C0042BD590
:101C0000E06DB0F5005F20D00DDCA0B1B0F5805FD5
:101C10000FD115E07A48001F0168A26C21F0300155
:101C200011430160E9E7B0F5405F13D0B0F5804F94
:101C300010D001250FE0386840F40030386009E02A
:101C40000021201D04F0F8FF03E00098002105F0BA
:101C50006BF8054685B12E432088800429D5206E77
:101C6000B0F5403F23D010DC08B3B0F5803F14D06E
:101C7000B0F5003F0FD115E0D8F80010E26D21F467
:101C8000E0411143C8F80010E6E7B0F5802F0ED010
:101C9000B0F5A02F0BD001250AE00121201D04F092
:101CA000CBFF03E00098012105F03EF805468DB119
:101CB0002E43208840042AD5D4F8AC00B0F1405F10
:101CC00023D010DC08B3B0F1805F14D0B0F1005F16
:101CD0000FD115E0D8F80010226E21F4E021114355
:101CE000C8F80010E5E7B0F1804F0ED0B0F1A04F7A
:101CF0000BD001250AE00121201D04F09DFF03E027
:101D00000098012105F010F805466DB12E4320889A
:101D100000041FD5E06ED8B1B0F1805F0ED0B0F1F5
:101D2000005F10D0012514E0D9F80010D4F8AC20E1
:101D300021F0E0411143C9F80010E8E7386840F4A9
:101D40000030386004E00121201D04F075FF0546D5
:101D50006DB12E432068C0011ED5606CD0B1012842
:101D60000ED0022811D0032814D0012513E0D8F892
:101D70000010E26E21F040511143C8F80010E9E76D
:101D8000386840F40030386004E00221201D04F07F
:101D900053FF054675B12E432068DFF86CB0400252
:101DA0005AD51A48016841F480710160FEF758FC69
:101DB00082460EE01248001F0168626C21F00301A8
:101DC00011430160E8E7FEF74BFCA0EB0A00642832
:101DD0003AD80E480068C005F5D5B5BB094818309B
:101DE0000068B4F8B01000F4407001F4407188420B
:101DF00019D00448183001680AE000002C44025849
:101E0000504402585844025810440258004802589E
:101E1000026821F4407142F480320260026822F4C8
:101E2000803202600160D4F8B000B0F5807F22D12A
:101E3000FEF716FC824609E0FEF712FCA0EB0A0151
:101E400041F28830814201D9032504E0FE48006850
:101E50008007F1D57DB12E432078DFF8F0A3C007CD
:101E60003CD0A06F182837D025DC78B3082828D0BC
:101E7000102824D12BE0D4F8B000C0F301210329AD
:101E80000ED0DBF8001021F47C51CBF80010EE48A6
:101E90000168B4F8B020C2F30B0211430160DBE724
:101EA000DBF80020EA4B22F47C5203EA10100243D4
:101EB000CBF80020EBE720280ED028280CD00125F5
:101EC0000BE00121201D04F0B7FE04E004E00098BF
:101ED000012104F029FF05465DB12E4320788007DB
:101EE0001ED5606F062819D2DFE800F0160C111617
:101EF0001616DAF80010A26F21F038011143CAF863
:101F00000010EBE70121201D04F096FE03E000988D
:101F1000012104F009FF054675B100E001252E43BB
:101F2000207840071FD5D4F89000062819D2DFE8A2
:101F300000F0160C11161616DAF80010626F21F078
:101F400007011143CAF80010EAE70121201D04F03F
:101F500073FE03E00098012104F0E6FE05469DB102
:101F600000E001252E43207880062BD5D4F88C0084
:101F7000B0F1405F24D011DC10B3B0F1805F15D018
:101F8000B0F1005F10D116E0D9F80010D4F890201D
:101F900021F007011143C9F80010E4E7B0F1804FC8
:101FA0000ED0B0F1A04F0BD001250AE00021201D7A
:101FB00004F042FE03E00098022104F0B5FE05465D
:101FC0008DB12E43207840062BD5D4F89800B0F57B
:101FD000406F24D011DC10B3B0F5806F15D0B0F590
:101FE000006F10D116E0DAF80010D4F88C2021F040
:101FF000E0411143CAF80010E4E7B0F5805F0ED06D
:10200000B0F5A05F0BD001250AE00021201D04F0EF
:1020100013FE03E00098022104F086FE05468DB110
:102020002E43207800062BD5D4F89C00B0F5C04F85
:1020300024D011DC10B3B0F5005F15D0B0F5804F9F
:1020400010D116E0D9F80010D4F8982021F4E0510E
:102050001143C9F80010E4E7B0F5004F0ED0B0F519
:10206000204F0BD001250AE00021201D04F0E4FDE3
:1020700003E00098022104F057FE054665B32E43A5
:10208000207800070BD5D4F88000B0F5805F2DD004
:10209000DAF8002022F440520243CAF800202078E7
:1020A000C0060BD5D4F89400B0F5807F24D0D9F8C1
:1020B000002022F440720243C9F800202068000387
:1020C0002CD5D4F8A000E8B1B0F5803F1FD0B0F512
:1020D000003F21D0012520E0D9F80010D4F89C2041
:1020E00021F460411143C9F80010C9E700980221AA
:1020F00004F01AFE0643D2E70098022104F014FE11
:102100000643DBE70021201D04F096FD03E0009864
:10211000022104F009FE054685B12E4320684003E4
:1021200022D5D4F88400B0F5801F11D0B0F5001F7F
:1021300013D0B0F5401F15D0012514E0D9F80010D8
:10214000D4F8A02021F440311143C9F80010E5E78C
:10215000386840F40030386004E00098012104F051
:10216000E3FD054655B12E432068C0031CD5E06C45
:1021700070B1B0F5803F10D0012514E0DAF80010FE
:10218000D4F8842021F440111143CAF80010EBE781
:10219000386840F40030386004E00221201D04F06B
:1021A0004BFD0546C5B12E432068800004D500983C
:1021B000022104F0B9FD0643206880031BD5E06FBF
:1021C000B8B1B0F5807F10D0B0F5007F11D0B0F578
:1021D000407F0ED001250DE01C4808380168E26CF4
:1021E00021F4803111430160DEE7386840F40030AB
:1021F000386045B32E432068C00207D5D8F80000E8
:10220000226F20F000401043C8F800002068C00092
:1022100008D5DBF80010D4F8B42021F48041114334
:10222000CBF800102068800207D5D8F80010A26E05
:1022300021F080711143C8F800102068400014D5C7
:10224000DBF8001006E01EE07044025854440258C7
:10225000CFFFFF0021F40041CBF80010DBF80010A5
:10226000D4F8B8201143CBF800102068002806DA13
:102270000A480168226D21F04051114301605EB1AE
:102280000120BDE8F88FDAF80010E26F21F4407108
:102290001143CAF80010AEE70020F2E74C440258A0
:1022A00070B504000D4603D094F82C0010B107E07F
:1022B000012070BD002084F82D00204600F018F8A1
:1022C000022084F82C002068211DFEF7A5FBD4E92C
:1022D00000022946FEF7E0FB0448016841F0004196
:1022E0000160012084F82C00002070BD00400052E5
:1022F000444800B587B0016841F002010160006800
:1023000000F0020005903F482038016841F48051F8
:102310000160006800F4805005903A481438016864
:1023200041F004010160016801F0040105910168B8
:1023300041F008010160016801F0080105910168A0
:1023400041F010010160016801F010010591016880
:1023500041F020010160016801F020010591016850
:1023600041F040010160016801F040010591016800
:1023700041F080010160016801F080010591016870
:1023800041F4807101600068694600F48070059036
:102390000D20009002200190012002900320039064
:1023A0000C2004901848FEF74CF94CF20370009092
:1023B00016486946FEF745F94FF6837000901448B9
:1023C0006946FEF73EF94FF63F0000901148694616
:1023D000FEF737F948F2371000900F486946FEF7CC
:1023E00030F94FF47F4000900C486946FEF729F918
:1023F00040F2FF6000900A486946FEF722F907B0F4
:1024000000BD0000F444025800080258000C0258B5
:10241000001002580014025800180258001C0258FC
:102420000020025810B5044690F82C00022809D06C
:10243000022084F82C002068FEF716FB012084F8A7
:102440002C00002010BD70B5044690F82C000D46FD
:1024500002280CD0022084F82C002068FEF70AFB2A
:102460002868022804D0012084F82C00002070BDC8
:102470000520F9E72DE9F05F04004FF000053DD09D
:10248000DFF8C4812068714E714F4045A36A06D0C1
:10249000B04204D0B84202D0E1680F292ED8E26BD6
:1024A0004FF0010B0BEB521CE26802F10801C90866
:1024B000404501FB0CF105D0B04203D0B84201D039
:1024C00008291BD8404503D0B04201D0B84201D101
:1024D000102913D84FF480094B4512D1404507D03D
:1024E000B04205D0B84203D0206BB0F5702F05D8AC
:1024F000256B05B91504B2EB154F02D90120BDE8D3
:10250000F09F94F881004FF0000A20B9204684F82B
:1025100080A000F09FF8022084F881002068016804
:1025200021F001010160A069B0F1806F09D16068FC
:10253000484506D1A06B20B92068016841F480515C
:102540000160A16AE0690843E16B29430843E1683F
:10255000084321688860616A606BA2690843A16BC7
:10256000114308432169084361690843216A08430C
:1025700061680843E16C0843A1680843A16C084303
:10258000A16D08432168C860A06A484529D1206C24
:1025900001282068016827D021F400410160606CA7
:1025A00001282068016822D021F480410160206860
:1025B000404506D0B04204D0B84202D0B5F5702FE5
:1025C00018D0404503D0B04201D0B84202D1B5F591
:1025D000F81F0FD0016821F4005101602168E06A02
:1025E0000864606850B119E041F40041D6E741F455
:1025F0008041DBE7016841F40051EEE7A06A30B9A1
:102600002068816821F4C05141F400618160206834
:10261000816821F4C06141F4806181602068016DAE
:1026200021F0010101656068400206D52068C1689B
:10263000626D21F000411143C160C4F884A084F8A8
:1026400081B000205BE7000000300140003800400E
:10265000003C0040164800B5B5B0016841F00201E9
:102660000160006800F002003490114808300168F1
:1026700041F480410160006800F4804034904FF4E0
:1026800080500090002017906846FFF7B1F94FF492
:1026900060402F9002203090012031900320329032
:1026A0000520339003482FA9FDF7CBFF35B000BDBF
:1026B000E0440258000402582DE9F84F044690F80F
:1026C00080001F4692460A9D01288B4613D04FF08A
:1026D000010984F88090FDF7C3FF94F88120064635
:1026E0000020012A4FF480010ED062688A4209D18D
:1026F000A2683AB902E00220BDE8F88F94F8812080
:10270000042A01D0022136E0BBF1000F32D0BAF129
:10271000000F2FD077B394F88120042A02D005222D
:1027200084F881208046C4F88400C4F864A0A4F82A
:102730006A70A4F86870C4F85CB0A4F86270A4F879
:10274000607020676067206842686FF30F023A4349
:1027500042602068026842F00102026060688842BC
:1027600004D12068016841F400710160E0680F281D
:1027700040D848E0012184F880000846BCE7B4F85E
:10278000620070B12068416989070AD5E16D096866
:102790000162E06D001DE065B4F86200401EA4F81F
:1027A0006200B4F86A0080B12068416948F208020A
:1027B00011420AD0006B616E0860606E001D606699
:1027C000B4F86A00401EA4F86A00681C12D0FDF735
:1027D00047FF801BA8420DD3204605F081F984F8FD
:1027E0008080D4F8840040F48070C4F8840084F8B9
:1027F0008190EBE0B4F862000028C0D1B4F86A0020
:102800000028BCD1C8E0072849D8BDE0B4F8620070
:10281000F0B12068416989071AD5B4F8621001291E
:102820000BD9E16B49B1E16D09680162E06D001DF2
:10283000E065B4F86200801E08E0E16D098801845B
:10284000E06D801CE065B4F86200401EA4F86200F0
:10285000B4F86A00E0B12068416911F4604F17D004
:102860004169090409D5006B616E0860606E001D46
:102870006066B4F86A00801E08E0008E616E088011
:10288000606E801C6066B4F86A00401EA4F86A009E
:10289000681C04D0FDF7E4FE801BA8429CD2B4F86B
:1028A00062000028B2D1B4F86A000028AED173E00B
:1028B000B4F8620080B32068416989072CD5B4F868
:1028C000621003290CD9E16B402909D9E16D09682F
:1028D0000162E06D001DE065B4F86200001F19E0C0
:1028E000B4F8621001290BD9E16B49B1E16D098897
:1028F0000184E06D801CE065B4F86200801E09E090
:10290000E16D097880F82010E06D401CE065B4F8B6
:102910006200401EA4F86200B4F86A0068B3206840
:10292000416911F4604F28D04169090409D5006B51
:10293000616E0860606E001D6066B4F86A00001F7A
:1029400019E0416901F4C041B1F5005F09D9008E79
:10295000616E0880606E801C6066B4F86A00801E3C
:1029600009E090F83000616E0870606E401C60668F
:10297000B4F86A00401EA4F86A00681C04D0FDF791
:102980006FFE801BA84289D2B4F8620000288FD164
:10299000B4F86A0000288BD1002233460821204673
:1029A000009505F00CF928B1D4F8840040F020001F
:1029B000C4F88400204605F093F884F8808084F8F9
:1029C0008190D4F8840000283FF4D8AE012093E62B
:1029D00070B5040015460E4603D094F8450010B1BA
:1029E00007E0012070BD002084F84400204600F07C
:1029F00021F8206804F10801FDF7A4FFA268314620
:102A00002068FDF7DBFFE36A2946D4E90102FDF700
:102A100079FFA168206850F8212042F0010240F8B7
:102A200021200348016841F000410160002070BD91
:102A3000004000521A4800B587B0016841F4805147
:102A40000160006800F48050059015480C30016862
:102A500041F008010160016801F008010591016879
:102A600041F0100101600068694600F01000059017
:102A70004EF2B370009002200190012002900320DA
:102A800003900C2004900748FDF7DBFD4FF68070A3
:102A9000009005486946FDF7D4FD07B000BD000071
:102AA000D4440258000C02580010025810B504001B
:102AB00003D094F83D0010B107E0012010BD0020C4
:102AC00084F83C00204600F00CF8022084F83D0019
:102AD0002068211D05F0B0F8012084F83D00002099
:102AE00010BD70470168CA6842F00102CA60006800
:102AF000018841F001010180002070477047704754
:102B000090F8791090F87A000843704770B5026821
:102B10000446D0691368916810F00F0F64D0594DC6
:102B200003F490760D40354376D0C50707D0DD0518
:102B300005D501251562E26F42F00102E2678207C6
:102B400008D5CA0706D0256802222A62E26F42F041
:102B50000402E267420708D5CA0706D025680422A6
:102B60002A62E26F42F00202E26702070ED503F02A
:102B7000200201F080552A4352EAC17206D025682E
:102B800008222A62E26F42F00802E267E26F002A3E
:102B90003AD0800608D503F0200001F080510843A8
:102BA00002D0204605F07CF9E06F000703D42068CE
:102BB000806840062AD5204605F064F920688168BF
:102BC00049061ED5816821F040018160606FC0B167
:102BD0002D490165606FFEF7B3FB002814D0606FCC
:102BE000016DBDE870400847850615D503F0200546
:102BF00001F0805635430FD02046BDE8704005F007
:102C00004FB92046FFF77BFF70BD05E02046FFF778
:102C100076FF0020E067F7E7C6024FF020050CD5ED
:102C20004E020AD5E803106284F8795084F87A508D
:102C30002046BDE87040FFF761BF06060AD503F0E5
:102C4000800601F400010E4304D02046BDE8704028
:102C500005F0B6BB41060BD5590609D511682046CB
:102C600021F04001116084F8795000F097F8CBE72B
:102C70000002C9D55800C7D5106820F08040106008
:102C8000C2E7000001000010717E009010B5040042
:102C900003D094F8790010B107E0012010BD0020A6
:102CA00084F878002046FDF7E0FC242084F87900C1
:102CB0002068016821F001010160204605F02CF92F
:102CC0000128EBD0606B10B1204605F03FF820687A
:102CD000416821F4904141602068816821F02A0117
:102CE00081602068016841F0010101602046BDE873
:102CF000104005F08FB890F87A30202B4CD1B9B144
:102D0000B2B190F87830012B46D0012380F87830AA
:102D10004166A0F86820A0F86A20FF228168B1F51A
:102D2000805F07D07F2351B1B1F1805F0CD010E0FC
:102D300001207047016921B940F2FF1107E00169E4
:102D400009BBA0F86C2004E00169E1B13F21A0F8C3
:102D50006C100021C167222280F87A2080F8781058
:102D600001688A6842F001028A6001680A6892007C
:102D70000CD50A6842F480720A600068816841F0EC
:102D80008051816006E0A0F86C30E2E7086840F40A
:102D90009070086000207047022070477047FEE77F
:102DA0001CB504460020009001210190164880883F
:102DB00002040D2004F08EF81449486B019002467D
:102DC00001E04A6B019212F0450FFAD0D00705D00E
:102DD000886B40F00100886301201CBD500705D5B9
:102DE000886B40F00400886303201CBD08690D282F
:102DF00001D010201CBD0648886348690090C0F3CC
:102E00004320207000201CBD3400002400700052BC
:102E1000FF0FE01F1B4870B586B0016841F001014B
:102E20000160016801F001010591016841F00401B0
:102E30000160016801F004010591016841F0800121
:102E40000160006803240025694600F080000590B9
:102E500002200126CDE902040B48CDE90065FDF70B
:102E6000F0FB700303948DE8610008486946FDF7A4
:102E7000E8FB0C20009006486946FDF7E2FB06B02F
:102E800070BD0000E04402580000025800080258DB
:102E9000001C02580E490F4A70B506460888126891
:102EA000002422B13046BDE8704002F0F3BD4D88E9
:102EB00000214543084602F047FC02F0B3FDB1B2E1
:102EC000054801E00180641CAC42FBD370BD0000EA
:102ED0005403002440040024000008602DE9F05F42
:102EE000394C3A4DA071296839B102F0F7FDE88AF2
:102EF0002080288B6080BDE8F09F33492C232A2551
:102F00004FF0F0092B2649F2413A4FF4305E45F27A
:102F1000105B89884FF448774FF4A07845F2103C55
:102F20004FF4F07258B1A4F800805145A4F8029013
:102F300001D0614529D123816581A68139E0A4F8BA
:102F400000905145A4F8028001D0614508D1238149
:102F500061456581A68131D1A4F8008062802DE0B1
:102F6000594508D1A4F808E04FF4285060814FF487
:102F70002C50A08106E0A1F5C85063381ED12381F2
:102F80006681A5812280678018E0594508D1A4F8A0
:102F900008E04FF4285060814FF42C50A08106E0E7
:102FA000A1F5C850633804D123816581A6812780AB
:102FB0006280614502D12280A4F802800020BDE831
:102FC000F05F02F0E5BA000054030024400400243E
:102FD0002DE9F04104463A480D46006820B12046EC
:102FE000BDE8F04102F08EBD364E270A4FEA1528A3
:102FF0003146B0884989A0F51343413B0CD0A0F578
:10300000A643103B08D0A0F5AA43103B11D0A0F571
:10301000C853633B27D04BE0084602F0F7FC384624
:1030200002F0E8FCE0B202F0E5FCB08902F0EEFC50
:1030300038E0084602F0EAFC384602F0DBFC708912
:10304000401C80B202F0E2FCE0B202F0D3FCB08996
:1030500002F0DCFC404602F0CDFCB089401C80B29E
:1030600002F0D4FC21E0B07918B93088001B401E72
:1030700084B2084602F0CAFC270A384602F0BAFCBD
:10308000E0B202F0B7FC384602F0B4FCE0B202F065
:10309000B1FCB08902F0BAFC404602F0ABFCE8B2E9
:1030A00002F0A8FC404602F0A5FCE8B202F0A2FC47
:1030B000054930890880881C0280BDE8F081000045
:1030C0004004002454030024FEFF07602DE9F84368
:1030D0001F46144B804608981B6833B13B4600904E
:1030E000404602F02DFDBDE8F883A2EB0802DFF8B0
:1030F0003890521C0C4696B285B20FE021464046ED
:1031000002F022FB02F08EFC0020494602E00D8016
:10311000401C80B2B042FAD3641CA4B2BC42EDD9C8
:10312000E1E7000040040024000008602DE9F04FB2
:1031300095B002F01DFFFE4D4FF6FF7A49F241397E
:1031400045F21036A5F14C0845F2105441F66317CC
:10315000A88018B102F04AFD02F08DB9F548016867
:1031600041F00201016000680EA900F00200139016
:1031700020200E9001200F90109003201190EE4817
:10318000FDF75FFA02F0A4F9EC491022C8F800102C
:103190004046EB49C8F804100021C8F80810C8F8E8
:1031A0000C10C0E904121202C8F81810C8F81C105C
:1031B000C0E908129200C0E90A129201C8F8301062
:1031C0001120C8E90D12CDE90701552009901520FD
:1031D0000290CDE90001D6486A460D914C3806911F
:1031E00007A9FFF7F5FB3220FDF744FAD32002F0E0
:1031F0000DFC02F099F9A88002F096F9A88002F07F
:1032000093F90AEA00205246A88002F08DF9A988B5
:103210000843A880484546D0D42002F0F7FB02F0CE
:1032200083F9A88002F080F9A88002F07DF902EA13
:103230000020A88002F078F9A9880843A880B0424D
:1032400031D04FF45A4002F0E1FB02F06DF9A88052
:103250004FF45B4002F0DAFB02F066F902EA00206C
:10326000A8804FF45C4002F0D1FB02F05DF9A98820
:103270000843A880B0F5004F7DD0A04213D0A12014
:1032800002F0C4FB02F050F9A88002F04DF902EA06
:103290000020A88002F048F9A9880843A880A0F57A
:1032A000AE41613968D080B2484566D1CF2002F086
:1032B000ADFB002002F09EFBC12002F09BFB302002
:1032C00002F098FBED2002F0A1FB642002F092FBDB
:1032D000032002F08FFB122002F08CFB812002F011
:1032E00089FBE82002F092FB852002F083FB10208E
:1032F00002F080FB7A2002F07DFBCB2002F086FBFF
:10330000392002F077FB2C2002F074FB002002F041
:1033100071FB342002F06EFB022002F06BFBF72001
:1033200002F074FB202002F065FBEA2002F06EFB45
:10333000002002F05FFB002002F05CFBC02002F0E6
:1033400065FB1B2002F056FBC12002F05FFB012051
:1033500002F050FBC52002F059FB302002F04AFB7E
:10336000302002F047FBC72002F050FBB72002F0EC
:1033700041FB362002E0B4E0B0E0B4E002F046FBEE
:10338000482002F037FB3A2002F040FB552002F0C3
:1033900031FBB12002F03AFB002002F02BFB1A2097
:1033A00002F028FBB62002F031FB0A2002F022FBDB
:1033B000A22002F01FFBF22002F028FB002002F006
:1033C00019FB262002F022FB012002F013FBE02073
:1033D00002F01CFB0F2002F00DFB2A2002F00AFB7A
:1033E000282002F007FB082002F004FB0E2002F068
:1033F00001FB082002F0FEFA542002F0FBFAA9209B
:1034000002F0F8FA432002F0F5FA0A2002F0F2FA8C
:103410000F2002F0EFFA002002F0ECFA002002F098
:10342000E9FA002002F0E6FA002002F0E3FAE120D7
:1034300002F0ECFA002002F0DDFA152002F0DAFAD0
:10344000172002F0D7FA072002F0D4FA112002F078
:10345000D1FA062002F0CEFA2B2002F0CBFA562049
:1034600002F0C8FA3C2002F0C5FA052002F0C2FAC8
:10347000102002F0BFFA0F2002F0BCFA3F2002F049
:10348000B9FA3F2002F0B6FA0F2002F0B3FA2B206F
:1034900002F0BCFA002002F0ADFA002002F0AAFA15
:1034A000012002F0A7FA3F2002F0A4FA2A2002F03D
:1034B000ADFA002002F09EFA002002F09BFA0020F4
:1034C00002F098FAEF2002F095FA112002F09EFA2D
:1034D0007820FDF7CFF8292001F010BFAF8001F070
:1034E00012BFAC80FDE3B0427ED1ED2002F08EFA37
:1034F000012002F07FFAFE2002F07CFAEE2002F0BA
:1035000085FADE2002F076FA212002F073FAF1202B
:1035100002F07CFA012002F06DFADF2002F076FA68
:10352000102002F067FAC42002F070FA8F2009E040
:1035300054030024E04402580004025800400052A2
:103540000441005202F056FAC62002F05FFA002051
:1035500002F050FAE22002F04DFAE22002F04AFABC
:10356000E22002F047FABF2002F050FAAA2002F04F
:1035700041FAB02002F04AFA0D2002F03BFA002096
:1035800002F038FA0D2002F035FA002002F032FA8B
:10359000112002F02FFA002002F02CFA192002F07C
:1035A00029FA002002F026FA212002F023FA002056
:1035B00002F020FA2D2002F01DFA002002F01AFA83
:1035C0003D2002F017FA002002F014FA5D2002F00C
:1035D00011FA002002F00EFA5D2002F00BFA002032
:1035E00002F008FAB12000E0FEE302F00FFA8020BA
:1035F00002F000FA002002F0FDF98B2002F0FAF947
:10360000002002F0F7F9962002F0F4F9002002F011
:10361000F1F9B22002F0FAF9002002F0EBF90020F3
:1036200002F0E8F9022002F0E5F9002002F0E2F9E8
:10363000032002F0DFF9002002F0DCF9B32002F0F1
:10364000E5F9002002F0D6F9002002F0D3F90020BD
:1036500002F0D0F9002002F0CDF9002002F0CAF902
:10366000002002F0C7F9002002F0C4F9002002F0A7
:10367000C1F9002002F0BEF9002002F0BBF90020E1
:1036800002F0B8F9002002F0B5F9002002F0B2F91A
:10369000002002F0AFF9002002F0ACF9002002F0A7
:1036A000A9F9002002F0A6F9002002F0A3F90020F9
:1036B00002F0A0F9002002F09DF9002002F09AF932
:1036C000002002F097F9002002F094F9002002F0A7
:1036D00091F9B42002F09AF98B2002F08BF90020C6
:1036E00002F088F9962002F085F9002002F082F9B4
:1036F000A12002F07FF9002002F07CF9B52002F051
:1037000085F9022002F076F9002002F073F9032017
:1037100002F070F9002002F06DF9042002F06AF95D
:10372000002002F067F9B62002F070F9002002F0E4
:1037300061F9002002F05EF9B72002F067F900207D
:1037400002F058F9002002F055F93F2002F052F93A
:10375000002002F04FF95E2002F04CF9002002F048
:1037600049F9642002F046F9002002F043F98C2068
:1037700002F040F9002002F03DF9AC2002F03AF9E5
:10378000002002F037F9DC2002F034F9002002F0CA
:1037900031F9702002F02EF9002002F02BF9902070
:1037A00002F028F9002002F025F9EB2002F022F9BE
:1037B000002002F01FF9DC2002F01CF9002002F0CA
:1037C00019F9B82002F022F9002002F013F90020C4
:1037D00002F010F9002002F00DF9002002F00AF9C1
:1037E000002002F007F9002002F004F9002002F0A6
:1037F00001F9002002F0FEF8BA2002F007F92420B7
:1038000002F0F8F8002002F0F5F8002002F0F2F8DB
:10381000002002F0EFF8C12002F0F8F8202002F0BA
:10382000E9F8002002F0E6F8542002F0E3F8002066
:1038300002F0E0F8FF2002F0DDF8002002F0DAF8F4
:10384000C22002F0E3F80A2002F0D4F8002002F0CF
:10385000D1F8042002F0CEF8002002F0CBF8C3200B
:1038600002F0D4F83C2002F0C5F8002002F0C2F8C3
:103870003A2002F0BFF8002002F0BCF8392002F034
:10388000B9F8002002F0B6F8372002F0B3F80020B3
:1038900002F0B0F83C2002F0ADF8002002F0AAF8E7
:1038A000362002F0A7F8002002F0A4F8322002F03F
:1038B000A1F8002002F09EF82F2002F09BF80020D3
:1038C00002F098F82C2002F095F8002002F092F80F
:1038D000292002F08FF8002002F08CF8262002F058
:1038E00089F8002002F086F8242002F083F80020F6
:1038F00002F080F8242002F07DF8002002F07AF82F
:10390000232002F077F8002002F074F83C2002F047
:1039100071F8002002F06EF8362002F06BF80020FB
:1039200002F068F8322002F065F8002002F062F838
:103930002F2002F05FF8002002F05CF82C2002F04B
:1039400059F8002002F056F8292002F053F8002020
:1039500002F050F8262002F04DF8002002F04AF85C
:10396000242002F047F8002002F044F8242002F05E
:1039700041F8002002F03EF8232002F03BF800203E
:1039800002F038F8C42002F041F8622002F032F868
:10399000002002F02FF8052002F02CF8002002F0A1
:1039A00029F8842002F026F8002002F023F8F02005
:1039B00002F020F8002002F01DF8182002F01AF89A
:1039C000002002F017F8A42002F014F8002002F002
:1039D00011F8182002F00EF8002002F00BF8502029
:1039E00002F008F8002002F005F80C2002F002F8BE
:1039F000002001F0FFFF172001F0FCFF002001F084
:103A0000F9FF952001F0F6FF002001F0F3FFF3200D
:103A100001F0F0FF002001F0EDFFE62001F0EAFFE9
:103A2000002001F0E7FFC52001F0F0FF322001F097
:103A3000E1FF002001F0DEFF442001F0DBFF002069
:103A400001F0D8FF652001F0D5FF002001F0D2FF82
:103A5000762001F0CFFF002001F0CCFF882001F09C
:103A6000C9FF002001F0C6FFC62001F0CFFF2020D3
:103A700001F0C0FF002001F0BDFF172001F0BAFFE8
:103A8000002001F0B7FF012001F0B4FF002001F099
:103A9000B1FFC72001F0BAFF002001F0ABFF00200A
:103AA00001F0A8FF002001F0A5FF002001F0A2FF17
:103AB000C82001F0ABFF002001F09CFF002001F0C6
:103AC00099FF002001F096FF002001F093FFC9202C
:103AD00001F09CFF002001F08DFF002001F08AFF23
:103AE000002001F087FF002001F084FF002001F09A
:103AF00081FF002001F07EFF002001F07BFF00200D
:103B000001F078FF002001F075FF002001F072FF46
:103B1000002001F06FFF002001F06CFF002001F099
:103B200069FF002001F066FF002001F063FF002024
:103B300001F060FFE02001F069FF162001F05AFF5C
:103B4000002001F057FF1C2001F054FF002001F07D
:103B500051FF212001F04EFF002001F04BFF3620E5
:103B600001F048FF002001F045FF462001F042FF30
:103B7000002001F03FFF522001F03CFF002001F047
:103B800039FF642001F036FF002001F033FF7A2076
:103B900001F030FF002001F02DFF8B2001F02AFF03
:103BA000002001F027FF992001F024FF002001F000
:103BB00021FFA82001F01EFF002001F01BFFB9200B
:103BC00001F018FF002001F015FFC42001F012FFE2
:103BD000002001F00FFFCA2001F00CFF002001F0CF
:103BE00009FFD22001F006FF002001F003FFD920D9
:103BF00001F000FF002001F0FDFEE02001F0FAFEE0
:103C0000002001F0F7FEF32001F0F4FE002001F0A7
:103C1000F1FEE12001F0FAFE162001F0EBFE00209B
:103C200001F0E8FE1C2001F0E5FE002001F0E2FEBC
:103C3000222001F0DFFE002001F0DCFE362001F042
:103C4000D9FE002001F0D6FE452001F0D3FE002071
:103C500001F0D0FE522001F0CDFE002001F0CAFE9E
:103C6000642001F0C7FE002001F0C4FE7A2001F0BC
:103C7000C1FE002001F0BEFE8B2001F0BBFE002043
:103C800001F0B8FE992001F0B5FE002001F0B2FE6F
:103C9000A82001F0AFFE002001F0ACFEB92001F039
:103CA000A9FE002001F0A6FEC42001F0A3FE002022
:103CB00001F0A0FECA2001F09DFE002001F09AFE56
:103CC000D22001F097FE002001F094FED82001F0F0
:103CD00091FE002001F08EFEE02001F08BFE00201E
:103CE00000E08BE301F086FEF32001F083FE00206C
:103CF00001F080FEE22001F089FE052001F07AFE4D
:103D0000002001F077FE0B2001F074FE002001F08E
:103D100071FE1B2001F06EFE002001F06BFE3420CE
:103D200001F068FE002001F065FE442001F062FE13
:103D3000002001F05FFE4F2001F05CFE002001F04A
:103D400059FE612001F056FE002001F053FE79205B
:103D500001F050FE002001F04DFE882001F04AFEE7
:103D6000002001F047FE972001F044FE002001F002
:103D700041FEA62001F03EFE002001F03BFEB720F0
:103D800001F038FE002001F035FEC22001F032FEC5
:103D9000002001F02FFEC72001F02CFE002001F0D2
:103DA00029FED12001F026FE002001F023FED620BE
:103DB00001F020FE002001F01DFEDD2001F01AFEC2
:103DC000002001F017FEF32001F014FE002001F0A6
:103DD00011FEE32001F01AFE052001F00BFE002089
:103DE00001F008FE0A2000E006E301F003FE0020D7
:103DF00001F000FE1C2001F0FDFD002001F0FAFDA5
:103E0000332001F0F7FD002001F0F4FD442001F023
:103E1000F1FD002001F0EEFD502001F0EBFD00204F
:103E200001F0E8FD622001F0E5FD002001F0E2FD77
:103E3000782001F0DFFD002001F0DCFD882001F09A
:103E4000D9FD002001F0D6FD972001F0D3FD002020
:103E500001F0D0FDA62001F0CDFD002001F0CAFD4B
:103E6000B72001F0C7FD002001F0C4FDC22001F021
:103E7000C1FD002001F0BEFDC72001F0BBFD002008
:103E800001F0B8FDD12001F0B5FD002001F0B2FD38
:103E9000D52001F0AFFD002001F0ACFDDD2001F0E8
:103EA000A9FD002001F0A6FDF32001F0A3FD0020F4
:103EB00001F0A0FDE42001F0A9FD012001F09AFD30
:103EC000002001F097FD012001F094FD002001F099
:103ED00091FD022001F08EFD002001F08BFD2A20D3
:103EE00001F088FD002001F085FD3C2001F082FDFD
:103EF000002001F07FFD4B2001F07CFD002001F04F
:103F000079FD5D2001F076FD002001F073FD742045
:103F100001F070FD002001F06DFD842001F06AFDCC
:103F2000002001F067FD932001F064FD002001F006
:103F300061FDA22001F05EFD002001F05BFDB320D9
:103F400001F058FD002001F055FDBE2001F052FDAA
:103F5000002001F04FFDC42001F04CFD002001F0D5
:103F600049FDCD2001F046FD002001F043FDD320A6
:103F700001F040FD002001F03DFDDD2001F03AFDA3
:103F8000002001F037FDF32001F034FD002001F0A6
:103F900031FDE52001F03AFD002001F02BFD00206D
:103FA00001F028FD002001F025FD002001F022FD98
:103FB000022001F01FFD002001F01CFD292001F06E
:103FC00019FD002001F016FD3C2001F013FD00203A
:103FD00001F010FD4B2001F00DFD002001F00AFD65
:103FE0005D2001F007FD002001F004FD742001F0C8
:103FF00001FD002001F0FEFC842001F0FBFC00200C
:1040000001F0F8FC932001F0F5FC002001F0F2FC37
:10401000A22001F0EFFC002001F0ECFCB32001F045
:10402000E9FC002001F0E6FCBE2001F0E3FC0020EA
:1040300001F0E0FCC42001F0DDFC002001F0DAFC1E
:10404000CD2001F0D7FC002001F0D4FCD32001F0FA
:10405000D1FC002001F0CEFCDC2001F0CBFC0020E4
:1040600001F0C8FCF32001F0C5FC002001F0C2FC07
:10407000E62001F0CBFC112001F0BCFC002001F097
:10408000B9FC342001F0B6FC002001F0B3FC56204E
:1040900001F0B0FC002001F0ADFC762001F0AAFC9C
:1040A000002001F0A7FC772001F0A4FC002001F023
:1040B000A1FC662001F09EFC002001F09BFC882002
:1040C00001F098FC002001F095FC992001F092FC91
:1040D000002001F08FFCBB2001F08CFC002001F0DF
:1040E00089FC992001F086FC002001F083FC662009
:1040F00001F080FC002001F07DFC552001F07AFCED
:10410000002001F077FC552001F074FC002001F044
:1041100071FC452001F06EFC002001F06BFC432097
:1041200001F068FC002001F065FC442001F062FC15
:10413000002001F05FFCE72001F068FC322001F074
:1041400059FC002001F056FC552001F053FC0020E2
:1041500001F050FC762001F04DFC002001F04AFCFB
:10416000662001F047FC002001F044FC672001F0CC
:1041700041FC002001F03EFC672001F03BFC0020E8
:1041800001F038FC872001F035FC002001F032FC02
:10419000992001F02FFC002001F02CFCBB2001F045
:1041A00029FC002001F026FC992001F023FC0020CE
:1041B00001F020FC772001F01DFC002001F01AFC2A
:1041C000442001F017FC002001F014FC562001F0FF
:1041D00011FC002001F00EFC232001F00BFC00205C
:1041E00001F008FC332001F005FC002001F002FC86
:1041F000452001F0FFFB002001F0FCFBE82001F06E
:1042000005FC002001F0F6FB002001F0F3FB9920F3
:1042100001F0F0FB002001F0EDFB872001F0EAFB4C
:10422000002001F0E7FB882001F0E4FB002001F012
:10423000E1FB772001F0DEFB002001F0DBFB6620D4
:1042400001F0D8FB002001F0D5FB882001F0D2FB63
:10425000002001F0CFFBAA2001F0CCFB002001F0F0
:10426000C9FBBB2001F0C6FB002001F0C3FB992075
:1042700001F0C0FB002001F0BDFB662001F0BAFB9D
:10428000002001F0B7FB552001F0B4FB002001F045
:10429000B1FB552001F0AEFB002001F0ABFB442048
:1042A00001F0A8FB002001F0A5FB442001F0A2FBD7
:1042B000002001F09FFB552001F09CFB002001F045
:1042C00099FBE92001F0A2FBAA2001F093FB00205A
:1042D00001F090FB002001F08DFB002001F08AFB33
:1042E000002001F093FBAA2001F084FBCF2001F015
:1042F0008DFB002001F07EFB002001F07BFB002005
:1043000001F078FB002001F075FB002001F072FB4A
:10431000002001F06FFB002001F06CFB002001F099
:1043200069FB002001F066FB002001F063FB002028
:1043300001F060FB002001F05DFB002001F05AFB62
:10434000002001F057FB002001F054FB002001F099
:1043500051FB002001F04EFBF02001F057FB002044
:1043600001F048FB502001F045FB002001F042FB2A
:10437000002001F03FFB002001F03CFBF32001F0A6
:1043800045FB002001F036FBF92001F03FFB062041
:1043900001F030FB102001F02DFB292001F02AFB59
:1043A000002001F027FB3A2001F030FB552001F0FE
:1043B00021FB112001F02AFB6420FCF75BF9292086
:1043C00001F024FB352001F021FB002001F012FB5D
:1043D000512001F01BFBFF2001F00CFB532001F0EA
:1043E00015FB2C2001F006FB552001F00FFB82206D
:1043F00001F000FB2C20FDE3A0427DD14FF470437F
:104400005521184601F018FB4FF2010BAA2158461E
:1044100001F012FB52214FF2020001F00DFB0821C6
:104420004FF2030001F008FB01214FF2040001F0FC
:1044300003FB0D214FF4304001F0FEFA0D214BF249
:10444000010001F0F9FA0D214BF2020001F0F4FA3B
:1044500034214FF4364001F0EFFA34214BF2016081
:1044600001F0EAFA34214BF2026001F0E5FA0D2185
:104470004FF4314001F0E0FA0D214BF2011001F050
:10448000DBFA0D214BF2021001F0D6FA34214FF481
:10449000374001F0D1FA34214BF2017001F0CCFA2F
:1044A00034214BF2027001F0C7FA00214FF4324080
:1044B00001F0C2FA00214BF2012001F0BDFA002107
:1044C0004BF2022001F0B8FA24214FF4384001F0F9
:1044D000B3FA24214BF6010001F0AEFA24214BF689
:1044E000020001F0A9FA01214FF43F4001F0A4FAC3
:1044F0000F214FF4334000E0FEE301F09DFA0F215D
:104500004BF2013001F098FA0F214BF2023001F02A
:1045100093FA34214FF4394001F08EFA34214BF6EE
:10452000011001F089FA34214BF6021001F084FAEF
:1045300008214FF4354001F07FFA08214BF2015079
:1045400001F07AFA08214BF2025001F075FA0321CA
:104550004FF4424001F070FA24214FF43A4001F048
:104560006BFA24214BF6012001F066FA24214BF668
:10457000022001F061FA00214FF43C4001F05CFAA6
:1045800078214BF6014001F057FA00214BF602402A
:1045900001F052FA00214FF43D4001F04DFA78212C
:1045A0004BF6015001F048FA00214BF6025001F0A1
:1045B00043FA00214FF43E4001F03EFA64214BF6ED
:1045C000016001F039FA00214FF4514001F034FA52
:1045D00033214DF2011001F02FFA00214DF20210AB
:1045E00001F02AFA34214DF2031001F025FA0021DE
:1045F0004DF2041001F020FA3A214DF2051001F0BD
:104600001BFA00214DF2061001F016FA4A214DF274
:10461000071001F011FA00214DF2081001F00CFA18
:104620005C214DF2091001F007FA00214DF20A1049
:1046300001F002FA81214DF20B1001F0FDF9002189
:104640004DF20C1001F0F8F9A6214DF20D1001F019
:10465000F3F900214DF20E1001F0EEF9E5214DF2D3
:104660000F1001F0E9F901214DF2101001F0E4F909
:1046700013214DF2111001F0DFF901214DF212105A
:1046800001F0DAF954214DF2131001F0D5F90121AE
:104690004DF2141001F0D0F982214DF2151001F005
:1046A000CBF901214DF2161001F0C6F9CA214DF2E5
:1046B000171001F0C1F902214DF2181001F0BCF9F8
:1046C00000214DF2191001F0B7F902214DF21A1034
:1046D00001F0B2F901214DF21B1001F0ADF90221F8
:1046E0004DF21C1001F0A8F934214DF21D1001F01B
:1046F000A3F902214DF21E1001F09EF967214DF23F
:104700001F1001F099F902214DF2201001F094F9E7
:1047100084214DF2211001F08FF902214DF2221077
:1047200001F08AF9A4214DF2231001F085F902214C
:104730004DF2241001F080F9B7214DF2251001F05F
:104740007BF902214DF2261001F076F9CF214DF2CE
:10475000271001F071F902214DF2281001F06CF9D7
:10476000DE214DF2291001F067F902214DF22A10E5
:1047700001F062F9F2214DF22B1001F05DF90221F6
:104780004DF22C1001F058F9FE214DF22D1001F0E0
:1047900053F903214DF22E1001F04EF910214DF284
:1047A0002F1001F049F903214DF2301001F044F9C6
:1047B00033214DF2311001F03FF903214DF2321057
:1047C00001F03AF96D214DF2331001F035F9002175
:1047D0004FF4524001F030F933214DF2012001F045
:1047E0002BF900214DF2022001F026F934214DF27F
:1047F000032001F021F900214DF2042001F01CF901
:104800003A214DF2052001F017F900214DF2062062
:1048100001F012F94A214DF2072001F00DF90021B3
:104820004DF2082001F008F95C214DF2092001F059
:1048300003F900214DF20A2001F0FEF881214DF22A
:104840000B2001F0F9F800214DF20C2001F0F4F8F2
:10485000A6214DF20D2001F0EFF800214DF20E20BF
:1048600001F0EAF8E5214DF20F2001F0E5F8012111
:104870004DF2102001F0E0F813214DF2112001F06B
:10488000DBF801214DF2122001F0D6F854214DF24F
:10489000132001F0D1F801214DF2142001F0CCF8E1
:1048A00082214DF2152001F0C7F801214DF21620AA
:1048B00001F0C2F8CA214DF2172001F0BDF8022123
:1048C0004DF2182001F0B8F800214DF2192001F046
:1048D000B3F802214DF21A2001F0AEF801214DF299
:1048E0001B2001F0A9F802214DF21C2001F0A4F8D0
:1048F00034214DF21D2001F09FF802214DF21E20BF
:1049000001F09AF867214DF21F2001F095F802217D
:104910004DF2202001F090F884214DF2212001F089
:104920008BF802214DF2222001F086F8A4214DF2ED
:10493000232001F081F802214DF2242001F07CF8BF
:10494000B7214DF2252001F077F802214DF2262003
:1049500001F072F8CF214DF2272001F06DF802210D
:104960004DF2282001F068F8DE214DF2292001F0F7
:1049700063F802214DF22A2001F05EF8F2214DF297
:104980002B2001F059F802214DF22C2001F054F8AF
:10499000FE214DF22D2001F04FF803214DF22E2083
:1049A00001F04AF810214DF22F2001F045F80321C3
:1049B0004DF2302001F040F833214DF2312001F06A
:1049C0003BF803214DF2322001F036F86D214DF213
:1049D000332001F031F800214FF4534001F02CF85E
:1049E00033214DF2013001F027F800214DF2023061
:1049F00001F022F834214DF2033001F01DF80021BE
:104A00004DF2043001F018F83A214DF2053001F072
:104A100013F800214DF2063001F00EF84A214DF254
:104A2000073001F009F800214DF2083001F004F8D8
:104A30005C214DF2093000F0FFFF00214DF20A30F9
:104A400000F0FAFF81214DF20B3000F0F5FF00215C
:104A50004DF20C3000F0F0FFA6214DF20D3000F0C9
:104A6000EBFF00214DF20E3000F0E6FFE5214DF2A4
:104A70000F3000F0E1FF01214DF2103000F0DCFFBB
:104A800013214DF2113000F0D7FF01214DF2123009
:104A900000F0D2FF54214DF2133000F0CDFF012180
:104AA0004DF2143000F0C8FF82214DF2153000F0B5
:104AB000C3FF01214DF2163000F0BEFFCA214DF2B6
:104AC000173000F0B9FF02214DF2183000F0B4FFAA
:104AD00000214DF2193000F0AFFF02214DF21A30E3
:104AE00000F0AAFF01214DF21B3000F0A5FF0221CA
:104AF0004DF21C3000F0A0FF34214DF21D3000F0CB
:104B00009BFF02214DF21E3000F096FF67214DF20F
:104B10001F3000F091FF02214DF2203000F08CFF99
:104B200084214DF2213000F087FF02214DF2223026
:104B300000F082FFA4214DF2233000F07DFF02211E
:104B40004DF2243000F078FFB7214DF2253000F00F
:104B500073FF02214DF2263000F06EFFCF214DF29F
:104B6000273000F069FF02214DF2283000F064FF89
:104B7000DE214DF2293000F05FFF02214DF22A3094
:104B800000F05AFFF2214DF22B3000F055FF0221C8
:104B90004DF22C3000F050FFFE214DF22D3000F090
:104BA0004BFF03214DF22E3000F046FF10214DF255
:104BB0002F3000F041FF03214DF2303000F03CFF78
:104BC00033214DF2313000F037FF03214DF2323006
:104BD00000F032FF6D214DF2333000F02DFF002147
:104BE0004FF4544000F028FF33214DF2014000F013
:104BF00023FF00E082E300214DF2024000F01CFFA1
:104C000034214DF2034000F017FF00214DF2044023
:104C100000F012FF3A214DF2054000F00DFF002197
:104C20004DF2064000F008FF4A214DF2074000F027
:104C300003FF00214DF2084000F0FEFE5C214DF222
:104C4000094000F0F9FE00214DF20A4000F0F4FEA8
:104C500081214DF20B4000F0EFFE00214DF20C409F
:104C600000F0EAFEA6214DF20D4000F0E5FE002125
:104C70004DF20E4000F0E0FEE5214DF20F4000F055
:104C8000DBFE01214DF2104000F0D6FE13214DF263
:104C9000114000F0D1FE01214DF2124000F0CCFE97
:104CA00054214DF2134000F0C7FE01214DF2144093
:104CB00000F0C2FE82214DF2154000F0BDFE012140
:104CC0004DF2164000F0B8FECA214DF2174000F038
:104CD000B3FE02214DF2184000F0AEFE00214DF26D
:104CE000194000F0A9FE02214DF21A4000F0A4FE86
:104CF00001214DF21B4000E003E300F09DFE022184
:104D00004DF21C4000F098FE34214DF21D4000F0A1
:104D100093FE02214DF21E4000F08EFE67214DF2FF
:104D20001F4000F089FE02214DF2204000F084FE79
:104D300084214DF2214000F07FFE02214DF22240FD
:104D400000F07AFEA4214DF2234000F075FE02210E
:104D50004DF2244000F070FEB7214DF2254000F0E6
:104D60006BFE02214DF2264000F066FECF214DF28F
:104D7000274000F061FE02214DF2284000F05CFE69
:104D8000DE214DF2294000F057FE02214DF22A406B
:104D900000F052FEF2214DF22B4000F04DFE0221B8
:104DA0004DF22C4000F048FEFE214DF22D4000F067
:104DB00043FE03214DF22E4000F03EFE10214DF245
:104DC0002F4000F039FE03214DF2304000F034FE58
:104DD00033214DF2314000F02FFE03214DF23240DD
:104DE00000F02AFE6D214DF2334000F025FE002137
:104DF0004FF4554000F020FE33214DF2015000F0F9
:104E00001BFE00214DF2025000F016FE34214DF23F
:104E1000035000F011FE00214DF2045000F00CFE92
:104E20003A214DF2055000F007FE00214DF20650E8
:104E300000F002FE4A214DF2075000F0FDFD002176
:104E40004DF2085000F0F8FD5C214DF2095000F0E1
:104E5000F3FD00214DF20A5000F0EEFD81214DF2EC
:104E60000B5000F0E9FD00214DF20C5000F0E4FD84
:104E7000A6214DF20D5000F0DFFD00214DF20E5045
:104E800000F0DAFDE5214DF20F5000F0D5FD0121D3
:104E90004DF2105000F0D0FD13214DF2115000F0F2
:104EA000CBFD01214DF2125000F0C6FD54214DF210
:104EB000135000F0C1FD01214DF2145000F0BCFD73
:104EC00082214DF2155000F0B7FD01214DF2165030
:104ED00000F0B2FDCA214DF2175000F0ADFD0221E5
:104EE0004DF2185000F0A8FD00214DF2195000F0CD
:104EF000A3FD02214DF21A5000F09EFD01214DF25A
:104F00001B5000F099FD02214DF21C5000F094FD61
:104F100034214DF21D5000F08FFD02214DF21E5044
:104F200000F08AFD67214DF21F5000F085FD02213F
:104F30004DF2205000F080FD84214DF2215000F010
:104F40007BFD02214DF2225000F076FDA4214DF2AE
:104F5000235000F071FD02214DF2245000F06CFD51
:104F6000B7214DF2255000F067FD02214DF2265089
:104F700000F062FDCF214DF2275000F05DFD0221CF
:104F80004DF2285000F058FDDE214DF2295000F07E
:104F900053FD02214DF22A5000F04EFDF2214DF258
:104FA0002B5000F049FD02214DF22C5000F044FD41
:104FB000FE214DF22D5000F03FFD03214DF22E5009
:104FC00000F03AFD10214DF22F5000F035FD032185
:104FD0004DF2305000F030FD33214DF2315000F0F1
:104FE0002BFD03214DF2325000F026FD6D214DF2D4
:104FF000335000F021FD00214FF4564000F01CFD1D
:1050000033214DF2016000F017FD00214DF20260E6
:1050100000F012FD34214DF2036000F00DFD00217F
:105020004DF2046000F008FD3A214DF2056000F0F9
:1050300003FD00214DF2066000F0FEFC4A214DF216
:10504000076000F0F9FC00214DF2086000F0F4FC6C
:105050005C214DF2096000F0EFFC00214DF20A6086
:1050600000F0EAFC81214DF20B6000F0E5FC00212C
:105070004DF20C6000F0E0FCA6214DF20D6000F056
:10508000DBFC00214DF20E6000F0D6FCE5214DF274
:105090000F6000F0D1FC01214DF2106000F0CCFC5B
:1050A00013214DF2116000F0C7FC01214DF2126096
:1050B00000F0C2FC54214DF2136000F0BDFC012150
:1050C0004DF2146000F0B8FC82214DF2156000F042
:1050D000B3FC01214DF2166000F0AEFCCA214DF286
:1050E000176000F0A9FC02214DF2186000F0A4FC4A
:1050F00000214DF2196000F09FFC02214DF21A6070
:1051000000F09AFC01214DF21B6000F095FC022199
:105110004DF21C6000F090FC34214DF21D6000F057
:105120008BFC02214DF21E6000F086FC67214DF2DF
:105130001F6000F081FC02214DF2206000F07CFC39
:1051400084214DF2216000F077FC02214DF22260B3
:1051500000F072FCA4214DF2236000F06DFC0221EE
:105160004DF2246000F068FCB7214DF2256000F09C
:1051700063FC02214DF2266000F05EFCCF214DF26F
:10518000276000F059FC02214DF2286000F054FC29
:10519000DE214DF2296000F04FFC02214DF22A6021
:1051A00000F04AFCF2214DF22B6000F045FC022198
:1051B0004DF22C6000F040FCFE214DF22D6000F01D
:1051C0003BFC03214DF22E6000F036FC10214DF225
:1051D0002F6000F031FC03214DF2306000F02CFC18
:1051E00033214DF2316000F027FC03214DF2326093
:1051F00000F022FC6D214DF2336000F01DFC5521C2
:10520000184600F019FCAA21584600F015FC52215E
:105210004FF2020000F010FC08214FF2030000F0F2
:105220000BFC00214FF2040000F006FCCC214FF4EF
:10523000314000F001FC00214BF2011000F0FCFBBA
:1052400005214FF4364000F0F7FB70214FF4374052
:1052500000F0F2FB70214BF2017000F0EDFB012138
:105260004FF4384000F0E8FB03214BF6010000F05A
:10527000E3FB03214BF6020000F0DEFB03214BF6BB
:10528000030000F0D9FB02214FF43C4000F0D4FBB6
:1052900000214BF6014000F0CFFB00214BF602400D
:1052A00000F0CAFBD0214FF4494000F0C5FB0221B9
:1052B0004CF6011000F0C0FB50214CF6021000F03B
:1052C000BBFB50214CF6031000F0B6FB50214CF60E
:1052D000041000F0B1FB00214FF4545000F0ACFB7F
:1052E00055214FF4685000F0A7FB4FF4885000F0B0
:1052F0008DFB7820FBF7C3F94FF4245000F086FBB8
:10530000B9E0B842FCD1E22000F080FB1D2000F0A3
:1053100071FB022000F06EFB042000F06BFB6420A8
:10532000FBF7ADF9E02000F071FB012000F062FB1B
:105330000A20FBF79FF9E02000F068FB032000F053
:1053400059FB0C20FBF796F9012000F05FFB0A20C7
:10535000FBF790F9E62000F059FB2F2000F04AFB04
:10536000FF2000F047FBFF2000F044FBB02000F0DE
:105370004DFB202000F03EFB002000F03BFB032013
:1053800000F038FB40F21F3000F034FB012000F049
:1053900031FB40F2DF1000F02DFB002000F02AFB73
:1053A000B42000F033FB042000F024FB40F21F4047
:1053B00000F020FB002000F01DFB2E2000F01AFB67
:1053C000002000F017FB002000F014FB002000F08C
:1053D00011FB002000F00EFBB62000F017FB0220AE
:1053E00000F008FB4FF4037000F004FB002000F015
:1053F00001FB172000F0FEFA152000F0FBFA002058
:1054000000F0F8FA002000F0F5FAF02000F0FEFAC3
:10541000032000F0EFFA292000F0F8FAD02000F085
:10542000F5FA002000F0E6FABE2000F0EFFA0520C1
:1054300000F0E0FAFE2000F0DDFA012000F0DAFAD8
:10544000002000F0D7FA002000F0D4FA002000F08D
:10545000D1FAB82000F0DAFA032000F0CBFA0120EC
:1054600000F0C8FABA2000F0D1FA012000F0C2FA28
:10547000642000F063F8A888484505D0B04203D006
:10548000A04201D0B84209D105200090029069469F
:10549000D8F82C30D8E90102FBF734FAA98808A023
:1054A000FAF7E4FD0020FDF719FD0848012220214C
:1054B000FBF7EAF85046FDF7EDFC15B0BDE8F08FBC
:1054C0004C43442049443A25780D0A000004025810
:1054D0001FB5FBF7DEF8032201218DF800105007FD
:1054E00001901B208DF8080000208DF80C008DF82D
:1054F00009008DF80D008DF80A008DF80E00684641
:105500008DF801208DF80B208DF80F10FBF7C6F8F1
:105510000420FBF7C8F81FBD0346012000E05843F4
:10552000491EC9B2FBD27047034808B50088ADF8E0
:105530000000BDF8000008BD000008600246BE2063
:1055400000B500F063FA052000F054FA00EE102ACE
:105550009FED0D1BB8EE400B20EE010BBCEEC00B17
:1055600010EE100A80B200F045FA012000F042FA75
:10557000FF2000F03FFA002000F03CFA5DF804EB59
:10558000002000F037BA0000666666666666044072
:10559000F0B56C4D002341F663142946AA79898839
:1055A000012A01D01AB11BE0A14202D118E0A142A8
:1055B00016D1082814D2DFE800F00406080A0C0E01
:1055C000101206200CE007200AE0042008E0052065
:1055D00006E0012004E0002002E0032000E00220B9
:1055E00045F21032A1F5134745F21056413F05D060
:1055F000914203D0B14201D0A14277D1082812D202
:10560000DFE800F0110406080A0C0E1080230AE0FF
:10561000402308E0C02306E0202304E0602302E0EA
:10562000A02300E0E023B14202D14FF4585000E043
:105630003620914205D0B14203D0A14201D043F0BF
:105640000803194600F0F8F9AA88A2420AD069882E
:105650009806288802D5884202D303E0884201D9FF
:1056600029806880B242688941D100F0CFF90020DA
:1056700000F0C0F96889401C80B200F0C7F9002032
:1056800000F0B8F96889801C80B200F0BFF9288862
:10569000401EC0F30F2000F0ADF96889C01C80B235
:1056A00000F0B4F92878401EC0B200F0A3F9A88930
:1056B00000F0ACF9002000F09DF9A889401C80B2F0
:1056C00000F0A4F9002000F095F9A889801C80B2B0
:1056D00000F09CF96888401EC0F30F2000F08AF9A2
:1056E000A889C01C80B200F091F922E028E000F007
:1056F0008DF9002000F07EF9002000F07BF9288869
:10570000401EC0F30F2000F075F92878401EC0B28B
:1057100000F070F9A88900F079F9002000F06AF92A
:10572000002000F067F96888401EC0F30F2000F0E9
:1057300061F9A878BDE8F040401EC0B200F05AB947
:10574000F0BD000054030024F0B53F4D060A0C469E
:1057500002462846270AA9884089A1F51343413B00
:1057600028D0A1F5A643103B24D0A1F5C853633B34
:105770002FD0A1F5AA43103B64D100F047F9304681
:1057800000F038F96889401C80B200F03FF9D0B2CF
:1057900000F030F9A88900F039F9384600F02AF90C
:1057A000A889401C80B200F031F9E0B2BDE8F040B9
:1057B00000F020B900F02AF9304600F01BF9D0B211
:1057C00000F018F9A88900F021F9384600F012F924
:1057D000EBE7A97929B300F019F9304600F00AF98E
:1057E000D0B200F007F92888401EC0F30F2000F067
:1057F00001F92878401EC0B200F0FCF8A88900F03A
:1058000005F9384600F0F6F8E0B200F0F3F86888E1
:10581000401EC0F30F2000F0EDF8A878401EC0B283
:10582000C4E72988891A491E8AB200F0EFF80020DF
:1058300000F0E0F8002000F0DDF8100A00F0DAF8DF
:10584000D0B2D9E7F0BD0000540300242DE9F84F91
:105850001F460E4682468B46580700D00120790825
:1058600000EBD700203A10FB01F0002502F0FF0901
:10587000C0B2009047E00C2F10D0102F12D0182F7C
:1058800014D0202F42D1224901EBC9104FF000085B
:10589000445D200610D51F48026811E01E4909EB3F
:1058A000490006E01D4901EB0910EFE71C4909EB2F
:1058B000C90001EB8000E9E70A9828B91548426859
:1058C00031465046FDF784FB6006761C040E1548F1
:1058D000B6B24088B04219D9A6EB0B00B84209D144
:1058E0000AF101005E461FFA80FA0E480188514510
:1058F0000CD906E008F1010000F0FF08B8F1080F2C
:10590000C7D36D1CEDB200988542B4D3BDE8F88FC3
:1059100040D200902000002480BA0090F4BE009095
:10592000E4C40090540300242DE9FF4F81B01D46CC
:105930000027924680463C46DDF838B0B9464FEA2B
:105940005B0627E0281B401EC1B20A20FFF7E4FDDA
:10595000BAFBF0F00A21B0FBF1F201FB120027B90B
:10596000691E8C4201DA48B101275B463030CDF820
:105970000090C2B206FB048080B206E006FB048001
:1059800020225B4680B2CDF800900299FFF75EFFBF
:10599000641CE4B2AC42D5D305B0BDE8F08F2DE96C
:1059A000F84F00F0FF08044610190D461FFA80FA60
:1059B0004FF0000B58191FFA80F9DDE90A7611E063
:1059C000544502D3E819444685B24D450FD23B46B3
:1059D00029462046CDF800B0FFF738FF04EB57000A
:1059E00084B2761C3278A2F120005E28E8D9BDE8A6
:1059F000F88F000001B5BDF80000ADF80000BDF85B
:105A000000000149088008BD0000086001B5BDF82C
:105A10000000ADF80000BDF800000149088008BD95
:105A2000FEFF0760024803490089088070470000B4
:105A300054030024FEFF0760024A1080901C01807E
:105A400070470000FEFF0760104810B586B001687F
:105A500041F002010160006801210D4C00F00200DC
:105A600005900320CDE90001CDE9021069462046EA
:105A7000FAF7E7FD012220461146FAF705FE01225A
:105A800020460221FAF700FE06B010BDE04402589D
:105A90000004025808B500900548018BC08A491ED1
:105AA0008BB2401E82B20021084600F049F808BDC2
:105AB0004004002400B5AFB04FF000530093CDE98F
:105AC000090102200B90CDE90C026846FBF790FF1C
:105AD000002800D001202FB000BD0000084B10B5F9
:105AE0001C465875A1888AB2218889B220B1012844
:105AF00001D1D9821A8310BDDA82198310BD00004A
:105B000040040024F0B50C4F94B2DFF830C03D469D
:105B10007E7D2B68EA692D7D5CF8255026B103FB5C
:105B200001004243AC52F0BD7E68301A401E03FBB8
:105B3000001050432C52F0BD4004002428000024E3
:105B40002DE9F043254E0024DDF81C90757D0DB144
:105B5000054606E077680D46B91A1A463B1A491EF3
:105B60005B1E3068521B96F814C0DFF87480871AE9
:105B700000FB0150F6697F1E58F82CC0BFB206FB2F
:105B800000C51848066846F40006066016484FF43B
:105B900040360660022646630764066826F0010662
:105BA0000660C563591A4FF48033491C03EB024267
:105BB00011434164C0F83890016841F0010101606F
:105BC000420202E0641C944202D241688907F9D57E
:105BD000816841F002018160BDE8F0834004002447
:105BE00028000024D8440258001000522DE9FF5F1D
:105BF00000F0BEF9B84D0123082704460626A0F59B
:105C0000864042384FF4F0723AD0A4F5E0404FF0AD
:105C1000170A84384FF4487140D003204FF08C09A4
:105C2000A4F5E04CBCF1160C4FF4806B4FF4167EDB
:105C300042D0A4F5E048B8F118084FF4A06C47D062
:105C4000A4F50048B8F1160845D0A4F58058B8F17D
:105C5000180843D04AF2010844454FF4407949D12D
:105C600040F25651C5E900198F2129814621298228
:105C7000D521A98168811821E9811C226882ADE0C3
:105C80004FF48870C5E900202B8128206B81A88102
:105C90000520EF81582228826F829FE0C5E900121B
:105CA0002B812E206B81A881D220A5F80EA02882FE
:105CB00016201822688291E0C5E900BE14212981CE
:105CC0006881A020A5F80C90E98128820C2055E07D
:105CD000C5E900C186E0C5E900BE83E0C5E900C1B1
:105CE000A5F80C900A21298210222981E981698274
:105CF000688173E0A4F52048B8F1020816D0A4F535
:105D00002048B8F103081FD0A4F5204CBCF1040CC6
:105D100029D0A4F52040053833D0A4F5204006381A
:105D20003ED0A4F52040073849D05BE0C5E900C16A
:105D300020212981302129825021A9816E810E21C3
:105D4000E9811622688249E0C5E900C9202129813C
:105D50005021A98130212982072169810C21E98103
:105D6000172268823AE0C5E900B988212981182103
:105D70002982A021A9816E811D21E98112226882D8
:105D80002CE04FF45470C5E9000270202881A881EE
:105D9000102028822F226F81A5F80EA06E821DE0B0
:105DA000C5E9001E802028815820A881282028824B
:105DB00004206881A5F80EA028226B820EE04FF423
:105DC0002070C5E90002602028812F823820A88138
:105DD000022068812921E9813E226882A0210520D4
:105DE000FFF768FE3D484FF000082A683D4F3E4BE4
:105DF0000280696841800220E8613948386036488D
:105E0000A838C0E90038C0F80880A4F58053C0F86D
:105E10000C80183BC0F8108002D14FF08053036112
:105E20002C89631E43616B89A3F1010CC0F818C073
:105E3000B5F80CC06444A4F1010CC0F81CC0B5F85E
:105E40000EC06344A3F1010CC0F820C0A2F1010C04
:105E5000A444C0F824C0A1F1010C9C44C0F828C09F
:105E6000B5F810C062442244521EC2626A8A1144CC
:105E70001944491E016380F8368080F8358080F827
:105E800034801548A838FBF7CFFA0720CDE9008603
:105E9000CDE902083968FF230222002000F028F82B
:105EA000A8880022114680B20090288883B210464C
:105EB00000F04CF80020FFF711FE0C4801222021D1
:105EC00085F81480FAF7E0FB04B04FF0FF30BDE82E
:105ED000F05FFFF7DFBD00004004002454030024FE
:105EE000000000C0280000240010005000040258E8
:105EF0002DE9F0438DB0164614AA134D00240DF180
:105F0000240E92E88013009402942A6801926D682E
:105F1000CDE904634FEA08230395CDE906734FEA00
:105F2000092308938EE82600024607488DF8324080
:105F300069468DF83140A8388DF830C0FBF74AFA31
:105F40000DB0BDE8F08300004004002470B51E468B
:105F5000044603460548049DFBF742FB23462A46B8
:105F600031460248BDE87040FBF764BB980300244B
:105F70002B4830B587B0016841F4007101600168B9
:105F800001F400710591016841F4806101600068CD
:105F90006946244C00F48060059040200090002069
:105FA0000190032003902046FAF74BFB1E4D44203E
:105FB000694600902846FAF744FB40212046FAF74C
:105FC00077FB042104462846FAF772FB44EA4004B2
:105FD00028464021FAF76CFB44EA800010F0FF00ED
:105FE0000CD001280DD002280ED003280FD0042891
:105FF00010D0052811D0002007B030BD44F2423047
:10600000FAE747F28400F7E747F21600F4E747F2B1
:106010001800F1E748F21600EEE741F21800EBE74E
:10602000E04402580024025800280258F0B50468E1
:106030008B88E568C5F30B452B441D04882303EBCF
:10604000C213E65806F47046E65004680F68E66826
:10605000C6F30B46761C3E442E43E65003688C89FB
:10606000DD68C5F30A052C4425048C2404EBC21416
:106070001E5906F470461E5103688F68DE68C6F329
:106080000A06761C3E442E431E510468942303EBFB
:10609000C213E55825F00705E55005680C69EC507A
:1060A00091F8313005681F0291F832301C040B7EE4
:1060B0001E069C2303EBC21355F803C04FF0000CDF
:1060C00045F803C091F8305034433D4325430468FC
:1060D000E5500468982303EBC213E55825F0FF054B
:1060E000E55005684C69EC500468A02303EBC2132B
:1060F000E55840F20776B543E550D1E907452C4312
:106100000568EC500468AC2303EBC213E55844F86F
:1061100003C005684C6AEC500B698BB3012B32D07D
:10612000042B32D0022B30D0032B2ED0072B2CD0B7
:1061300001230568B02404EBC2142E5906F0E026B2
:106140002E51D1E90065AD1B0E8D5D435E43ED1D03
:1061500045EA064305682B510468B42303EBC213D8
:10616000E5586FF30A05E5500468C96AE150006814
:10617000842101EBC211425842F001024250F0BDAD
:10618000FFE70423D5E70323D3E70223D1E7000089
:106190002DE9F84F1C46904600230E460A9FADF8A5
:1061A000003068498979B0FBF1F2B6FBF1F1D20712
:1061B000B2EBC17F7ED1DFF890B199468BF80090A9
:1061C000624981F8009081F800900870020A0A7014
:1061D000000C087035208BF80000002000F014FC43
:1061E00020B9012000F010FC050002D00220BDE81B
:1061F000F88F85218BF80010544880F800804FEA12
:10620000182101700670310A0170310C01701E20D6
:1062100000F0E6F8F8054FF0004A12D000F0FCFD5F
:10622000ADF80090504607E014F8011B0170BDF86E
:106230000010491CADF80010BDF80010B942F3D3AE
:1062400070E07E0ADFF8FC904FEA5827DFF8008103
:106250002FE000F0E1FDD8F88000414640F040001A
:10626000C8F880000020ADF800004FF400735246DB
:1062700007E014F8010B1070BDF80000401CADF8E9
:106280000000BDF800009842F3D3D8F8840040061F
:10629000FBD500F0C1FDD8F89420EB1909EB830180
:1062A000CA61D8F8801021F04001C8F880106D1C38
:1062B000EDB200E041E0B542CBD3B9F802101020B6
:1062C00000EB87004A460844ADF80000232000F0A8
:1062D00087F885218BF80010BDF800001B49087075
:1062E000BDF80000000A0870232000F079F80020B3
:1062F000ADF8000002EB870455461C340EE000F0B8
:106300008BFD002014F8011B2970401CC0B204282A
:10631000F8D3BDF80000401CADF80000BDF8000047
:10632000B042ECD310208BF800004FF4AF70FAF7B6
:10633000A6F900F055FB402801D0012057E70020C6
:1063400055E70000A0170024000001800000028033
:10635000004000522DE9F0410C461E498979B0FBFE
:10636000F1F2B4FBF1F1D207B2EBC17F2DD11A4F9C
:1063700000263E70194D2E702E702870010A29706B
:10638000000C287035203870304600F03DFB18B9FD
:10639000012000F039FB10B10220BDE8F08185201A
:1063A00038702E702E702C70200A2870200C2870E7
:1063B0001E2000F015F8102038704FF4AF70FAF777
:1063C0005EF900F00DFB402801D00120E5E7002038
:1063D000E3E70000A0170024000001800000028015
:1063E00001B5009801E0401E00900028FBD108BDD7
:1063F0002DE9F0419046054601200E4600F042F896
:1064000004463146002000F03DF807464146012091
:1064100000F038F806464146002000F033F884EAE0
:10642000070272404240A2F57060FF3805D00AA012
:10643000F9F71CFE0120BDE8F08174400DA0214653
:10644000F9F714FEE108012204F00703685C9A40A2
:10645000504068540020EEE732626974206563633F
:10646000206572726F72206F72206D6F72650D0AF7
:10647000000000006572726F72706F733A25640DD0
:106480000A00000070B505460C46002001260246B1
:1064900002F00101A94208D124FA02F1C90704D08F
:1064A000510806FA01F3184480B2521CD2B2182ADD
:1064B000EED370BD104910B5104A0969914201D15F
:1064C000C00103E00E4A914200D180010D4A6021D3
:1064D00011700D490870030A0B70000C0870D02071
:1064E00010700420FAF7C6F800F07AFA402801D0BC
:1064F000012010BD002010BDA017002489260048EF
:10650000569590DC000001800000028010B588B034
:1065100000F05EF8274904AA254808604FF480700F
:10652000486000208860C86008614FF4003048610E
:106530000A208861C861694600900190029003902A
:1065400004900590069007901A48FBF79DF800F01C
:1065500035FA6420FAF78EF800F07EF8154C014603
:106560004034206114A0F9F781FD042000F056F8B2
:106570004FF48052144B20695110984207D14FF4C8
:1065800087502080E0206280A080802008E00F4BB0
:1065900098420BD14FF40460208061804020A0809D
:1065A000A07100202181628108B010BD0120FBE7AD
:1065B00080400052601700244E414E442049443A26
:1065C0002523780D0A00000089260048569590DCA6
:1065D0001FB5FAF75EF801218DF8001004208DF840
:1065E00001008DF80C100322400701901B208DF84C
:1065F000080000208DF809008DF80D008DF80A00C4
:106600008DF80E008DF80B208DF80F006846FAF714
:1066100045F80420FAF747F81FBD00000C4BEF21A6
:1066200000B50246197001210A4B19702320FFF7AB
:10663000D7FE4FF000410A70002008700870087003
:1066400000F0CEF9402801D0012000BD002000BD9F
:106650000000018000000280154990201CB50870E0
:106660000020144908701E20FFF7BAFE4FF00040CA
:1066700001788DF8001001788DF8011001788DF8FF
:10668000021001788DF8031000788DF80400DDF811
:10669000010000BA20F0FF049DF80400044300F05C
:1066A0009FF9402802D04FF0FF301CBD20461CBD92
:1066B00000000180000002802DE9FC5F1C461546A9
:1066C0008A4683464FF00009ADF80490774AC846E1
:1066D00082F8009076480170090A017080F800B0D5
:1066E0004FEA1B2101704FEA1B41017030201070EE
:1066F000002000F089F920B9012000F085F906009A
:1067000002D00220BDE8FC9FE0054FF000410ED012
:10671000484605E0087805F8010BBDF80400401C68
:10672000ADF80400BDF80400A042F3D3B6E0670A58
:1067300000954FEA5A2431E000F06EFB5D49D1F834
:10674000800040F04000C1F880000020ADF8040057
:106750004A044FF4007307E0107805F8010BBDF808
:106760000400401CADF80400BDF804009842F3D3C7
:106770008946D9F884004006FBD500F04DFBD9F8D6
:10678000942033194C4901EB8301CA61D9F8801078
:1067900021F04001C9F88010761CF6B2BE42CBD37E
:1067A000454E102101EB840170880844ADF80400C7
:1067B0003220FFF715FE3D4805210170BDF8042089
:1067C0003B490A70BDF80420120A0A70E0210170EA
:1067D0001E20FFF705FE06EB84053C3500F01CFB90
:1067E0000021ADF804104FF0004207E0107805F8E2
:1067F000010BBDF80400401CADF80400BDF8040016
:10680000B0EB870FF2D3ADF8041043E0BDF80400FD
:10681000BDF80410204406EB8000C06B214406EB59
:106820008101C969884230D0BDF80400204406EBDC
:106830008000C26BBDF80400204406EB8000C169F3
:106840001EA0F9F713FC23A022463946F9F70EFCE7
:1068500026A052465946F9F709FCBDF80400204429
:1068600006EB8000C269BDF80400BDF80430204486
:1068700006EB8000C16B009800EB4320FFF7B8FDEA
:1068800008B1042000E003208046BDF80400401C4D
:10689000ADF80400BDF80400B842B7D300F0A0F88A
:1068A000402801D04FF0010840462BE7000001804E
:1068B0000000028000400052A01700246572722080
:1068C00068642C72643A307825782C307825780DFD
:1068D0000A0000006563636E756D2C6563637374F5
:1068E0006172743A25642C25640D0A005061676555
:1068F0004E756D2C436F6C4E756D3A25642C256476
:106900000D0A00002DE9F0411D46184B00241646E3
:10691000069F1C70164A1170090A11701070010A46
:106920001170000C107030201870204600F06CF8C8
:1069300018B9012000F068F810B10220BDE8F0811C
:1069400000F06AFA4FF0004004E00168B14203D160
:10695000641CA4B2AC42F8D33C8000F041F840285B
:1069600001D00120EAE70020E8E7000000000180F4
:106970000000028030B4064D2C79641AE4B2A342C0
:1069800000D923466C88214430BC89B2FFF794BEFD
:10699000A017002408B500208DF8000070200649DB
:1069A00008701E20FFF71CFD4FF0004000788DF8A6
:1069B00000009DF8000008BD000001800749FF208D
:1069C00010B508700320F9F755FE00F009F84028CB
:1069D00001D0012010BD002010BD0000000001808A
:1069E00008B5084A00200090FFF7D4FF400606D4FF
:1069F0000098401C00909042F6D3022008BD402031
:106A000008BD0000FFFF010071B583B000240094B1
:106A10008DF804406FF07E450F4E40210098401CD9
:106A200000903046F9F744FE9DF80C10884205D1DD
:106A30009DF80410491C8DF8041001E08DF8044005
:106A40009DF80400022802D9002004B070BD00980F
:106A5000A842E2D30120F8E7000C02582DE9F84FD4
:106A600014461D460022ADF8002080274F4B1646E5
:106A70001F704F4B19700F0A1F701870070A1F7094
:106A8000000C18702320FFF7ABFCE8054FF0004323
:106A90000FD0ADF8002007E014F8010B1870BDF816
:106AA0000000401CADF80000BDF80000A842F3D380
:106AB0006BE06D0ADFF8FC80DFF8FCA04F0A93461C
:106AC00099462EE000F0A8F9D8F88000414640F041
:106AD0004000C8F88000ADF800B04FF400734A469B
:106AE00007E014F8010B1070BDF80000401CADF871
:106AF0000000BDF800009842F3D3D8F884004006A7
:106B0000FBD500F089F9D8F89420F3190AEB83013A
:106B1000CA61D8F8801021F04001C8F88010761CB6
:106B2000F6B2AE42CED3BAF80210102000EB8700C6
:106B300052460844ADF800002320FFF751FC1B48E3
:106B400085210170BDF8001019480170BDF80010D2
:106B5000090A01702320FFF743FC02EB8701ADF81F
:106B600000B01C314A460CE0002011F8013B1370C4
:106B7000401CC0B20428F8D3BDF80000401CADF89A
:106B80000000BDF80000A842EED3084910200870AC
:106B90004FF4AF70F9F773FDFFF722FF402802D0E2
:106BA0000120BDE8F88F0020FBE700000000018015
:106BB0000000028000400052A017002470B5134E60
:106BC00000241D4680233370114B1970090A197077
:106BD0001870010A1970000C18702320FFF700FCD0
:106BE000F00302E00260641CA4B2AC42FAD31020AD
:106BF00030704FF4AF70F9F742FDFFF7F1FE402817
:106C000001D0012070BD002070BD00000000018097
:106C10000000028030B4064D2C79641AE4B2A3421D
:106C200000D923466C88214430BC89B2FFF716BFD7
:106C3000A0170024704770472DE9F047DFF8E48083
:106C400004460F464FF00009D8F80000C043800703
:106C500009D0344D283D286820F080602860F9F77D
:106C6000FFFC064607E00120BDE8F087F9F7F8FCD5
:106C7000801B02284ED828680001F7D4D8F80010ED
:106C8000226821F47C3141EA0231C8F80010207AF0
:106C90004FF4FE02A1884002491EA0F5007080B2A8
:106CA000C1F308010843A189491E02EA01410843D2
:106CB000217C1202491E02EA016108431949103180
:106CC00008601848001D0168626921F0C001114385
:106CD00001600168A26921F02001114301606FB1D8
:106CE0000168012F0ED041F400110160286840F0C6
:106CF00080602860F9F7B4FC04460DE0016841F4B7
:106D00000021F2E741F48011EFE7F9F7A9FC001B3D
:106D1000022801D90320A7E728680001F5D54846D5
:106D2000A2E70000284402582DE9F047DFF8E4808C
:106D300004460F464FF00009D8F80000C043800712
:106D400009D0344D283D286820F080502860F9F79C
:106D500087FC064607E00120BDE8F087F9F780FCD4
:106D6000801B02284ED828688000F7D4D8F800107D
:106D7000228821F07C7141EA0251C8F80010207A83
:106D80004FF4FE02A1884002491EA0F5007080B2B7
:106D9000C1F308010843A189491E02EA01410843E1
:106DA000217C1202491E02EA016108431949183187
:106DB00008601848001D0168626921F440611143B0
:106DC00001600168A26921F40071114301606FB193
:106DD0000168012F0ED041F080710160286840F0F9
:106DE00080502860F9F73CFC04460DE0016841F44E
:106DF0008001F2E741F40001EFE7F9F731FC001BF5
:106E0000022801D90320A7E728688000F5D5484665
:106E1000A2E70000284402580E49002070B508601F
:106E2000BFF34F8F081F006843F6FF740A4DC0F38D
:106E30004E31C0F3C90304EA4112184642EA807693
:106E40002E60401EFAD2491EF5D2BFF34F8FBFF31A
:106E50006F8F70BD84ED00E074EF00E03CB5002161
:106E60000C460091019100B1022413484069800151
:106E700001D50E203CBD114D6946A88880B2FAF7B5
:106E800003FA0028F6D10198400313D5A888012100
:106E90000204372000F01EF83720F9F74DFC0028D7
:106EA000E8D101212246062000F014F80620F9F767
:106EB00043FC3CBD25203CBD007000523400002442
:106EC000034A51686FF309010143516070470000A4
:106ED00000700052044B9A6000F03F0040EA01202D
:106EE00040F48050D86070470070005210B5094CD3
:106EF000606221F07E40A062E06A03F0010120F0B0
:106F0000FF0040EA021040EA410040F00100E06268
:106F100010BD0000007000521548012200B5134951
:106F200087B0202301600021C0E901120822C0E9D6
:106F30000323402343615301C0E906311302036276
:106F40005302C0E90931062102200090CDE9012158
:106F5000CDE903100590694606900548FBF7A0F9B6
:106F6000034800F007F807B000BD000040410052A0
:106F700064030024002301221846114610B500F0D6
:106F800021F84FF4FA70F9F77AFB00230122184632
:106F9000022100F017F8002308221846032100F010
:106FA00011F8012240F222230421002000F00AF807
:106FB000BDE81040024840F2A521FBF733BA0000BB
:106FC000640300241FB5002410B1012802D002E0A0
:106FD000102400E008240748CDE902234FF6FF7291
:106FE000CDE900146946FBF72EFA002800D00120F5
:106FF00004B010BD640300240E4910B504460020FF
:107000000978032906D019B1012901D0022902D13A
:10701000022C01D3272010BDE0B2FFF71FFF00288C
:10702000F9D1054A516821F4404141EA843189B2DD
:10703000516010BD34000024007000522DE9F0476B
:1070400083494FF0000CDFF80CA24FF001090B78D8
:1070500080F856308988A0F85410DAF800100A0E2B
:1070600095090570C2F38305457002F00302827032
:107070000A0CC2700A0A02714171DAF80420110E7A
:107080000C01C2F3074101F00F0844EA1114C48057
:10709000C2F3072180F80880CC094472C1F3801440
:1070A0008472C1F34014C472C1F3001404735446D3
:1070B00080F80DC0A468260EC4F30745C4F3072763
:1070C00033B1012B04D0032B02D0022B30D03EE091
:1070D0008907D2B2090D41EA820141EA96120261A2
:1070E000C6F3C201017506F0070141756909817592
:1070F000C5F38201C175A9074B0F394643EAD11583
:107100000576AD1C09FA05F3DE17521CA2FB0357E6
:107110000CFB037302FB063309FA08F20265A5FBB8
:10712000026703FB027205FB0C22C0E912620EE04B
:107130009106890A41EA062239462A430261521C15
:10714000530BD204C0E912234FF400720265C1F35D
:107150008012427689064A0EE1B242EAD112827664
:1071600001F07F01C176DAF80C20110ECB0903770C
:10717000C1F341134377C1F38203890700F81E3F2F
:107180000B0FC2F3074143EA91134370C1F340135D
:10719000837001F0010180F803C00171C2F307217F
:1071A000CB094371C1F380138371C1F34013C371E1
:1071B000C1F300130372C1F38103437201F00301B1
:1071C0008172C2F34601234AC1724B46103280F8E5
:1071D0000C9011680C0E84730C0CC1F3072545EA62
:1071E000042404820C0651680D0E44EA0544C1F3E0
:1071F000074544EA0524C1F307252C43C0F8124093
:10720000817591680C0EC4750C0CC1F3072524061A
:10721000C9B244EA054444EA0124D16844EA11644D
:10722000C0F81A40847FC1F3074244EA12148477FD
:107230001207C1F3072444EA12520284C1F3460143
:1072400080F8221080F823306046BDE8F087000007
:1072500034000024E8140024374810B586B00168D3
:1072600041F480310160006800F4803005903248BC
:107270000C30016841F004010160016801F0040173
:107280000591016841F00801016000680024694629
:1072900000F0080005904FF4F85000900220CDE96E
:1072A0000104032003900C2004902448F9F7C9F945
:1072B0000420009022486946F9F7C3F92148046088
:1072C00044608460C46044628462C4621E49816315
:1072D000C463002202213120F9F7EFF93120F9F7D8
:1072E000F1F900F09BF8194C030014D100F032F8CA
:1072F000030010D12046FFF7A1FE03000BD1B4F824
:107300005400000400F02CFA030004D10120FFF720
:1073100073FE030003D00E480078032807D194F8C9
:10732000560038B1012805D00420FFF7C9FD06B08A
:10733000184610BD0620F8E7D44402580008025849
:10734000000C025800700052FF0FE01F08150024C7
:107350003400002438B52E4C0120ADF80000206820
:1073600080071ED02B4D287804284ED00022032100
:107370000220FFF7AFFDF9F701FA002812D1616989
:1073800025480160A1694160E1698160216AC160AD
:10739000287840B1012806D0062804D0022802D05F
:1073A0000CE0252038BD002201210320FFF792FDCB
:1073B00003206946F9F71CFA0028F3D1287803283E
:1073C0000AD1BDF80000012102040320FFF782FD6D
:1073D000F9F7D4F90028E5D12878042815D0BDF8AC
:1073E00000000321686002040920FFF773FDF9F72C
:1073F000C5F90028D6D16169074810380160A16934
:107400004160E1698160216AC160002038BD0000EF
:107410000070005234000024F81400242DE9F04FCD
:10742000DFF8F4A000273E463C463D46B9465346A9
:10743000CAF80470FA20FFF743FD03201860002209
:1074400011461046FFF746FDF9F760F928B17F1C99
:10745000FFB24A2FF3D3BDE8F08F01214FF4D5726C
:107460000820FFF737FDF9F7F7F9DFF8B0B020B9DA
:1074700001218BF800104FF08049002201213720B4
:10748000FFF728FD3720F9F757F94FF6FF78D8B105
:10749000234F5646A5B336E0002201213720FFF7DF
:1074A00019FD3720F9F748F90028D4D101213A46CF
:1074B0002920FFF70FFDF9F785F90028CBD1DAF87D
:1074C0001460F50F641C02E0164949EA01070DB982
:1074D0004445E1D3444518D216F0804FBBD0022278
:1074E0008BF80020B7E701213A460846FFF7F2FC87
:1074F000F9F768F90028AED17169CD0F641CC9E7AE
:10750000FFE74445EFD3444501D31B20A3E7032104
:107510008BF800109FE70000007000523400002438
:107520000080FF80000010802DE9F05FDFF874B16B
:107530000021DDE90A97164605464FF0FF34CBF8E7
:107540002C10DFF864A19AF80000022804D1560A32
:107550004FF4007946EAC3564A4601211020FFF74E
:10756000B9FC1020F9F7E8F85FEA000806D00146F8
:107570004EA0F8F77BFD4046BDE8F09F07FB09F100
:10758000012320460922FFF7B1FCDBF80C10D84696
:1075900041F04001CBF80C10012F32464FF00101B1
:1075A0000BD91220FFF796FC1220F9F7C5F8060058
:1075B0000BD043A0F8F75AFD71E01120FFF78AFCC9
:1075C0001120F9F7B9F80600D6D1F9F780F8444947
:1075D00010E0D8F8340000040AD50020D8F8802044
:1075E00045F82020401C0828F8D320350C4601E03F
:1075F000BCB1641ED8F8340010F4957FE9D0D8F8F7
:107600000C0020F04000C8F80C00F9F765F8D8F835
:107610003400000707D5D8F8380040F00800C8F853
:1076200038000420A8E7D8F83400800711D5D8F82E
:10763000380040F00200C8F83800012F07D90022B6
:1076400001210C20FFF746FC0C20F9F775F8022009
:1076500092E7D8F83400800607D5D8F8380040F013
:107660002000C8F83800062086E7D8F83400C005A6
:1076700012D5012F10D99AF8000018B1012801D0B5
:10768000022809D1002201210C20FFF723FC0C2045
:10769000F9F752F80600C5D11248C8F8380030464C
:1076A0006AE70000007000523400002453444D4D3E
:1076B000435F53656E645F436D643D25640D0A004E
:1076C00053445F434D445F524541445F4D554C54D4
:1076D0005F424C4F434B204572726F720D0A00009F
:1076E000FFFF7F00FF0FE01F2DE9FC5F0D461A49E9
:1076F0004FF000080746404692460646097809B111
:10770000EE0D6D02BA074FF4007119D000248346C4
:10771000894612E00120CDE90090600242190F482D
:107720004BEB0603FFF700FF0C4980464A463846FC
:10773000F8F724FE641C07F500775445EAD307E008
:10774000CDE9001A2A4633463846FFF7EDFE80465B
:107750004046BDE8FC9F0000340000246015002472
:1077600001210246072000B5FFF7B4FB5DF804EBEA
:107770000720F8F7E1BF00002DE9F84F90460022FE
:10778000DDE90A97040015468DF8002007FB09FA89
:107790001ED08948C262DFF824B29BF8000002289C
:1077A00005D14FEA58204FF4007940EAC3584A46C1
:1077B00001211020FFF78EFB1020F8F7BDFF0028F5
:1077C00007D1012F2BD907FB09F0B0F1007F02D3BD
:1077D0002620BDE8F88F9BF8000018B1012801D0E1
:1077E000022815D1BBF80400012102043720FFF75D
:1077F00071FB3720F8F7A0FF0028EAD101213A46B3
:107800001720FFF767FB1720F8F796FF0028E0D155
:10781000012142461920FFF75DFB19202BE0BBF840
:107820000400012102040D20FFF754FB0D20F8F79E
:1078300083FF0028CDD1604948694FF0FF360EE044
:10784000BBF804000121761E02040D20FFF742FB65
:107850000D20F8F771FF0028BBD157484069C005DB
:1078600002D4002EECD11DE0E6B1012142461820E1
:10787000FFF730FB1820F8F75FFF0028A9D1461E5C
:1078800007FB09F1002330460922FFF72FFBDFF841
:107890002881D8F80C1041F04001C8F80C10F8F716
:1078A00016FF27E0292094E7D8F8340040041FD5BC
:1078B000AAEB050020280ED281074FEA900100D0E4
:1078C000491C002004E004CCC8F88020401C2D1D79
:1078D0008842F8D309E0002054F82010C8F880103E
:1078E000401C0828F8D3203420356FF0404601E0D2
:1078F000BEB1761ED8F8340010F48D7FD4D0D8F8FD
:107900000C0020F04000C8F80C00F8F7E5FED8F8AD
:107910003400000707D5D8F8380040F00800C8F850
:107920003800042055E7D8F83400800711D5D8F87E
:10793000380040F00200C8F83800012F07D90022B3
:1079400001210C20FFF7C6FA0C20F8F7F5FE022003
:107950003FE7D8F83400C00607D5D8F8380040F023
:107960001000C8F83800052033E7D8F83400C00507
:1079700012D5012F10D99BF8000018B1012801D0B1
:10798000022809D1002201210C20FFF7A3FA0C20C4
:10799000F8F7D2FE002886D10948C8F838006846B2
:1079A000FBF7FEF90028BDD19DF800100729F6D09D
:1079B0000629F4D00DE700000070005234000024C6
:1079C000FF0FE01F2DE9FC5F0D4618490746904662
:1079D000002002460978164609B1EE0D6D02BB077C
:1079E0004FF400711AD00024924689464FF0010BE3
:1079F00010E00F484A463946F8F7C0FC60024219C9
:107A00000B48CDE9009B4AEB0603FFF7B5FE641C6B
:107A100007F500774445ECD3BDE8FC9FCDE900189D
:107A20002A4633463846FFF7A7FEF5E73400002420
:107A30006015002410B5154C072113484FF0007253
:107A400004F1080320604FF480006060002083E8A8
:107A50000700521062619200A261CA07606362650A
:107A60000A07C4E907206062C4E90A012046FAF760
:107A700001FD2068016841F001010160BDE810408E
:107A8000FF2000F005B8000000380040600400242A
:107A900001B582B04FF47A700123009001AA034827
:107AA00002A9FAF709FE9DF804000EBD6004002447
:107AB0000A4A11680B6823F001030B6011688B6898
:107AC00023F0E0438B6011688B6803438B60106880
:107AD000016841F00101016070470000600400246A
:107AE00010B502685169936943F008039361026815
:107AF000936943F0100393610268136823F0010354
:107B000013600268136940F26B34A3431361026887
:107B1000936823F44043936090F88120042A0CD0AA
:107B20008A060AD5D0F8842042F08002C0F884206A
:107B30000268936943F02003936190F88120032A3F
:107B40001DD04A060AD5D0F8842042F00402C0F8BD
:107B500084200268936943F040039361826AB2F51E
:107B6000800F0CD10A060AD5D0F8842042F0020218
:107B7000C0F884200268936943F0800393618A050A
:107B80000AD5D0F8842042F00102C0F884200268AF
:107B9000936943F400739361C9050AD5D0F8841042
:107BA00041F00801C0F8841001688A6942F48072CB
:107BB0008A610021A0F86210A0F86A1010BD2DE9BA
:107BC000F0411E4617460D468046069C0AE0601CA2
:107BD00008D024B1F8F744FD801BA04202D903204D
:107BE000BDE8F081D8F80000406935EA000004D013
:107BF0000020B842EBD00020F2E70120F9E77047FF
:107C0000F8F76FBD10B50A4C2068C068C043C007C4
:107C100009D1084800698047216800204862642033
:107C20002168C862E0606FF001002168086110BD42
:107C3000FC1700247C0000242DE9F04702884FF057
:107C4000804A254C254D264EA042264F264B09D072
:107C5000504507D0A84205D0B04203D0B84201D069
:107C6000984204D122F0700C4A6842EA0C02DFF814
:107C70007CC0DFF87C80A042DFF878900FD05045C0
:107C80000DD0A8420BD0B04209D0B84207D09842DC
:107C900005D0604503D0404501D0484503D122F4CA
:107CA0004075CA682A438D8A22F080022A430280E6
:107CB0008A68C2620A880285A04207D0984205D02D
:107CC000604503D0404501D0484501D1098A01866D
:107CD00001214161BDE8F08700000140000400403F
:107CE00000080040000C004000040140004001403A
:107CF0000044014000480140114A38B504460D4691
:107D0000106840F00400106010680322114600F073
:107D1000040000901E20F8F7D0FC1E20F8F7D2FCDB
:107D2000094A00210748C2E902141161C2E90005AD
:107D30001046FAF7BBFEBDE838400348FAF7D2BE5A
:107D4000E844025800080040FC17002490F8341062
:107D5000C90706D001684A68836B22F400321A43CF
:107D60004A6090F83410890706D501684A68C36BE9
:107D700022F480321A434A6090F83410490706D53D
:107D800001684A68036C22F480221A434A6090F822
:107D90003410090706D501684A68436C22F4004292
:107DA0001A434A6090F83410C90606D501688A68FB
:107DB000836C22F480521A438A6090F8341089064A
:107DC00006D501688A68C36C22F400521A438A609F
:107DD00090F83410490611D501684A68036D22F401
:107DE00080121A434A60016DB1F5801F06D1016807
:107DF0004A68436D22F4C0021A434A6090F8341076
:107E0000090606D501684A68806D22F40022024303
:107E10004A607047F8B500250446C567F8F720FCAE
:107E20000746206800686FF07E46000708D50022EC
:107E30003B464FF400112046009600F0FBFA60B973
:107E40002068006840070AD500223B464FF48001B5
:107E50002046009600F0EEFA08B10320F8BD20207D
:107E600084F8790084F87A00002084F87850F8BD0E
:107E700010B5806B0021A0F86A10A0F86210FAF724
:107E80003EFE10BD01680A6822F490720A60016823
:107E90008A6822F001028A60202180F87A107047F7
:107EA00010B5B0F86C2090F87A300168222B05D01C
:107EB000088B40F008000883022010BD898C83687D
:107EC000B3F5805F01D103696BB11140426E531C61
:107ED00043661170B0F86A10491E0904090CA0F835
:107EE0006A1007D015E0436E11401980416E891C5D
:107EF0004166EFE701680A6822F490720A6001683F
:107F00008A6822F001028A60202180F87A10F8F74E
:107F1000EDFB002010BD00002DE9F04F0446006885
:107F20008025FD4B0021D4F810C087B0A6680F460D
:107F3000D4F81C8046EA0C06D4F814C0A26A4CEAB5
:107F4000080C46EA0C0632430668DFF8D0C306EA9E
:107F50000C061643066020684268E66822F4405228
:107F6000324342602268A0699A4201D0266A3043B7
:107F7000A66AB6F1005F04D1D4E90B6C46EA0C06A0
:107F800030439668DFF898C306EA0C06064396600D
:107F90002068C26A666A22F00F023243C262E14E72
:107FA0002068E14AB04210D1126802F03802182A63
:107FB00074D005DCCAB3082A7AD0102A47D179E0F8
:107FC000202A7BD0282A7CD17AE0D84EB04209D131
:107FD000126802F00702062A73D2DFE802F0536942
:107FE0006B6D6F71D24EB04209D1126802F0070278
:107FF000062A66D2DFE802F0465C5E606264CD4E1F
:10800000B04209D1126802F00702062A59D2DFE80D
:1080100002F0394F51535557C74EB0420BD1126839
:1080200002F00702062A4CD200E00EE0DFE802F080
:108030002A4042444648C14EB04209D1126802F07B
:108040003802182A38D0BBDCB4E74FF0010538E01D
:10805000BB4EB04209D1126802F00702062A30D2A4
:10806000DFE802F01026282A2C2EB64EB0420BD1A3
:10807000126802F00702062A23D2DFE802F0031991
:108080001B1D1F2100251CE098421AD1A64A121D73
:10809000126802F00702062A13D202E00CE007E0A1
:1080A0000CE0DFE802F0030507090B0D022508E0EC
:1080B000042506E0402504E0082502E0102500E044
:1080C0002025DFF864B2A04E9842DFF880A2ABF121
:1080D000540B73D1102D31D006DC022D09D0042DA4
:1080E0000AD0082D2FD111E0202D29D0402D2AD1E2
:1080F00007E0F9F76BFB13E06846F9F77DFB0198A1
:108100000EE003A8F9F7F6FB049809E0DBF800108D
:108110005846890610D50068C0F3C1012AFA01F05B
:10812000002811D06168894601EB410181420AD8DB
:10813000B0EB093F07D808E05046F3E78448F1E781
:108140004FF40040EEE7012733E1102D4FF0000817
:108150004ED006DC022D0FD0042D15D0082D04D1F1
:108160002DE0202D4AD0402D13D00127794AA0F5CB
:108170004071914270D9E6E7F9F728FB626A002363
:10818000414636F812200DE06846F9F735FB0198B4
:1081900003E003A8F9F7AEFB04980023616A36F800
:1081A00011201946F8F748FA62680902030241EA09
:1081B00010615008181841EB080115E032E0DBF8B7
:1081C00000105846890609D500680023C0F3C10194
:1081D0002AFA01F0616A36F8112015E0606A00237E
:1081E00036F8102050460FE00023F8F725FABDE7D7
:1081F000606A002336F81020554805E0606A0023C5
:1082000036F810204FF400400021F8F715FA090263
:10821000020241EA10614FEA590010184A4641EB48
:108220000801E1E7E3694FF4004293424DD1082D84
:1082300023D005DC8DB1012D12D0042D06D112E022
:10824000102D35D0202D3AD0402D11D0012721F00E
:108250000F00C1F3420108435AE0F8F74CFA16E068
:10826000F8F74EFA13E06846F9F7C6FA01980EE0FF
:1082700003A8F9F73FFB049809E0DBF80010584623
:10828000890608D50068C0F3C1012AFA01F0616AC5
:1082900036F8111010E0606A36F81010BAFBF1F0F1
:1082A0004100606801EB5001B1FBF0F081B2CEE714
:1082B000606A36F810102648B0FBF1F0F0E7606A0B
:1082C00036F81000B2FBF0F0EAE7082D4AD00ADCDD
:1082D0000DB3012D43D0042D7FF44DAF6846F9F75F
:1082E0008BFA019809E0102D52D0202D55D0402D49
:1082F000F2D103A8F9F7FEFA0498616A36F8111072
:10830000B0FBF1F1606801EB5001B1FBF0F080B21D
:108310002168C8604DE01FE0000C0058F369FFCFF2
:10832000FFF4FF1100100140544402580044004083
:1083300000480040004C0040005000400014014044
:1083400000780040007C004068BA00900090D003A4
:1083500000093D00FFFC0F00F8F7CDF9CDE7F8F775
:10836000CFF9CAE7DBF80020594692060AD509681A
:10837000C1F3C1022AFA02F1626A36F81220B1FB97
:10838000F2F20FE0616A36F81120BAFBF2F209E06E
:10839000616A36F811200949F1E7616A36F811106F
:1083A000B2FBF1F2616802EB5102B2FBF1F189B26A
:1083B000C16007B03846BDE8F08F000000093D00FD
:1083C00090F87910212901D002207047B0F862108E
:1083D00021B18168B1F5805F13D014E001680A68AB
:1083E000920004D58A6822F400028A6003E00A68D9
:1083F00022F080020A600068016841F040010160DB
:108400000CE0016961B1C16D4A1CC265026809785E
:108410001185B0F86210491EA0F862100020704764
:10842000C16D02680988C1F308011185C16D891CFD
:10843000C165EEE72DE9F0411E4617468846044621
:10844000069D1CE0681C1AD025B1F8F709F9801BBD
:10845000A84214D92068016821F4D0710160206815
:10846000816821F001018160202084F8790084F87E
:108470007A00002084F878000320BDE8F0812068AD
:10848000C16938EA010004D00020B842DAD00020E7
:10849000F3E70120F9E7FEE770B5040300F052F9B5
:1084A00000F0FAF8134E4FF480650022294630465A
:1084B000F8F7EAF82020FFF7EBFA0F480088A0F55C
:1084C0006F41183902D1200EFFF7E2FAC4F30740DA
:1084D000FFF7DEFAC4F30720FFF7DAFAE0B2FFF79E
:1084E000D7FA012229463046F8F7CEF8BDE87040A9
:1084F00000F0D2B800140258300000241E4830B5F5
:1085000087B0016841F02001016000684FF4806489
:108510001A4D694600F02000059001200290CDE937
:108520000040032003902846F8F78BF801222146EB
:108530002846F8F7A9F8FFF77DFAE004FFF7B8FA44
:1085400000F05AF80E490880A0F56F41183911D192
:10855000032000F07DF8C0070CD1002221462846F8
:10856000F8F792F8B720FFF793FA01222146284640
:10857000F8F78AF807B030BDE044025800140258FA
:10858000300000242DE9F041DFF864804FF480676B
:1085900015460C460022064639464046F8F774F860
:1085A0000320FFF775FA13480088A0F56F411839CA
:1085B00002D1200EFFF76CFAC4F30740FFF768FA08
:1085C000C4F30720FFF764FAE0B2FFF761FA002472
:1085D00005E0FF20FFF75CFA3055641CA4B2AC4202
:1085E000F7D339464046BDE8F0410122F8F74CB8D0
:1085F00000140258300000242DE9F041134F0024EC
:108600004FF48066224631463846F8F73DF8902010
:10861000FFF73EFA0020FFF73BFA0020FFF738FA99
:108620000020FFF735FAFF20FFF732FA44EA002571
:10863000FF20FFF72DFA40EA0504314601223846B3
:10864000F8F722F82046BDE8F08100000014025837
:1086500070B5012803D0022803D0032803D00524D5
:1086600002E0352400E015240A4E4FF48065002214
:1086700029463046F8F708F82046FFF709FAFF20A8
:10868000FFF706FA0122044629463046F7F7FCFFB9
:10869000204670BD0014025810B50120FFF7D8FF26
:1086A000C007FAD110BD00002DE9F05FC1F30B0641
:1086B000DFF88C800F0B8A46C6F580548146A242B3
:1086C000154600D81446404639034FF480528B4675
:1086D000FFF758FF002006E0321818F80210FF29B3
:1086E00003D1401C80B2A042F6D3A04221D238462A
:1086F000FFF7D2FE002006E0831919F80020401C85
:1087000080B208F80320A042F6D34FF480525946B5
:10871000404600F02DF8A5420FD0281BA144A244EA
:1087200085B200267F1C4FF48054A542CBD82C463E
:10873000C9E7224651464846EBE7BDE8F09F0000F6
:10874000E804002470B5094D4FF4806400222146EE
:108750002846F7F799FF0620FFF79AF921462846A1
:10876000BDE870400122F7F78FBF000000140258E7
:108770002DE9F04107460E46C8B21546C0F5807493
:10878000A24200D814464FF480782246314638463B
:1087900000F00EF8A54208D0281B27442644444682
:1087A00085B2A542F1D82C46EFE7BDE8F081000084
:1087B0002DE9F04115460C460646FFF7C3FFDFF8EA
:1087C00064804FF48067002239464046F7F75CFF2B
:1087D0000220FFF75DF914480088A0F56F411839B1
:1087E00002D1200EFFF754F9C4F30740FFF750F908
:1087F000C4F30720FFF74CF9E0B2FFF749F9002472
:1088000004E0305DFFF744F9641CA4B2AC42F8D335
:10881000012239464046F7F737FFBDE8F041FFF740
:108820003BBF0000001402583000002430380A28F2
:1088300001D201207047002070472DE9F047891EC2
:108840000746006B4FF0010AC1F3C805984600EBDC
:108850001136914601F007010AFA01F0C4B231461F
:10886000761C384601F022FF10B10120BDE8F087E8
:108870004FF400735246791991F8380010EA040C4D
:1088800001D04FF0010CC44501D10220EEE7604059
:1088900081F83800B9F10100FA708146E6D0600035
:1088A00010F0FF04E7D101246D1C9D42E3D30025A5
:1088B000D5E7000010B504460020E070401E60635C
:1088C000204601F0F3FE08B1042010BD04F236206A
:1088D00001F064FEA0F52A41553901D0032010BDF6
:1088E0000B2211A104F1380001F0C5FE40B194F84B
:1088F0003800E92806D0EB2804D0E82802D011E09F
:10890000012010BD03220BA104F16E0001F0B3FEA3
:108910000028F6D0052208A104F18A0001F0ABFE80
:108920000028EED0022010BDEB7690455846415409
:1089300020202000464154004641543332000000BC
:1089400000E0401C02780AB18A42FAD1D0B27047E6
:10895000C269891E921E8A4201D800207047026BAC
:10896000408900FB012070472DE9F04705685FEA68
:10897000010807462BD04146384601F023FD022866
:1089800046D3411C45D0E969814242D84646A86990
:1089900000283ED028784FF0FF3904281ED04645E5
:1089A0005FD1E869741CA04200D8022438462146F1
:1089B00001F008FD01282CD0411C2AD080B3686941
:1089C00002284ED3E96981424BD9064649E06E69D7
:1089D00016B1E869B042DAD80126D8E7012231465B
:1089E000284601F0F2FA040062D0601C60D0012336
:1089F00021461A462846FFF720FF022808D0012802
:108A000009D0B8F1000F08D0F979022909D010E097
:108A10000120BDE8F0874846FBE70221F97143E0F9
:108A20001EE0711C8C423FD0B968711AB9610321F4
:108A3000F97108F101018C4206D1F96909B1491CAB
:108A400000E00221F9612FE0F869012600B9FE611A
:108A500022464146384601F09FFA30BBFE6129E0CC
:108A6000A4B93446E869641CA04202D80224022E4C
:108A70000AD32146384601F0A5FC38B10128C8D0F8
:108A8000411CC6D0B442EDD10020C2E74A4621467F
:108A9000284601F023FF40B9B8F100000AD0224671
:108AA0000146284601F01AFF20B101280FD0012409
:108AB0002046AEE76C61D5E90601891E884201D8DF
:108AC000401EA861287940F001002871F0E74C466B
:108AD000EEE7812803D3FE2801D80120704700204B
:108AE00070472DE9F04106680F460021044600F06A
:108AF0004BF9E8B90025A16B304601F0D7FDB8B9B4
:108B000031780429E16B097803D0E52905D021B13A
:108B100007E041F3C011491C03D06D1CBD420AD0CF
:108B200000E000252046012100F05CF80028E2D09A
:108B3000042800D10720BDE8F0812DE9F0470C465C
:108B4000054601F0A5FFA8BB21462846FFF700FF18
:108B50004FF400770646686305F1380000213A4675
:108B6000814601F09DFD6889BC01B4EB402F02D91C
:108B7000440200E06408BC421DD9204601F072F9AD
:108B80005FEA0008F6D00021224601F089FD670A5D
:108B9000002400E03C446889A04207D96878321973
:108BA0003B46414600F0D7F90028F3D0404601F09B
:108BB0005DF90FE011E00127002400E03C446889E2
:108BC000A04207D9687832193B46494600F0C3F9FC
:108BD0000028F3D06889A04202D00120BDE8F087C8
:108BE0000020FBE72DE9F04707680446066B89463D
:108BF000806B203630B13978042906D04FF400114B
:108C0000B14205D80420BDE8F0874FF08051F7E766
:108C1000F10540D1401CA063616B4FF0000829B101
:108C20007889401E10EA562F05D034E03889B0EB21
:108C3000561F1FD92FE0204601F0C4FB012805462E
:108C40001DD9681C14D0F869A8421ED8B9F1000FCC
:108C500010D0616B2046FFF787FE05000DD0012D77
:108C60000DD0681C04D029463846FFF766FF40B196
:108C70000120C8E7C4F83880C4E70720C3E7022012
:108C8000C1E7E07940F00400E071294638466563A9
:108C9000FFF75EFEA063C6F3080038442663383051
:108CA000E0630020AFE72DE9F04704260768FF25C1
:108CB00089460446A8465EE0384601F0F7FC060007
:108CC0005DD1E16B087898B13A78042A12D0CA7A5B
:108CD000E52802F03F02A27108D02E2806D022F02B
:108CE0002003082B1BD000234B451AD0FF2532E070
:108CF000042644E0B9F1000F02D0832841D02AE0D5
:108D0000852828D1206BE064204601F04CFC060049
:108D100035D13869007900F03F00A07131E00123BE
:108D2000E2E70F2A01D015BB1CE0420606D591F8F8
:108D30000D8000F0BF00226B0546E264A84208D116
:108D40004A7B424505D1F86801F090FD08B16D1EDF
:108D500000E0FF25EDB220460021FFF743FF0600AB
:108D600009D00CE0084601F042FE404509D04FF022
:108D7000FF30E06405E0A16B00299DD10EB1002019
:108D8000A0633046BDE8F0872DE9F041076806464C
:108D90000D463878042806D04FF40010A8423CD97C
:108DA000E8063AD102E04FF08050F7E73563B46847
:108DB00034B93878032807D3FC6A0020F0711CB15D
:108DC00078894FEA402812E03889B0EB551F24D942
:108DD000F86A12E0304601F0F5FA0446401C1AD059
:108DE000022C1AD3F869A04217D9A5EB0805214631
:108DF0004545EFD23846FFF7ABFDC6E90D4060B1FF
:108E000000EB5520B063C5F3080038443830F063F8
:108E10000020BDE8F0810120FBE70220F9E710B552
:108E200020B1012805D0022809D105E0FEF714FA87
:108E300004E0FFF763FB04E0F8F784F808B10120D1
:108E400010BD002010BD000070B54FF40073144633
:108E500028B101281CD002282BD0012070BD39B1C7
:108E6000204A01290BD0022904D003290ED103E0A6
:108E7000002070BD2360FBE7B2F8500024E0D2E987
:108E800012011A460023F7F7CCF829E0042070BD40
:108E90000029EDD0012908D0022904D00329F5D1F9
:108EA00008201080E4E71380E2E74FF448401060A8
:108EB000DEE70029DCD00C4D01296A8808D00229A0
:108EC00004D00329E2D1500A2080D1E72380CFE7E4
:108ED000E889A97948435043C11700EBD1504012AB
:108EE0002060C5E708150024A01700242DE9F041F3
:108EF0001C0015460E4607D048B101284FF40072F9
:108F000011D0022821D11BE00420BDE8F0811A46CF
:108F100002E0FEF7A1F9224629463046FEF7E4FBBF
:108F20000028F6D113E01746304669023A46FFF7AB
:108F300029FB641E05F1010506F50076F4D106E073
:108F400029463046F8F77CF808B10120DDE700201B
:108F5000DBE7002070472DE9F0411C0015460E4666
:108F600007D048B101284FF4007211D0022821D156
:108F70001BE00420BDE8F0811A4602E0FEF76CF920
:108F8000224629463046FEF71DFD0028F6D113E0A3
:108F90001746304669023A46FFF786FB641E05F124
:108FA000010506F50076F4D106E029463046F8F7CB
:108FB000DFF808B10120DDE70020DBE77CB50D46D6
:108FC0001446002101AA0091694600F041F80028EA
:108FD0000AD10199CA694B89921E00995A434B43A1
:108FE00051082960590821607CBD000070B5164DFC
:108FF00000244FF40E760020314601F021FC45F8A4
:10900000240018B1641CE4B2032CF4D34FF4167698
:109010000020314601F014FC0C4D31462860002040
:1090200001F00EFC4FF400716860002001F008FCB4
:10903000032CA86006D1296821B1696811B108B173
:10904000002070BD012070BD481800247401002468
:109050002DE9F7438EB01446002289460EA86946D2
:1090600000F0FCFF070078D1009820600098D0E95C
:109070000616B21E914202D8C9F800106DE00178C0
:109080000024012905D004291AD0D0F82880002511
:109090003BE00225029002A8294601F093F9411C09
:1090A00003D0012803D020B104E001274DE00227BE
:1090B0004BE0641C00986D1CC0698542EBD344E012
:1090C0000025D0F83080B61E00E045B90098414632
:1090D00008F1010801F0EAFA070036D1009A0820E9
:1090E000511991F8381007E0CB0700D1641C4908EA
:1090F000401EA6F1010601D0002EF5D16D1C002EF8
:10910000C5F30805E1D120E03DB90098414608F1DA
:10911000010801F0CBFA070017D100980178284424
:1091200000F13800022904D001F002FA000106D053
:1091300006E001F033FA00B9641CAD1C01E0641CC8
:109140002D1D761EC5F30805DED1C9F80040009834
:109150008461017941F00101017111B03846BDE827
:10916000F08300002DE9FF4F9BB098461BA81446E2
:10917000289E01F0C2F9002803DA0B201FB0BDE8D9
:10918000F08FFE4951F8201009B100220A70C0B2D8
:109190001090FFF744FEC10701D00320EEE740071F
:1091A00001D50A20EAE7109803210BAAFFF74CFE2D
:1091B0004FF4004130B90B9820B1884202D8421ECA
:1091C000104201D001200B904FF400752CB1B4F582
:1091D000007F64D3B4F1807F61D8601E04425ED109
:1091E000B4FBF5F7B8F1000011D0B6FBF5FA044670
:1091F0004FEA4A2BBAF1000F18D01098012108AAA3
:10920000FFF722FEC8B1B8F1000F11D013E08B4672
:1092100003E04FEA5B0BAB4504D3584600F022FE57
:109220000400F6D0BBFBF5FA002CE3D11120A5E732
:10923000204600F01BFE0120A0E71C9800076FEA03
:10924000A010810E08980991884204D3401A089012
:109250008028864607D2B8F1000F02D1204600F0E0
:1092600005FE0E208AE71C98410700F007000ED586
:1092700004284FF0806203D0964501D2802F10D988
:10928000BEF5805F4FF00409E5D3E7B123E0802FFE
:1092900007D9B8F1000F02D1204600F0E7FD1320F6
:1092A0006CE71C99890706D5022802D01C98C007D4
:1092B00004D1032003E01C98C007EAD0022040F646
:1092C000F572814690E20827BEF5002F03D34027B0
:1092D000964500D3BF00099820300690BEFBF7F0FA
:1092E000800008302844401EB0FBF5F106980D912F
:1092F00001440B980144401E491E81430A91B1EB81
:109300005E0FA8D208460999401A1890AEEB0000EB
:10931000B0FBF7F0049010289DD3994988429AD861
:10932000C01DC0080C90401E07FB050107FB05F09F
:109330000390B1FBF0F00A99139007FB0010019025
:1093400000200790064611900F900290059011980A
:1093500040B101282CD00F9880B212900F98304461
:1093600086B22CE0304600F0D3FD80B21290B042BD
:1093700002D0761CB6B224E0012001E00F98401C18
:109380000F90304400900004000C07D0009880B289
:1093900000F0BEFD009989B28842EFD00F98802876
:1093A00004D34FF6FF701290022009E001201190C3
:1093B0000F981296761CB6B2401E0F9001D1002075
:1093C000119002991298C0B26054079902F044FBC0
:1093D000029A014612982244000A507002F03CFBA7
:1093E00007900298801C02900598801C059016B189
:1093F00002985845ABD102982146019A2844401E54
:10940000B0FBF5F0009003461098FFF7A4FD00288C
:109410007FF4F9AEDDE900100844019000200290CD
:10942000002E94D10598401E07FB05010398B1FB5F
:10943000F0F01490012015900A9801900C9828449F
:10944000401EB0FBF5F00390DDE913014618761CD1
:109450005A460021204601F023F90020FF2102E0B6
:109460002154401C083E082E01D35845F8D3012151
:1094700005E0225C0A4349062254090E761E0EB10D
:109480005845F6D303985146504500D908460090F8
:10949000019A034610982146FFF75DFD0028B7D1D9
:1094A000DDE90010084401900398401A0390CFD1E1
:1094B0000698002601900D980E960F9603900021B5
:1094C0005A46204601F0ECF8002002900E98F8B9B8
:1094D0006FF00701204601F07EFA201D4FF0FF31AA
:1094E00001F079FA0820029002200E9010E0012E7F
:1094F00002D90E99491C01E04FF0FF31204401F0E0
:109500006AFA0298001D02900E98401C0E90761E7A
:109510001EB102985845EAD308E00F98032808D2F4
:1095200013A951F82060401C0F9016B102985845BD
:10953000EED303985146504500D908460090019A51
:10954000034610982146FFF706FD0028A7D1DDE964
:109550000010084401900398401A0390AFD10021F5
:109560005A46204601F09CF883202070812084F820
:109570002000022104F1340004E000003C18002423
:10958000FDFFFF7F01F027FA0C9904F1380001F08C
:1095900022FA822084F84000079904F1440001F087
:1095A0001AFA139904F154000E90891C01F013FA71
:1095B000059904F15800199001F00DFADDE9130145
:1095C0003E4601440A9807FB01000190564550466B
:1095D00000D83046019A8346034610982146FFF78B
:1095E000BAFC0028B2D100212A46204601F058F8E2
:1095F0000198B6EB0B0658440190E7D1002000908B
:10960000DDF824A004F1400006991290083017906C
:10961000A1EB0A00019004F1500002900C3005907B
:10962000001D0A90001D0690001D039000212A468F
:10963000204601F035F80B222046FEA101F027F864
:109640000999129801F0C7F90899179801F0C3F920
:10965000DDE9011001F0BFF9DDE90D1001F0BBF902
:10966000DDE9181001F0B7F9DDE9041001F0B3F9F4
:10967000DDE9130101440A98891C01F0ACF900F0FE
:109680003AFF0146069801F0A6F903984FF480715D
:1096900001F0A9F90022284684F86C2004E094F82F
:1096A0006C10491C84F86C104008F8D13E4684F8D0
:1096B0006D2004E094F86D00401C84F86D0076087D
:1096C000F8D1012084F86E0080204FF6EB6184F819
:1096D0006F0004F1780001F086F94AF6552B04F585
:1096E000FF70594601F07FF9002007900BE06A2EC9
:1096F00008D06B2E06D0702E04D0A05D079902F022
:10970000ABF90790761CAE42F1D352461098561C26
:1097100021460123FFF71FFC00287FF474AD0021D0
:109720002A46204600F0BCFF60195946801E01F011
:109730005AF94FF0010A4FF0000B07E014F80B0044
:109740000BF1010B079902F087F90790AB45F5D3B0
:109750001098012332462146761CFFF7FCFB0028B7
:10976000DBD10AF1010ABAF1090FE4D300212A463C
:10977000204600F095FF16E0834607E014F80B0042
:109780000BF1010B079902F067F90790AB45F5D390
:109790001098012332462146761CFFF7DCFB002897
:1097A000BBD10AF1010A4FF00000BAF10B0FE3D36D
:1097B00006E0079904EB0A0001F00DF90AF1040034
:1097C000A8428246F5D31098012306F1010A3246D9
:1097D0002146FFF7C0FB00289FD10098401C009055
:1097E0000228FFF423AFECE1B9F1030F3E4601D0AC
:1097F0002EB334E06EB90020DFF844C201264FEAF0
:109800005E4301E07600401C3CF8101009B199421B
:10981000F8D9BEFBF6F005EB8001C91DB1FBF5F1EF
:109820000D9120210A91002101914FF6F571884296
:109830007FF611AD834988423FF60DAD2AE0DFF88F
:1098400000C2002001264FEA1E33ACF10E0C01E0ED
:109850007600401C3CF8101009B19942F8D9BEFBC3
:10986000F6F0904203D9042101EB400007E0032108
:109870004FF0010900EB4000401C01EB5000284470
:10988000401EB0FBF5F00D9001200A908003B0FB64
:10989000F5F00190DDE9090108440D9906900144B5
:1098A000019801440B980B18401E5B1E8343581A05
:1098B000B9F1030F1CD00D9B18440D90099801EBD2
:1098C0000611091A7145B7D80A990D98AEEB010136
:1098D000091A0198081AB0FBF6F0B9F1030F0490C9
:1098E0000DD0B9F1020F16D0B9F1010F2DD02FE034
:1098F0000A9B03440A93069B18440690DEE70498EB
:109900004FF6F571884223D8002F7FF4A4AC770876
:109910007FF4D8AC9FE404984FF6F57188420CD9D7
:109920002FB94020B0EB460F01D377005CE71C98BD
:10993000800704D54FF0030956E7904208D8002F5E
:10994000E8D17700802FF1D985E404989042E1D8DE
:1099500000212A46204600F0A3FE0B2220463AA111
:1099600000F095FE04F10B00294601F03CF8667307
:109970000A9881B204F10E0001F035F8012020743C
:10998000B9F1030F0ED0410204F1110001F02BF8E0
:109990000899B1F5803F07D289B204F1130001F0B4
:1099A00022F805E00021EFE704F1200001F013F8B0
:1099B000F82060753F2104F1180001F014F8FF2130
:1099C00004F11A0001F00FF8099904F11C0001F0EC
:1099D00002F82927B9F1030F46D000F08CFD0146AB
:1099E00004F1270000F0F7FF0D9881B204F1160092
:1099F00000F0F9FF802084F82400132284F82670F8
:109A000014A104F12B0000F042FE4AF6552704F59C
:109A1000FF703946009000F0E6FF099A0123109884
:109A20002146FFF798FA00287FF4EDABB9F1030F58
:109A30003FD070E0EB7690455846415420202000FE
:109A4000EE010190F5FFFF0FEBFE904D53444F5395
:109A5000352E30004E4F204E414D452020202046CF
:109A6000415420202020200000F045FD014604F153
:109A7000430000F0B0FF0D9904F1240000F0ABFFAB
:109A8000022104F12C0000F0A6FF012104F13000B6
:109A900000F0A9FF062104F1320000F0A4FF8020AD
:109AA00084F84000132284F8427075A104F1470045
:109AB000A9E7099A012310982146921DFFF74BFA56
:109AC00000212A46204600F0EBFD7249204600F0B6
:109AD00082FF714904F5F27000F07DFF049904F5EE
:109AE000F470491E00F077FF022104F5F67000F0D3
:109AF00072FF0098394600F076FF099A012310980A
:109B00002146D21DFFF727FA099A01231098214612
:109B1000521CFFF720FA00215A46204600F0C0FDF3
:109B2000DDF818B000200290B9F1030F2CD0B9F184
:109B3000010F38D06FF00701204600F04CFF0D9F59
:109B40005046574500D838460090034610985A466C
:109B50002146FFF700FA00287FF455AB00212A4682
:109B6000204600F09DFD00997F1A8B44E8D10298B1
:109B7000401C0290D8D0B9F1030F00D0019E50468E
:109B8000564512D9074611E06FF00701204600F054
:109B900022FF201D4FF0FF3100F01DFF6FF07041DC
:109BA00004F10800C9E73D49C6E7374610983B462F
:109BB0005A462146FFF7CFF90028CDD1F61BBB440A
:109BC000DDD1B9F1040F08D0B9F1030F07D008981F
:109BD000B0F5803F05D3062607E0072605E00C26F2
:109BE00003E0B9F1020F42D001261C98000733D4DC
:109BF00000212A46204600F053FD04F5FF704AF686
:109C0000552100F0F0FE04F5DF75002001212870D9
:109C10006970A970E8702E71DDE90810084443F6F8
:109C2000C161B0FBF1F0FE216971810841F03F0193
:109C3000A971E87105F10800099900F0CCFE0899B6
:109C400005F10C0000F0C7FE109801230022214608
:109C5000FFF781F90028B0D1002210981146FFF7D4
:109C6000F3F80028A9D1B8F1000F02D004E00426CF
:109C7000BBE7204600F0FAF81FB00020BDE8F08FE7
:109C80004E4F204E414D4520202020464154333236
:109C9000202020005252614172724161F8FFFF00A2
:109CA00017B581B0144602980090684600F025FC74
:109CB000002802DA0B2004B010BD0A4B002253F832
:109CC000201001B10A70019901B10A7043F8201007
:109CD0002CB1002201A902A800F0C0F9EBE7002096
:109CE000E9E700003C180024F1B59CB002221AA953
:109CF0001CA800F0B3F9002863D11A984FF48037FC
:109D000014AE0078042806D00B223046202100F043
:109D1000C7FC00244CE016223046002100F0C0FCB5
:109D200000241DE01CA800F0D6FEB842054609D369
:109D3000681C45D00A2C43D2290C06EB440000F0E5
:109D400052FE641CE5B346482946FEF7F9FDB8BB50
:109D50000B2C35D2A9B206EB440000F044FE641C83
:109D60001C9800782028DDD234E01CA800F0B3FE57
:109D7000B84207D200F0CCF84FF46A7100F0A0F8B6
:109D8000054600E00025DDB135482946C01FFEF735
:109D9000D7FDA8B9FF2D01D90A2000E00B20A04271
:109DA0000ED9FF2D02D9280A3055641C3555641C84
:109DB0001C9800782028D8D29DF85000E52803D1BF
:109DC00006201DB0F0BD641E24B1301910F8010C3E
:109DD0002028F8D01A98009000200146029068468A
:109DE000FEF7D2FF0028ECD101216846FEF75BFFA9
:109DF0000125B8B10428E4D10020002CE1D00121D4
:109E00006846FEF76EFE0028DBD10F982022002165
:109E100000F046FC1A98007804281DD00F990820FD
:109E2000C87204E01A980078042804D064B10F982E
:109E30000B2214A905E00F98162214A944700F985C
:109E4000801C00F024FC02E00F99E52008701A98AD
:109E5000C57000F0D9FDB4E70F9983200870EAE7D8
:109E6000D40101900146002000F0EABC0146002028
:109E700000F0DABCF0B505460020802D01D228465E
:109E8000F0BDB1F56A7FFBD10C4E0023102245F2E4
:109E90002054E11A03EB510136F82170AF4206D08D
:109EA00001D20B4600E00C46521EF2D1F0BD002A52
:109EB000FCD006EB81004088F0BD00008056029087
:109EC000F0B50024802801D284B21DE0B0F5803FB7
:109ED0001AD2B1F56A7F17D10C4D002286B245F235
:109EE00020531021981A02EB500035F82070B74229
:109EF00006D001D2024600E00346491EF2D103E03B
:109F000011B105EB800044882046F0BDFC010190B2
:109F100030B5B0F5803F20D280B2B0F5805F01D27D
:109F20001B4900E01B4931F8022B002A15D0904252
:109F300013D331F8023BDDB21C0A52FA83F3834299
:109F400021D9092C09D2DFE804F005090E101214FA
:109F500016181A00801A31F8100030BD811A01F06D
:109F60000101401A0DE010380BE0203809E03038CC
:109F700007E01A3805E0083003E0503801E0A0F5AA
:109F8000E35080B230BD002CCDD101EB4501CAE7D2
:109F900004AB0390F6AC039070B516460D4604462C
:109FA000C0690FE0012802D92A1A921C00E032464B
:109FB000291A2068491C00F091FC002804D1E069AE
:109FC000401EE0610028EDD170BD2DE9F047064646
:109FD000C0698F1E9146801EB84200D80027002518
:109FE0003C464FF4007AB846306B00EB14313046F3
:109FF00000F05CFB18B14FF0FF30BDE8F0870120A6
:10A00000534604F00702C4F3C8019040F269C0B29D
:10A01000921E06EB010C641C9CF838C00CEA000C84
:10A020004006000E944202D3002419462046BCF19B
:10A03000000F05D00025A046BC4207D10020DCE778
:10A040006D1C4D45F8D108F10200D6E70028E0D19B
:10A050000120491C9942DCD3C6E700002DE9FF5FCF
:10A06000002790460E460F6000F047FA050003D522
:10A070000B2004B0BDE8F09FCC4850F825409CB1BF
:10A08000346008F0FE06207820B16078FEF761FFAA
:10A09000C1070BD02770B846E8B26070FEF7BFFE6C
:10A0A000C10708D00320E4E70C20E2E70EB1400727
:10A0B00004D40020DDE71EB1400701D50A20D8E70F
:10A0C000002520462946FEF7F5FB022820D16E46E2
:10A0D00004EB051090F8FA1100F5FB7019B1083087
:10A0E00000F026FA00E0002046F825006D1C042D43
:10A0F000EED3002756F8275025B129462046FEF713
:10A10000D9FB00E00320022802D37F1C042FF1D3E7
:10A1100004287AD002287AD201284FF0FF3A4FF46F
:10A1200000760CD004F1430000F038FAB0426ED152
:10A1300004F14E0000F032FA002869D084E00B20D0
:10A1400002E0401C402806D2211891F8381000295E
:10A15000F7D040285BD304F1A00000F01FFAB0F55F
:10A16000807F54D194F8A4000127B34607FA00F089
:10A1700058454CD104F1800000F0E5F9C14610EBE0
:10A18000050841EB0906012E41D204F18C0000F0D4
:10A19000CFF9206294F8A600A070012837D194F876
:10A1A000A50087403804000C608130D004F1940091
:10A1B00000F0BEF97E490746884228D8B81C65627F
:10A1C000E06104F1900000F0B3F92844206304F149
:10A1D000880000F0ADF92844A0626189226B7943C0
:10A1E000521849EB0900B8EB020186410FD304F184
:10A1F000980000F09DF90146E0622046FEF7A8FBBA
:10A200000146204600F052FA18B1012031E75FE024
:10A2100016E000255E46601990F83810812904D1B7
:10A220004C3000F085F9022802D02035B542F2D337
:10A23000B54269D0C4F818A00426C4F814A0ADE053
:10A2400004F15C0000F074F9206294F84870A77083
:10A25000012F01D0022F57D1474394F84500608168
:10A26000B0B3411E08424FD104F1490000F096F905
:10A270002081000748D104F14B0000F08FF906005F
:10A2800004D104F1580000F053F9064604F14600E9
:10A2900000F084F9010037D02389C81900EB1312AC
:10A2A000964231D3B01A6689B0FBF6F080B1DFF880
:10A2B00004C10026604500D803264FF6F57C6045B2
:10A2C00000D8022640F6F57C604502D8012601E060
:10A2D0001AE0CEB12944801C2A442263E061032E97
:10A2E000C4E9095112D07BB1022E3944E1621ED07B
:10A2F00000F0010100EB400001EB5000216A00F288
:10A30000FF10B1EB502F14D20D20B2E604F1620021
:10A3100000F044F90028F7D120890028F4D104F195
:10A32000640000F005F9E062E0698000E6E74000C3
:10A33000E4E7C4F818A08020C4F814A0032E20710C
:10A340002CD104F1680000F029F9012826D1691CFC
:10A35000204600F0ABF908BB04F2362084F80480F4
:10A3600000F01CF9A0F52A41553917D104F1380045
:10A3700000F0DEF81049884210D104F5077000F0B3
:10A38000D7F80E49884209D104F5087000F0D0F8DA
:10A39000A06104F5097000F0CBF8606108492670EF
:10A3A0000888401C0880E08083E600003C180024F8
:10A3B000FDFFFF7FF5FFFF0F525261417272416155
:10A3C000700100242DE9F041046802290D4673D381
:10A3D000E169A94270D921784FF0FF36012909D0EF
:10A3E00002292CD0F20D032902EA850736D0042970
:10A3F0007DD141E0A06A05EB550700EB57212046CF
:10A4000000F054F9002873D1C7F3080020447F1CE2
:10A4100090F83880A06A00EB5721204600F046F9FA
:10A4200048BBC7F30800204490F8381048EA0120E0
:10A43000E90701D006095BE0C0F30B0658E0A06A0B
:10A4400000EB1521204600F031F9A0B9E8B204EB89
:10A450004000383000F0A2F8064649E0A06A00EB60
:10A46000D511204600F022F928B93819383000F00B
:10A470005FF820F070463BE0D0E9042352EA030184
:10A4800001D0816809B9C179B1B981686FF0004C18
:10A49000691A521E43F1FF33520A42EAC3526389DA
:10A4A000B2FBF3F3C279022A07D0032A0DD0022AA5
:10A4B0001DD0C06920B90CE019E0994217D801D12C
:10A4C000664615E005F1010612E082698A42F9D874
:10A4D000EFE7A06A00EBD511204600F0E7F838B9A5
:10A4E0003819383000F024F820F0004600E001264A
:10A4F0003046BDE8F0810020704710B504464FF0AB
:10A50000FF302368190010D011F8012B202A0DD339
:10A510003A2AF9D11A78303A092A06D89B1C8B427C
:10A5200003D1032A01DA1046216010BD002010BDBE
:10A53000C178827842EA01214278007842EA01211A
:10A5400040EA0120704710B5C17982790B0E42EACA
:10A5500001211A02437942EA116243EA01211302FE
:10A56000027943EA116342EA01211A02C37842EAFE
:10A57000116243EA01211302827843EA116342EA3D
:10A5800001211B020A0243EA1163417800780A4361
:10A59000190241EA126140EA022010BD41780078B8
:10A5A00040EA012070472DE9F04104460068A16BA4
:10A5B000066900F07BF8002845D1E16B0878852812
:10A5C00040D12022304600F062F870784701A7F1B0
:10A5D00040002037B0F5007F34D800212046FEF738
:10A5E00001FB04282ED000282DD1A16B206800F09B
:10A5F0005DF8002827D1E16B0878C02822D12022FD
:10A6000006F1200000F043F896F823000F212C30CB
:10A61000B0FBF1F0B7EB401F14D340254FF418788E
:10A6200020460021FEF7DEFA04280BD000280AD1CC
:10A63000A16B206800F03AF8002804D1E16B08789B
:10A64000C12802D00220BDE8F081454503D270192F
:10A65000202200F01CF82035BD42E1D3454508D842
:10A66000304601F0DFF90446B01CFFF797FF844243
:10A67000E8D10020E7E710B510F8013B11F8014BD5
:10A680001B1B521E01D0002BF6D0184610BD002A0D
:10A6900005D011F8013B521E00F8013BF9D170477B
:10A6A000C9B2521E00F8011BFBD1704770B50446B9
:10A6B000406B00250E46B0420FD0204600F0E8F96E
:10A6C00005000AD16078012304F138013246FEF713
:10A6D0000DFC08B16E1E01256663284670BD0000A2
:10A6E000134A70B5131893F8383093B1114B53F8DF
:10A6F00020308B421AD90F4B02EB8002183B53F8E3
:10A700002030106AB1FBF3F150F8214000200346DD
:10A7100008E011688847012070BD156A0E18401CBA
:10A7200045F82630A042F8DB002070BD022070BD45
:10A7300080010024E4AD039030B504460748084D7D
:10A74000002150F82400820005EB8400006A00F02C
:10A7500087F80120291981F8380030BDB4AD039085
:10A76000800100242DE9F0411E4E002405460F46CD
:10A77000701990F8380010B93168284688474FF0B2
:10A78000FF326FB3184B53F82510B7FBF1FCB7FB42
:10A79000F1F001FB1C7101B1401C1349183951F84B
:10A7A0002510491E1CD406EB8506376A57F821C0D0
:10A7B000BCF1000F04D0002484420FD1002206E037
:10A7C000641CF9E7346A8F18521C44F8270082424F
:10A7D000F8D353F825004843BDE8F081491EE5D57C
:10A7E0001046F9E780010024CCAD03900C4B002209
:10A7F00010B50C4C114653F8203004EB800005E0F6
:10A80000046A54F8214004B1521C491C8B42F7D809
:10A810004FF47A704243B2FBF3F080B210BD0000F7
:10A82000B4AD039080010024002906D0034A02EB56
:10A8300080029268891AFFF753BF70478001002495
:10A8400010B50446FFF78EFF411C05D0034901EB0C
:10A8500084018968084410BD002010BD80010024D7
:10A8600001E000F8011B521EFBD270472DE9F047B2
:10A870000F46804601F11A00FFF790FE20BB3878A2
:10A880000126DFF854904FF6FF7A20F04000401E7A
:10A89000002500EB800101EBC00419F805003844E5
:10A8A000FFF77CFE36B1FF2C0ED228F81400641C92
:10A8B000064601E0504507D16D1C0D2DEDD33878CB
:10A8C000400607D5FF2C02D30020BDE8F087002109
:10A8D00028F814100120F8E7C00101902DE9F04795
:10A8E0000226174602290D4604466FD3E069A842A6
:10A8F0006CD920784FF00109012806D0022838D001
:10A90000032846D0042861D143E0A16A05EB55082D
:10A91000204601EB5821FFF7C9FE060056D1C8F3C7
:10A92000080020443830E90708F1010804D0017814
:10A93000FAB262F31F1100E03946017084F8039007
:10A940002046A16A01EB5821FFF7B0FE06003DD179
:10A95000C8F3080020443830E90702D0C7F30711D4
:10A9600005E00178C7F3032201F0F0011143017003
:10A970002AE0A06A00EB15212046FFF797FE0600AB
:10A9800024D1E8B2B9B204EB4000383000F02BF823
:10A990001AE0A06A00EBD5112046FFF787FE0600FB
:10A9A00014D140F2FF10217800EA850005193835EE
:10A9B000042905D02846FFF7BBFD67F31B000746B7
:10A9C0002846394600F007F884F803903046BDE881
:10A9D000F087006870470170090A4170090A8170A8
:10A9E000090AC17070470170090A41707047014639
:10A9F00000200B22430803EBC01011F8013B521E4C
:10AA00001844C0B2F6D1704770B5044600F040F863
:10AA1000050036D1207803282CD12079012829D1AE
:10AA2000420204F1380000210646FFF739FE04F225
:10AA300036204AF65521FFF7D6FF13493046FFF777
:10AA4000CAFF124904F50770FFF7C5FFA16904F5B5
:10AA50000870FFF7C0FF616904F50970FFF7BBFFDD
:10AA6000626A01233146521C62636078FEF773FA12
:10AA700000202071002260781146FEF7E5F900B150
:10AA80000125284670BD0000525261417272416139
:10AA900070B50446C078002548B104F138016078EB
:10AAA000626B01230E46FEF756FA10B101252846C7
:10AAB00070BD0020E070A16A606B421A216A8A4270
:10AAC000F5D2A278022AF2D14218607801233146E9
:10AAD000FEF741FAEBE72DE9F0410568064615F867
:10AAE000014B2046FDF7F5FF4FF0FF3760B115F839
:10AAF000010B402814D37E2803D9A0F180017E29C0
:10AB00000ED800EB042084B234B14FF46A712046B1
:10AB1000FFF7B0F9040003D020463560BDE8F081AE
:10AB20003846FBE770B594B0064613AB694611AAE8
:10AB300000F0DCF9002824D11E4C04258DF84000DB
:10AB400014E0206805EBC10113AB12AA405808A914
:10AB500000F0CCF9002814D108A8694600F001FCE7
:10AB600088B19DF84000401C8DF84000207D9DF884
:10AB700040108842E5D8207D9DF8401088420ED1D3
:10AB8000042014B070BD9DF848009DF84410884220
:10AB900001D90220F5E79DF84000A075EBE710A968
:10ABA000304600F057FA0028EBD19DF84000607560
:10ABB0000020E6E77C0000242DE9F0417E4E9AB0AB
:10ABC000B57D307DA8427CD93068042101EBC501F8
:10ABD00019AB18AA405810A900F088F910A977A05D
:10ABE000F5F744FA00240DF1180832E00121308B0A
:10ABF000A140084217D0222172A0F5F737FA20466B
:10AC000000F090FA811924316FA0F5F72FFA222174
:10AC10006CA0F5F72BFA204600F084FA304424307B
:10AC200048F824000BE0204600F07CFA3044416AEA
:10AC300048F82410F07D00B364A0F5F717FA9DF8EA
:10AC40006000401E844202D062A0F5F70FFA641C37
:10AC5000E4B29DF860008442C8D35FA0F5F706FA1D
:10AC600000F0A6FA707D0B2814D2DFE800F0080D82
:10AC700031384048525E6B78890058A0DDE7306873
:10AC800050F83500804704E0306850F835100698D9
:10AC90008847074600F058FA9DF8640001286ED0F6
:10ACA0004FA0F5F7E3F996F8EC0000280DD0D6F8A0
:10ACB000F0000A21B0FBF1F201FB1202B0FBF1F14E
:10ACC00000E002E047A0F5F7D1F91AB0BDE8F08145
:10ACD000306850F83520DDE906019047D9E7306843
:10ACE00006AC50F8353094E807009847D1E7306853
:10ACF00006AF50F8354097E80F00A047C9E70A981B
:10AD000006AF0090306850F8354097E80F00A04734
:10AD1000BFE7DDE90A0106AFCDE90001306850F870
:10AD2000354097E80F00A047B3E70AAB06AF93E8BA
:10AD300007008DE80700306850F8354097E80F00AD
:10AD4000A047A6E70AAC06AF94E80F008DE80F0015
:10AD5000306850F8354097E80F00A04799E70BACF2
:10AD600006AF94E80F0001AC84E80F000A98009049
:10AD7000306850F8354097E80F00A04789E711E0A8
:10AD80000CAC06AF94E80F0002AC84E80F00DDE9DC
:10AD90000A01CDE90001306850F8354097E80F000E
:10ADA000A04776E7F07D394618B116A0F5F75EF9B1
:10ADB00079E717A0FAE700007C0000240D0A25734C
:10ADC0002800000025630000257300003058255836
:10ADD000000000002C00000029000000256C640029
:10ADE0003B0D0A0046756E6374696F6E2052756E76
:10ADF0002054696D653A25642E2531646D730D0A02
:10AE0000000000003D305825583B0D0A00000000AE
:10AE10003D256C753B0D0A00F0B500252E462F46EA
:10AE20002C4603782C2B03D0292B04D01BB103E034
:10AE300014B9012600E00CB317B1222B2AD02AE066
:10AE4000A3F1300CBCF1090F19D92D2B17D02B2BE6
:10AE500015D0A3F1610CBCF1050F10D9A3F1410C81
:10AE6000BCF1050F0BD9582B09D0782B07D0222B1A
:10AE70000CD0202B1ED02C2B1CD0FF270CE05EB951
:10AE8000612B00D3203B01F8013B13E026B90127D9
:10AE90003C460FE0002426B10020087028461770B9
:10AEA000F0BD3CB15C2B02D16D1C401CEDB20378AF
:10AEB00001F8013B6D1C401CEDB2B2E730B5002536
:10AEC00015700AE001F8014B1478401C641CE4B2D0
:10AED00014709C4201D3012030BD0478202C01D095
:10AEE000002CEFD100200D7030BD00002DE9FF4F88
:10AEF0000024984682B089460125A2462746264668
:10AF000002992246EB4615E0202810D002F07F037C
:10AF1000052B0CD202B9802202F07F03042B01D151
:10AF20002A280AD1521C0BF80300D2B201E0852A6C
:10AF300004D0491C08780028E6D16AB102F07F02EB
:10AF4000002042A10BF80200584600F00AFA38B17E
:10AF5000012188F800100022029B4FF0000815E044
:10AF6000002088F80000F6E708F1010000F0FF0873
:10AF700013F8010F202801D02A2807D1184600F025
:10AF80007DF9282802D02A2800D0C246187828281F
:10AF900001D00028E8D10299BAF1000F01D0514444
:10AFA000491C4FF000084346087888B1282804D08F
:10AFB000292806D0222810D011E083B9641CE4B2FD
:10AFC0000DE063B924B1641E14F0FF0402D00DE05B
:10AFD0004FF00108012F27D02FE04BB100234CB1D7
:10AFE0002C280CD0202816D0282814D05AB110E0D4
:10AFF0000123F4E7202815D009F8010B12E0012500
:10B00000521CD2B207E0052E03D20BF80600761CC4
:10B01000F6B26D1CEDB2012C04D1022D02D1032534
:10B020007F1CFFB2491CBFE700200BF8060007A1F8
:10B03000684600F096F900B90027049807700020D0
:10B0400089F8000006B04046BDE8F08F766F69646D
:10B05000000000002DE9F043314D0024B5B08946D1
:10B06000214622466B18491CC9B20A299A76F9D39F
:10B0700002E010F8011F99B101782829F9D1461C86
:10B080004FF0010833AA69463046FFF7C5FE064473
:10B090009DF8CC0040B1012824D0FF2836D10BE028
:10B0A000012035B0BDE8F0839DF8000070B334A9ED
:10B0B000684600F0EBF808B10220F2E7204600F005
:10B0C00031F8284434994162298B08FA04F081430D
:10B0D0002983042029198876641CE4B20A2C15D926
:10B0E0000320DEE7684600F051F9471C204600F0D7
:10B0F00019F841196846243100F03FF9298B08FA04
:10B1000004F00143298328198776E5E73078292858
:10B1100001D00028B6D1002089F80040C1E7000026
:10B120007C0000240246074B0020014610B505E0D4
:10B130005C18491CC9B2A47E2044C0B29142F7D326
:10B1400010BD00007C000024094800680169C94363
:10B15000CA070849D1F8F02004D14FF6FF731A440A
:10B16000C1F8F020406A1044C1F8F00070470000B8
:10B17000FC1700247C00002400EBC00101EB001050
:10B180004FF0FF3110B501EB800081B24FF47A70BF
:10B19000FCF7B2FD01490120C87510BD7C000024F8
:10B1A0000346012000E05843491EC9B2FBD2704754
:10B1B00007486FF0010102681161090C0268D16251
:10B1C000C1600021006841620248C0F8F010704779
:10B1D000FC1700247C0000242DE9F041164E308835
:10B1E000010426D51549C0B2154F00250D54B96884
:10B1F0001248884704000FD0104800F0D1F8012809
:10B2000001D0040014D0012C09D0022C09D0032C49
:10B2100009D0042C0CD108E0F868804708E009A0A8
:10B2200004E00BA002E00DA000E00FA0F4F71EFF69
:10B230003580BDE8F08100000E000024C00100242C
:10B240007C000024BAAFCAFDB4EDCEF3210D0A0094
:10B25000B2CECAFDB4EDCEF3210D0A00B2CECAFDC6
:10B26000CCABB6E0210D0A00CEB4D5D2B5BDC6A593
:10B27000C5E4B5C4BAAFCAFD210D0A0010F8011F1C
:10B28000202901D10028F9D1C8B270472DE9F04337
:10B290000E464FF00A0800240146254634600A781D
:10B2A000A2F13003092B14D903782D2B01D02B2BBD
:10B2B00000D174B1A2F14103052B0AD9582A05D057
:10B2C00012F0FF0F17D00120BDE8F083012C02D04F
:10B2D000F9E7412A01D34FF0100802782D2A04D053
:10B2E0002B2A04D0641CE4B203E0022500E001250F
:10B2F000401C491CD3E7B8F1100F074601D084B1B8
:10B3000012E0032C01D20220DEE73878302802D187
:10B310007878582801D00320D6E7A41EBF1CE4B2D9
:10B3200001E00420D0E70CB1641EE4B23878014695
:10B330003038092801D8814601E0A1F137092146BA
:10B340004046FFF72DFF326809FB0020306017F8F8
:10B35000011F0029E7D1022D01D1404230600020B9
:10B36000B2E702780B789A4201D00120704712B1FF
:10B37000401C491CF5E70020704702780A700278EB
:10B38000002A02D0401C491CF7E7704700210278D0
:10B390001AB1491C401CC9B2F9E7084670470000C1
:10B3A000F0B58DB004461E23694608AAFFF786FD56
:10B3B0000028099072D19DF8200027183E4C0025E6
:10B3C0008DF820509DF8200054F820106846FFF7B3
:10B3D000C8FF38B19DF82000401CC0B28DF8200095
:10B3E0000728EFD39DF820000426344C072855D2B7
:10B3F000DFE800F00404395A605F5E0030A0F4F723
:10B4000035FE30A0F4F732FE3EA0F4F72FFE4DA03B
:10B41000F4F72CFE5BA0F4F729FE6AA0F4F726FEF1
:10B4200078A0F4F723FE86A0F4F720FE8BA0F4F7B3
:10B430001DFE93A0F4F71AFE97A0F4F717FE9CA048
:10B44000F4F714FEA1A0F4F711FEA7A0F4F70EFE86
:10B45000B3A0F4F70BFEC0A0F4F708FECBA0F4F7FE
:10B4600005FED7A01BE016A0F4F700FEE4A0F4F759
:10B47000FDFD8DF820500BE0216806EBC000095857
:10B48000EFA0F4F7F3FD9DF82000401C8DF820009C
:10B49000217D9DF820008142EED856E257E2F4F774
:10B4A000E5FD00200DB0F0BD05A0F4F7DFFDCBE118
:10B4B0002CE20CE2EBE10000400000247C000024C0
:10B4C0000D0A00002D2D2D2D2D2D2D2D2D2D2D2D49
:10B4D0002D2D2D2D2D2D2D2D2D2D2D2D55534D411A
:10B4E00052542056332E332D2D2D2D2D2D2D2D2D17
:10B4F0002D2D2D2D2D2D2D2D2D2D2D2D2D2D2D2089
:10B500000D0A00002020202055534D415254CAC737
:10B51000D3C9414C49454E54454BBFAAB7A2B5C407
:10B52000D2BBB8F6C1E9C7C9B5C4B4AEBFDAB5F786
:10B53000CAD4BBA5BDBBD7E9BCFE2CCDA8B9FD20A4
:10B540000D0A0000CBFC2CC4E3BFC9D2D4CDA8B9EE
:10B55000FDB4AEBFDAD6FACAD6B5F7D3C3B3CCD0F2
:10B56000F2C0EFC3E6B5C4C8CEBACEBAAFCAFD2C9E
:10B57000B2A2D6B4D0D02ED2F2B4CB2CC4E3BFC981
:10B580000D0A0000D2D4CBE6D2E2B8FCB8C4BAAF00
:10B59000CAFDB5C4CAE4C8EBB2CECAFD28D6A7B36B
:10B5A000D6CAFDD7D62831302F3136BDF8D6C62CB5
:10B5B000D6A7B3D6B8BACAFD29A1A2D7D6B7FBB4CD
:10B5C000AE0D0A00A1A2BAAFCAFDC8EBBFDAB5D86A
:10B5D000D6B7B5C8D7F7CEAAB2CECAFD292CB5A525
:10B5E000B8F6BAAFCAFDD7EEB6E0D6A7B3D63130BB
:10B5F000B8F6CAE4C8EBB2CECAFD2CB2A2D6A7B345
:10B60000D60D0A00BAAFCAFDB7B5BBD8D6B5CFD4F0
:10B61000CABE2ED6A7B3D6B2CECAFDCFD4CABEBD3F
:10B62000F8D6C6C9E8D6C3B9A6C4DC2CD6A7B3D60B
:10B63000BDF8D6C6D7AABBBBB9A6C4DC2E0D0A007E
:10B64000BCBCCAF5D6A7B3D63A7777772E6F7065AC
:10B650006E6564762E636F6D0D0A000055534D4183
:10B660005254D3D037B8F6CFB5CDB3C3FCC1EE2812
:10B67000B1D8D0EBD0A1D0B4293A0D0A0000000017
:10B680003F3A202020202020BBF1C8A1B0EFD6FAFD
:10B69000D0C5CFA20D0A000068656C703A2020204A
:10B6A000BBF1C8A1B0EFD6FAD0C5CFA20D0A0000F9
:10B6B0006C6973743A202020BFC9D3C3B5C4BAAF34
:10B6C000CAFDC1D0B1ED0D0A0A00000069643A203C
:10B6D00020202020BFC9D3C3BAAFCAFDB5C4494496
:10B6E000C1D0B1ED0D0A0A006865783A202020200B
:10B6F000B2CECAFD3136BDF8D6C6CFD4CABE2CBA3A
:10B70000F3B8FABFD5B8F12BCAFDD7D6BCB4D6B4BE
:10B71000D0D0BDF8D6C6D7AABBBB0D0A0A00000020
:10B720006465633A20202020B2CECAFD3130BDF8D6
:10B73000D6C6CFD4CABE2CBAF3B8FABFD5B8F12B4F
:10B74000CAFDD7D6BCB4D6B4D0D0BDF8D6C6D7AA19
:10B75000BBBB0D0A0A00000072756E74696D653A14
:10B76000312CBFAAC6F4BAAFCAFDD4CBD0D0BCC668
:10B77000CAB13B302CB9D8B1D5BAAFCAFDD4CBD001
:10B78000D0BCC6CAB13B0D0A0A000000C7EBB0B47A
:10B79000D5D5B3CCD0F2B1E0D0B4B8F1CABDCAE4CB
:10B7A000C8EBBAAFCAFDC3FBBCB0B2CECAFDB2A2F1
:10B7B000D2D4BBD8B3B5BCFCBDE1CAF82E0D0A008B
:10B7C0002D2D2D2D2D2D2D2D2D2D2D2D2D2D2D2DA9
:10B7D0002D2D2D2D2D2D2D2D2D2D414C49454E54EA
:10B7E000454B2D2D2D2D2D2D2D2D2D2D2D2D2D2D53
:10B7F0002D2D2D2D2D2D2D2D2D2D2D200D0A000023
:10B800002D2D2D2D2D2D2D2D2D2D2D2D2D2D2D2D68
:10B810002D2D2D2D2D2D2D2D2DBAAFCAFDC7E5B502
:10B82000A52D2D2D2D2D2D2D2D2D2D2D2D2D2D2DD0
:10B830002D2D2D2D2D2D2D2D2D2D2D2D200D0A00B5
:10B8400025730D0A0000000042A0F4F70FFC8DF8EC
:10B85000205016E0216806EBC0000BAB0AAA08587E
:10B860006946FFF743FB9DF82010206850F831200F
:10B8700048A06946F4F7FAFB9DF82000401C8DF8BB
:10B880002000217D9DF820008142E3D85DE0AFF2E9
:10B89000D030F4F7EBFB08AA69463846FFF7BCFA4C
:10B8A0009DF82000002843D109A96846FFF7EEFC67
:10B8B0008DF8200010B104283AD102E009993AA08D
:10B8C0001CE03CA0F4F7D2FB0120E0753DE038A07D
:10B8D000F4F7CCFB08AA69463846FFF79DFA9DF8B5
:10B8E000200028BB09A96846FFF7D0FC8DF820008E
:10B8F00010B104281CD104E0099933A0F4F7B6FB79
:10B9000023E034A0F4F7B2FBE5751EE028A0F4F7BD
:10B91000ADFB08AA69463846FFF77EFA9DF820007D
:10B9200030B909A96846FFF7B1FC8DF8200008B1CD
:10B930000220B7E5099810F0FF0084F8EC0001D070
:10B9400029A000E02FA0F4F791FB19A0A7E50120A2
:10B95000A8E500002D2D2D2D2D2D2D2D2D2D2D2D3E
:10B960002D2D2D2D2D2D2D2D2D2D2D2D2DBAAFCA5B
:10B97000FD204944202D2D2D2D2D2D2D2D2D2D2D0E
:10B980002D2D2D2D2D2D2D2D2D2D2D2D2D2D2D2DE7
:10B99000200D0A0025732069642069733A0D0A306E
:10B9A00058253038580D0A004845583A305825581F
:10B9B0000D0A00003136BDF8D6C6B2CECAFDCFD4CE
:10B9C000CABE210D0A0000004445433A256C750D9E
:10B9D0000A0000003130BDF8D6C6B2CECAFDCFD4C1
:10B9E000CABE210D0A00000052756E2054696D65B3
:10B9F0002043616C63756C6174696F6E204F4E0DEE
:10BA00000A00000052756E2054696D652043616C18
:10BA100063756C6174696F6E204F46460D0A0000B5
:10BA20000160704730B5034640784FF4004544014B
:10BA30000020203401460AE002290BD0C20700D0C2
:10BA40002A4602EB50005A5C104480B2491CA142C5
:10BA5000F2D330BD0321F9E7CA0701D04FF000420D
:10BA600002EB510108447047010002000400060087
:10BA700008000A000C0010002000400080000001B7
:10BA800000000000000000000000000000000000B6
:10BA90003F40000000000000000030004000300087
:10BAA0004000000009000BC03D000BC03D00090034
:10BAB00018C024407FE0224031800000180024C0DC
:10BAC0001B000D803240018003801C4027401C80F9
:10BAD000074000401000600000000000000000006F
:10BAE0000000000000001F80204040200000402097
:10BAF00020401F8000000000090006001F80060093
:10BB000009000000040004003F800400040000005D
:10BB100000100060000000000000000004000400AD
:10BB200004000400040000000000004000000000C9
:10BB300000000000002001C00600380040000000A6
:10BB40001F802040204020401F8000000000104047
:10BB50003FC000400000000018C0214022402440A7
:10BB60001840000010802040244024401B8000002A
:10BB700002000D0011003FC0014000003C80244045
:10BB800024402440238000001F802440244034406F
:10BB9000038000003000200027C038002000000093
:10BBA0001B802440244024401B8000001C0022C035
:10BBB000224022401F8000000000000008400000DA
:10BBC0000000000000000000046000000000000011
:10BBD000000004000A001100208040400900090014
:10BBE0000900090009000000000040402080110009
:10BBF0000A00040018002000234024001800000060
:10BC00001F802040274029401F400000004007C0FF
:10BC100039000F0001C0004020403FC024402440B4
:10BC20001B8000001F80204020402040308000000A
:10BC300020403FC0204020401F80000020403FC0E7
:10BC400024402E4030C0000020403FC024402E0041
:10BC5000300000000F00108020402240338002009E
:10BC600020403FC0040004003FC02040204020404E
:10BC70003FC02040204000000060202020203FC026
:10BC80002000200020403FC024400B0030C0204056
:10BC900020403FC020400040004000C03FC03C006A
:10BCA00003C03C003FC0000020403FC00C402300C8
:10BCB0003FC020001F802040204020401F80000007
:10BCC00020403FC024402400180000001F80214075
:10BCD000214020E01FA0000020403FC0244026005B
:10BCE00019C0004018C02440244022403180000088
:10BCF000300020403FC020403000000020003F8046
:10BD0000004000403F80200020003E0001C00700AE
:10BD100038002000380007C03C0007C03800000091
:10BD2000204039C0060039C02040000020003840C3
:10BD300007C0384020000000304021C02640384075
:10BD400020C00000000000007FE0402040200000F4
:10BD5000000070000C000380004000000000402044
:10BD600040207FE000000000000020004000200094
:10BD70000000000000100010001000100010001063
:10BD800000000000400000000000000000000280F1
:10BD90000540054003C0004020003FC0044004406F
:10BDA00003800000000003800440044006400000BF
:10BDB00000000380044024403FC000400000038096
:10BDC0000540054003400000000004401FC024401F
:10BDD00024402000000002E00550055006500420D9
:10BDE00020403FC00440040003C000400000044065
:10BDF00027C000400000000000100010041027E0E1
:10BE00000000000020403FC00140070004C0044083
:10BE1000204020403FC000400040000007C0040018
:10BE200007C0040003C00000044007C00440040031
:10BE300003C0004000000380044004400380000071
:10BE4000041007F004500440038000000000038049
:10BE50000440045007F00010044007C002400400F2
:10BE600004000000000006400540054004C000003A
:10BE7000000004001F800440004000000400078010
:10BE80000040044007C000400400070004C00180D7
:10BE900006000400060001C0070001C00600000003
:10BEA000044006C0010006C0044000000410071052
:10BEB00004E00180060004000000044005C00640C4
:10BEC000044000000000000004007BE0402000006F
:10BED000000000000000FFF0000000000000402013
:10BEE0007BE00400000000004000800040002000D3
:10BEF00020004000000000000000000000000000E2
:10BF0000000000000000000000001FCC000C00003A
:10BF10000000000000000800300060000800300051
:10BF200060000000022003FC1E20022003FC1E20F3
:10BF30000220000000000E1811043FFF10840C784E
:10BF4000000000000F0010840F3800C0077818842C
:10BF50000078000000780F8410C411240E9800E4CB
:10BF60000084000808006800700000000000000065
:10BF70000000000000000000000007E01818200486
:10BF800040020000000040022004181807E00000F2
:10BF9000000000000240024001800FF001800240DA
:10BFA000024000000080008000800FF800800080C8
:10BFB000008000000001000D000E000000000000E5
:10BFC00000000000000000800080008000800080F1
:10BFD000008000800000000C000C00000000000049
:10BFE000000000000000000600180060018006004C
:10BFF00018002000000007F00808100410040808CA
:10C0000007F000000000080408041FFC00040004FE
:10C010000000000000000E0C1014102410441184C5
:10C020000E0C000000000C181004110411041288FA
:10C030000C700000000000E00320042408241FFC12
:10C040000024000000001F981084110411041088BF
:10C0500010700000000007F008881104110418880F
:10C060000070000000001C00100010FC13001C00F9
:10C070001000000000000E38114410841084114498
:10C080000E38000000000700088C10441044088897
:10C0900007F00000000000000000030C030C00008B
:10C0A0000000000000000000000101060000000088
:10C0B0000000000000000080014002200410080879
:10C0C0001004000002200220022002200220022090
:10C0D00002200000000010040808041002200140A3
:10C0E0000080000000000E001200100C106C108088
:10C0F0000F00000003E00C1813E4142417C40828F0
:10C1000007D000000004003C03C41C40074000E4CA
:10C11000001C000410041FFC1104110411040E88FB
:10C120000070000003E00C18100410041004100844
:10C130001C10000010041FFC100410041004080858
:10C1400007F0000010041FFC1104110417C41004B0
:10C150000818000010041FFC1104110017C0100083
:10C160000800000003E00C181004100410441C78B0
:10C170000040000010041FFC108400800080108428
:10C180001FFC10040000100410041FFC1004100415
:10C190000000000000030001100110011FFE10004C
:10C1A0001000000010041FFC110403801464181C0C
:10C1B0001004000010041FFC10040004000400041C
:10C1C000000C000010041FFC1F0000FC1F001FFCDF
:10C1D0001004000010041FFC0C04030000E0101801
:10C1E0001FFC100007F008081004100410040808D1
:10C1F00007F0000010041FFC1084108010801080D5
:10C200000F00000007F0081810241024101C080A62
:10C2100007F2000010041FFC1104110011C01130BE
:10C220000E0C000400000E1C110410841084104435
:10C230001C3800001800100010041FFC100410002F
:10C240001800000010001FF810040004000410047F
:10C250001FF8100010001E0011E0001C0070138079
:10C260001C0010001FC0103C00E01F0000E0103C4C
:10C270001FC000001004180C163401C001C0163491
:10C28000180C100410001C00130400FC13041C0004
:10C29000100000000804101C1064108413041C0417
:10C2A000101800000000000000007FFE4002400265
:10C2B00040020000000030000C0003800060001C01
:10C2C0000003000000004002400240027FFE000028
:10C2D000000000000000000020004000400040007E
:10C2E0002000000000010001000100010001000128
:10C2F000000100010000400040002000000000009C
:10C3000000000000000000980124014401440144A1
:10C3100000FC000410001FFC0088010401040088D8
:10C320000070000000000070008801040104010496
:10C33000008800000000007000880104010411085A
:10C340001FFC0004000000F80144014401440144C2
:10C3500000C800000000010401040FFC11041104D6
:10C3600011001800000000D601290129012901C986
:10C370000106000010041FFC0084010001000104FC
:10C3800000FC000400000104190419FC000400046E
:10C39000000000000000000300010101190119FE66
:10C3A0000000000010041FFC0024004001B4010C38
:10C3B000010400000000100410041FFC000400042D
:10C3C00000000000010401FC0104010001FC010463
:10C3D000010000FC010401FC0084010001000104D3
:10C3E00000FC0004000000F8010401040104010441
:10C3F00000F80000010101FF00850104010400882C
:10C4000000700000000000700088010401040105B4
:10C4100001FF00010104010401FC0084010401008A
:10C4200001800000000000CC01240124012401242B
:10C430000198000000000100010007F80104010458
:10C4400000000000010001F80004000400040108DD
:10C4500001FC0004010001800170000C001001606B
:10C460000180010001F0010C003001C00030010C1E
:10C4700001F0010000000104018C00740170018CC6
:10C4800001040000010101810171000E001801602A
:10C490000180010000000184010C01340144018489
:10C4A000010C0000000000000000000001003EFC44
:10C4B000400240020000000000000000FFFF0000FA
:10C4C000000000000000400240023EFC01000000AD
:10C4D000000000000000600080008000400040007C
:10C4E000200020000000000000000000000000000C
:10C4F000000000000000000000000000000000003C
:10C50000000000000000000000000000000000002B
:10C51000000000000000000F80380FFE380F803848
:10C52000000000000000000000000000000000000B
:10C5300000000100000600000C000038000031007F
:10C54000000600000C000038000030000000000071
:10C550000000000061800067F807F980006180003A
:10C5600061800061800061800067F807F9800061E8
:10C570008000000000000000000001C0E003E0F0C7
:10C580000630080418081FFFFE040E080787F00392
:10C5900081E000000000000001F000060C0004042F
:10C5A00008060C7001F9C0000E00003BE000EC181A
:10C5B000070808040C180003E00000000001E00078
:10C5C00007F003F818041C0804170807E1D003C09B
:10C5D000E00023B0003C080020080000100000002C
:10C5E0000000000100003100003200001C000000CB
:10C5F000000000000000000000000000000000003B
:10C60000000000000000000000000000000000002A
:10C61000000000007F0001FFC00780F00C00181030
:10C6200000042000020000000000002000021000B2
:10C63000040C00180780F001FFC0007F000000001C
:10C6400000000000000000000000000000000000EA
:10C650004200006600006600003C0000180003FF76
:10C66000C0001800003C00006600006600004200A8
:10C67000000000000800000800000800000800009A
:10C68000080001FFC00008000008000008000008C2
:10C69000000008000000000000010000310000322E
:10C6A00000001C000000000000000000000000006E
:10C6B000000000000000000000000000080000086A
:10C6C0000000080000080000080000080000080042
:10C6D0000008000008000008000000000000000042
:10C6E00000000000380000380000380000000000A2
:10C6F000000000000000000000000000000000003A
:10C7000000000000000600001C0000700001800016
:10C710000E0000380000C0000700001C00003000C0
:10C7200000000000000000007F8001FFE003807037
:10C7300006001804000804000806001803807001B1
:10C74000FFE0007F8000000000000000000001000A
:10C750000801000801000803FFF807FFF8000008BF
:10C7600000000800000800000000000000000001B8
:10C77000C03802C0580400980401180402180404C8
:10C7800018061C1803F81801E0F80000000000006B
:10C7900000000001C0E003C0F00400080408080421
:10C7A000080806180803F41801E7F00001E000008B
:10C7B00000000000000000000300000D0000110058
:10C7C00000610000810803010807FFF80FFFF8006F
:10C7D00001080001080000000000000000E007FC64
:10C7E000D0060808061008061008061008061838B3
:10C7F000060FF00607C00000000000000000000067
:10C800003F8001FFE0038430020818041008041080
:10C8100008041008071810030FF00007C0000000FC
:10C8200000000000000003C0000700000600000632
:10C8300000F80607F806180006E0000700000600EA
:10C840000000000000000001E1E003F7F0063410F2
:10C85000041808041808040C08040C080616180329
:10C86000F3F001C1E000000000000000F80003FC4C
:10C870003003063804020804020804020804041005
:10C880000308F001FFC0007F00000000000000006E
:10C890000000000000000000000000007038007080
:10C8A00038007038000000000000000000000000A8
:10C8B0000000000000000000000000000000000078
:10C8C000301A00301C0000000000000000000000D2
:10C8D000000000000000000000000008000014003C
:10C8E000002200004100008080010040020020047E
:10C8F00000100800080000000000000021000021D6
:10C900000000210000210000210000210000210082
:10C9100000210000210000210000000000000000B4
:10C920000000080008040010020020010040008000
:10C9300080004100002200001400000800000000F8
:10C9400000000003C00004C0000400000800380814
:10C950000F380808380810000C300007E00003C04A
:10C9600000000000000000003F8000FFE003807036
:10C97000020F1006708804C088048308047F8802B0
:10C98000C09003012000FE400000080000180001D4
:10C99000F8003E0801C20007020007E20000FE00A6
:10C9A000001FC80001F80000380000080400080754
:10C9B000FFF807FFF804080804080804080804083A
:10C9C0000806180803F41801E7F00001E000000071
:10C9D000000000003F8001FFE003807002001804A7
:10C9E0000008040008040008040010060020078066
:10C9F000C000000004000807FFF807FFF804000863
:10CA000004000804000804001802001003807001EC
:10CA1000FFE0007F8000000004000807FFF807FF28
:10CA2000F8040808040808040808040808043E0874
:10CA30000400080600180100600000000400080758
:10CA4000FFF807FFF80408080408000408000408B9
:10CA500000043E0006000006000001800000000007
:10CA6000000000003F8001FFE00380700600180412
:10CA700000080402080402080203F00783F0000221
:10CA80000000020004000807FFF807FFF804080888
:10CA9000000800000800000800000800040808075B
:10CAA000FFF807FFF8040008000000000000040081
:10CAB0000804000804000807FFF807FFF80400084E
:10CAC000040008040008000000000000000000004E
:10CAD000000600000700000104000104000104003A
:10CAE0000307FFFE07FFFC04000004000004000031
:10CAF00004000807FFF807FFF8040C0800180000FE
:10CB00003E0004C7800503C80600F804003804008E
:10CB10001800000804000807FFF807FFF8040008E1
:10CB200000000800000800000800000800000800DD
:10CB3000001800006000000004000807FFF80780EC
:10CB40000807FC00007FC00003F80007C000780061
:10CB500007800807FFF807FFF8040008040008072B
:10CB6000FFF807000803C00000E000003800001EC6
:10CB7000000007000001C00400F007FFF8040000F7
:10CB8000000000007F8001FFE003807006001804B1
:10CB9000000804000806001803003001FFE0007FD1
:10CBA0008000000004000807FFF807FFF8040408ED
:10CBB000040400040400040400040400060C000340
:10CBC000F80001F000000000000000007F8001FF7D
:10CBD000E00380700600880400880400C806003C5A
:10CBE00003003E01FFE6007F840000000400080708
:10CBF000FFF807FFF8040808040800040C00040FFD
:10CC000000040BC00610F003F03801E00800000833
:10CC100000000001E0F803F03006301004180804AA
:10CC20001808040C08040C080206180207F0078113
:10CC3000E000000001800006000004000004000085
:10CC400004000807FFF807FFF804000804000004C8
:10CC5000000006000001800004000007FFE007FF5D
:10CC6000F004001800000800000800000800000898
:10CC700000000804001007FFE004000004000006A4
:10CC8000000007E00007FE00041FE00001F80000BC
:10CC9000380001E0043E0007C00006000004000068
:10CCA00004000007E00007FFC0041FF80007C007EA
:10CCB000F80007FF80043FF80007C004F8000700F1
:10CCC0000004000000000004000806001807C078F7
:10CCD00005F1C8003E00001F800463E80780F806E5
:10CCE000001804000800000004000006000007808F
:10CCF0000007E008047C08001FF80007F800180887
:10CD000004E0080700000600000400000000000125
:10CD100000080600380400F80403E8040F08047C47
:10CD20000805F00807C008070018040060000000AC
:10CD30000000000000000000000000000000003FB4
:10CD4000FFFE20000220000220000220000220003E
:10CD500002000000000000000000080000070000C2
:10CD600000C0000038000006000001C000003000D4
:10CD7000000E000001000000000000000000200084
:10CD8000022000022000022000022000023FFFFEDD
:10CD90000000000000000000000000000000000093
:10CDA000000000000008000010000030000020001B
:10CDB000003000001000000800000000000000002B
:10CDC000000001000001000001000001000001005E
:10CDD000000100000100000100000100000100004E
:10CDE0000100000100000000000000000020000021
:10CDF00020000010000010000000000000000000F3
:10CE000000000000000000000000000000F0001919
:10CE1000F8001B180022080026080024080024102F
:10CE2000003FF8001FF80000080000180000000490
:10CE3000000007FFF80FFFF000181800100800208E
:10CE400008002008003018001FF0000FC00000008C
:10CE50000000000007C0001FF0001830002008008C
:10CE60002008002008003C08001C100000600000A2
:10CE7000000000000000000007C0001FF00038188C
:10CE800000200800200800200804101007FFF80FF9
:10CE9000FFF000001000000000000000000000078C
:10CEA000C0001FF0001230002218002208002208E3
:10CEB000003208001E10000E2000000000000000DC
:10CEC000200000200800200801FFF803FFF80620DA
:10CED00008042008042008072000030000000000C8
:10CEE00000000000000E000E6E001FF30031B100C4
:10CEF00020B10020B1003191001F13002E1E002030
:10CF00000E00300000000004000807FFF80FFFF8D3
:10CF1000001008002000002000002008003FF8005A
:10CF20001FF80000080000000000000000000020C2
:10CF300008002008002008063FF8063FF800000817
:10CF400000000800000800000000000000000000D1
:10CF50000000000003000003002001002001002069
:10CF600003063FFE063FFC0000000000000000003A
:10CF700000000004000807FFF80FFFF80001880018
:10CF80000300002FC00038F80020380020080000FF
:10CF90000800000000000000000004000804000871
:10CFA00004000807FFF80FFFF80000080000080061
:10CFB0000008000000000000002008003FF8003FCB
:10CFC000F8001008002000003FF8003FF8001008AB
:10CFD000002000003FF8003FF800000800000000BB
:10CFE0002008003FF8003FF8001008001000002063
:10CFF00000002008003FF8001FF8000008000000B3
:10D000000000000007C0000FF000183000300800DA
:10D010002008002008003008001830000FF000073A
:10D02000C0000000000000002001003FFF003FFFA3
:10D0300000101100200900200800200800303800EE
:10D040001FF0000FC00000000000000007C0001F1C
:10D05000F0003818002008002008002009001011F6
:10D06000001FFF003FFF000001000000002008003B
:10D070002008002008003FF8003FF80008080010D2
:10D0800008002008002000003000003000000000F0
:10D09000000000000000000C78001E18003308009B
:10D0A00023080021080021880021980030F0003872
:10D0B00060000000000000002000002000002000B0
:10D0C00000FFF003FFF800200800200800200800FF
:10D0D0000030000000000000000000002000003FC1
:10D0E000F0007FF800001800000800000800201081
:10D0F000003FF8007FF0000010000000000000007A
:10D100002000003000003C00003F800023F00000C1
:10D1100078000070002380003C00003000002000F8
:10D12000002000003C00003FE00023F80000E00089
:10D130002700003E00003FE00021F80001E0003E33
:10D1400000002000000000002008002008003838FF
:10D15000003E680027800003C8002CF80038380023
:10D16000201800200800000000000000200000300F
:10D1700003003C01003F830023EC0000700023808B
:10D18000003C000020000020000000000000000023
:10D1900000000038080020380020F80023E8002FA5
:10D1A00088003E08003808002018000070000000C9
:10D1B000000000000000000000000000000000006F
:10D1C00008000014001FF7FC3000062000020000D9
:10D1D000000000000000000000000000000000004F
:10D1E000000000000000FFFFFF0000000000000042
:10D1F000000000000000000000000000000020000F
:10D20000023000061FF7FC001400000800000000B8
:10D2100000000000000000000000000000000018F6
:10D2200000006000004000004000002000001000EE
:10D23000000800000400000400000C0000100000C2
:10D2400000000000000000000000000000000000DE
:10D2500000000000000000000000000000000000CE
:10D2600000000000000000000000000000000000BE
:10D2700000000000000000000000000000000000AE
:10D28000000000000000000000000000000000009E
:10D29000000000000000000000000000000000008E
:10D2A000000000000000000000000000000000007E
:10D2B000000000000000000000000000000000006E
:10D2C000000000000000000000000000000000005E
:10D2D000000000000000000007F000C007FFE1E0D0
:10D2E00007F001E0000000C00000000000000000A6
:10D2F000000000000000000000000000000000002E
:10D30000000000000000000000000000000000001D
:10D31000000000000000000000000000000000000D
:10D3200000000000000000000000000000000000FD
:10D3300000000000000000000000000000000000ED
:10D3400000000000000000000020000001C00000FC
:10D35000078000001F0000001E0000001C200000CD
:10D3600001C00000078000001F0000001E00000038
:10D370001C00000000000000000000000000000091
:10D38000000000000000000000000000000000009D
:10D39000000000000000000000000000000000008D
:10D3A000000000000000000000000000000000007D
:10D3B000000000000000000000000000000000006D
:10D3C0000000000000180C0000180C0000180FE00E
:10D3D000001FFC0003F80C0000180C0000180C00E3
:10D3E00000180C0000180C0000180FE0001FFC00D3
:10D3F00003F80C0000180C0000180C0000000000DE
:10D40000000000000000000000000000000000001C
:10D41000000000000000000000000000000000000C
:10D4200000000000000000000000000000000000FC
:10D4300000000000000000000000000000000000EC
:10D44000000000000000000000000780007807C016
:10D4500000FC0640010E002003070020020380208C
:10D460000FFFFFFC0201C0200200E06001307040AD
:10D4700001F03F8000F01F000000000000000000ED
:10D48000000000000000000000000000000000009C
:10D49000000000000000000000000000000000008C
:10D4A000000000000000000000000000000000007C
:10D4B000000000000000000000000000000000006C
:10D4C00000FE000001FF00000301800002008060F8
:10D4D000030181C001FF070000FE18000000E0000A
:10D4E0000003BF00000CFFC00071806001C100207C
:10D4F000030180600000FFC000003F00000000004A
:10D50000000000000000000000000000000000001B
:10D51000000000000000000000000000000000000B
:10D5200000000000000000000000000000000000FB
:10D5300000000000000000000000000000000000EB
:10D5400000001F0000007FC000FCC0C001FF806021
:10D550000303E0200202782002061E2003FC07409D
:10D5600001F00380000103C000011C600001E02005
:10D5700000010020000100400000018000000000C8
:10D58000000000000000000000000000000000009B
:10D59000000000000000000000000000000000008B
:10D5A000000000000000000000000000000000007B
:10D5B000000000000000000000000000000000006B
:10D5C00000000000002000001C6000001C40000063
:10D5D0001F8000000F00000000000000000000009D
:10D5E000000000000000000000000000000000003B
:10D5F000000000000000000000000000000000002B
:10D60000000000000000000000000000000000001A
:10D61000000000000000000000000000000000000A
:10D6200000000000000000000000000000000000FA
:10D6300000000000000000000000000000000000EA
:10D6400000000000000000000000000000000000DA
:10D650000000000000000000000000000007F800CB
:10D66000003FFF00007807C001C000E00300003069
:10D670000400000808000004100000020000000080
:10D68000000000000000000000000000000000009A
:10D69000000000000000000000000000000000008A
:10D6A000000000000000000000000000000000007A
:10D6B000000000000000000000000000000000006A
:10D6C0000000000010000002080000040400000830
:10D6D0000300003001C000E0007807C0003FFF00F9
:10D6E0000007F8000000000000000000000000003B
:10D6F000000000000000000000000000000000002A
:10D700000000000000000000000000000000000019
:10D710000000000000000000000000000000000009
:10D7200000000000000000000000000000000000F9
:10D7300000000000000000000000000000000000E9
:10D740000000000000000000000C1800000E38006F
:10D75000000E3800000630000003600000614380C6
:10D7600000FFFF80006143000003600000063000FE
:10D77000000E3800000E3800000C180000000000F9
:10D780000000000000000000000000000000000099
:10D790000000000000000000000000000000000089
:10D7A0000000000000000000000000000000000079
:10D7B0000000000000000000000000000000000069
:10D7C0000000000000000000000080000000800059
:10D7D0000000800000008000000080000000800049
:10D7E000007FFF000000800000008000000080003B
:10D7F00000008000000080000000800000000000A9
:10D800000000000000000000000000000000000018
:10D810000000000000000000000000000000000008
:10D8200000000000000000000000000000000000F8
:10D8300000000000000000000000000000000000E8
:10D840000000000000000001000000E3000000E212
:10D85000000000FC00000078000000000000000054
:10D8600000000000000000000000000000000000B8
:10D8700000000000000000000000000000000000A8
:10D880000000000000000000000000000000000098
:10D890000000000000000000000000000000000088
:10D8A0000000000000000000000000000000000078
:10D8B0000000000000000000000000000000000068
:10D8C00000000000000080000000800000008000D8
:10D8D0000000800000008000000080000000800048
:10D8E0000000800000008000000080000000800038
:10D8F00000008000000080000000800000000000A8
:10D900000000000000000000000000000000000017
:10D910000000000000000000000000000000000007
:10D9200000000000000000000000000000000000F7
:10D9300000000000000000000000000000000000E7
:10D940000000000000000000000000C0000001E036
:10D95000000001E0000000C0000000000000000026
:10D9600000000000000000000000000000000000B7
:10D9700000000000000000000000000000000000A7
:10D980000000000000000000000000000000000097
:10D990000000000000000000000000000000000087
:10D9A0000000000000000000000000000000000077
:10D9B0000000000000000000000000000000000067
:10D9C000000000000000000C00000038000000E033
:10D9D0000000038000000E00000038000000E0009E
:10D9E00000038000000E00000038000000E000008E
:10D9F000038000000E00000018000000000000007E
:10DA00000000000000000000000000000000000016
:10DA10000000000000000000000000000000000006
:10DA200000000000000000000000000000000000F6
:10DA300000000000000000000000000000000000E6
:10DA40000000000000000000000FF800007FFF0051
:10DA500000F00780018000C0030000600200002089
:10DA6000020000200200002003000060018000C0CE
:10DA700000E00380007FFF00000FF80000000000BE
:10DA80000000000000000000000000000000000096
:10DA90000000000000000000000000000000000086
:10DAA0000000000000000000000000000000000076
:10DAB0000000000000000000000000000000000066
:10DAC00000000000000000000000000000800020B6
:10DAD00000800020008000200080006001FFFFE047
:10DAE00003FFFFE0000000600000002000000020B5
:10DAF0000000002000000000000000000000000006
:10DB00000000000000000000000000000000000015
:10DB10000000000000000000000000000000000005
:10DB200000000000000000000000000000000000F5
:10DB300000000000000000000000000000000000E5
:10DB40000000000000000000007800E00098016084
:10DB50000100026002000460020008600200106020
:10DB600002002060020040600300806001830060CA
:10DB700001FE00E0007C07800000000000000000C3
:10DB80000000000000000000000000000000000095
:10DB90000000000000000000000000000000000085
:10DBA0000000000000000000000000000000000075
:10DBB0000000000000000000000000000000000065
:10DBC000000000000000000000F0078001F007C026
:10DBD000010000400200002002010020020100209C
:10DBE00002010020030380200186804001FCC0C0A8
:10DBF00000787F8000001E00000000000000000090
:10DC00000000000000000000000000000000000014
:10DC10000000000000000000000000000000000004
:10DC200000000000000000000000000000000000F4
:10DC300000000000000000000000000000000000E4
:10DC4000000000000000080000003800000048004C
:10DC50000001880000060800000C081000300810C1
:10DC60000040081001FFFFF003FFFFF003FFFFF08B
:10DC7000000008100000081000000810000000005C
:10DC80000000000000000000000000000000000094
:10DC90000000000000000000000000000000000084
:10DCA0000000000000000000000000000000000074
:10DCB0000000000000000000000000000000000064
:10DCC000000000000000000000000780001F8640E8
:10DCD00003E10020030200200304002003040020CD
:10DCE000030400200304002003060040030301C0D6
:10DCF0000301FF8003007E00000000000000000020
:10DD00000000000000000000000000000000000013
:10DD10000000000000000000000000000000000003
:10DD200000000000000000000000000000000000F3
:10DD300000000000000000000000000000000000E3
:10DD400000000000000000000007FC00003FFF0092
:10DD50000070C380008180C00101006003020020C8
:10DD60000202002002020020020200200203004002
:10DD700001C180C000C0FF8000007E0000000000E4
:10DD80000000000000000000000000000000000093
:10DD90000000000000000000000000000000000083
:10DDA0000000000000000000000000000000000073
:10DDB0000000000000000000000000000000000063
:10DDC000000000000000000000F0000003C00000A0
:10DDD0000380000003000000030007E003003FE0B1
:10DDE0000301C000030600000318000003600000E8
:10DDF000038000000300000000000000000000009D
:10DE00000000000000000000000000000000000012
:10DE10000000000000000000000000000000000002
:10DE200000000000000000000000000000000000F2
:10DE300000000000000000000000000000000000E2
:10DE40000000000000001F0000783F8000FC60C060
:10DE5000018EC040030780200203002002018020C1
:10DE6000020180200201C0200301E040018670C051
:10DE700000FC3F8000781F00000000000000000050
:10DE80000000000000000000000000000000000092
:10DE90000000000000000000000000000000000082
:10DEA0000000000000000000000000000000000072
:10DEB0000000000000000000000000000000000062
:10DEC00000000000003F000000FF81C001C0C1C091
:10DED00001006020020020200200202002002020FB
:10DEE00002002060020040C00100C18000C18F001C
:10DEF000007FFE00001FF000000000000000000096
:10DF00000000000000000000000000000000000011
:10DF10000000000000000000000000000000000001
:10DF200000000000000000000000000000000000F1
:10DF300000000000000000000000000000000000E1
:10DF400000000000000000000000000000000000D1
:10DF50000000000000000000000300C0000781E096
:10DF6000000781E0000300C0000000000000000086
:10DF700000000000000000000000000000000000A1
:10DF80000000000000000000000000000000000091
:10DF90000000000000000000000000000000000081
:10DFA0000000000000000000000000000000000071
:10DFB0000000000000000000000000000000000061
:10DFC0000000000000000000000000000000000051
:10DFD0000000000000000000000600660006007857
:10DFE0000000000000000000000000000000000031
:10DFF0000000000000000000000000000000000021
:10E000000000000000000000000000000000000010
:10E010000000000000000000000000000000000000
:10E0200000000000000000000000000000000000F0
:10E0300000000000000000000000000000000000E0
:10E040000000000000000000000080000001C0008F
:10E050000003600000063000000C180000180C00DF
:10E06000003006000060030000C001800100004095
:10E07000020000200400001000000000000000006A
:10E080000000000000000000000000000000000090
:10E090000000000000000000000000000000000080
:10E0A0000000000000000000000000000000000070
:10E0B0000000000000000000000000000000000060
:10E0C0000000000000041000000410000004100014
:10E0D00000041000000410000004100000041000F0
:10E0E00000041000000410000004100000041000E0
:10E0F00000041000000410000004100000000000E4
:10E10000000000000000000000000000000000000F
:10E1100000000000000000000000000000000000FF
:10E1200000000000000000000000000000000000EF
:10E1300000000000000000000000000000000000DF
:10E140000000000000000000040000100200002099
:10E150000100004000C001800060030000300600A4
:10E1600000180C00000C18000006300000036000CE
:10E170000001C0000000800000000000000000005E
:10E18000000000000000000000000000000000008F
:10E19000000000000000000000000000000000007F
:10E1A000000000000000000000000000000000006F
:10E1B000000000000000000000000000000000005F
:10E1C00000000000000000000078000001F80000DE
:10E1D0000238000002000000040000C0040079E0E2
:10E1E000040081E0040100C00403000002020000FA
:10E1F0000306000001FC000000F800000000000021
:10E20000000000000000000000000000000000000E
:10E2100000000000000000000000000000000000FE
:10E2200000000000000000000000000000000000EE
:10E2300000000000000000000000000000000000DE
:10E2400000000000000FF800003FFE000070078093
:10E2500000C000C00101F8400307FC20021E04209A
:10E260000230082002203020023FFC20013F044001
:10E2700001800CC000E03180001FC20000000000DF
:10E28000000000000000000000000000000000008E
:10E29000000000000000000000000000000000007E
:10E2A000000000000000000000000000000000006E
:10E2B000000000000000000000000000000000005E
:10E2C0000000002000000060000003E000003E208D
:10E2D0000003E020003E200003E020000380200037
:10E2E00007FC2000003FE0000003FE2000003FE0AC
:10E2F000000001E0000000200000002000000000FD
:10E30000000000000000000000000000000000000D
:10E3100000000000000000000000000000000000FD
:10E3200000000000000000000000000000000000ED
:10E3300000000000000000000000000000000000DD
:10E3400000000000020000200200002003FFFFE0A8
:10E3500003FFFFE002010020020100200201002073
:10E3600002010020020100200303002001868060DA
:10E3700001FCC0C000F87F8000001F00000000000A
:10E38000000000000000000000000000000000008D
:10E39000000000000000000000000000000000007D
:10E3A000000000000000000000000000000000006D
:10E3B000000000000000000000000000000000005D
:10E3C000000000000007F800003FFF000070078019
:10E3D00000C000C001000040030000200200002037
:10E3E0000200002002000020020000200100004086
:10E3F000018000C003C00180003006000000000062
:10E40000000000000000000000000000000000000C
:10E4100000000000000000000000000000000000FC
:10E4200000000000000000000000000000000000EC
:10E4300000000000000000000000000000000000DC
:10E4400000000000020000200200002003FFFFE0A7
:10E4500003FFFFE002000020020000200200002075
:10E46000020000200300006001000040018000C0A5
:10E4700000F00780007FFE00000FF80000000000A1
:10E48000000000000000000000000000000000008C
:10E49000000000000000000000000000000000007C
:10E4A000000000000000000000000000000000006C
:10E4B000000000000000000000000000000000005C
:10E4C00000000000020000200200002003FFFFE027
:10E4D00003FFFFE0020100200201002002010020F2
:10E4E000020100200201002002038020020FE02030
:10E4F0000300006003C000E00060030000000000B3
:10E50000000000000000000000000000000000000B
:10E5100000000000000000000000000000000000FB
:10E5200000000000000000000000000000000000EB
:10E5300000000000000000000000000000000000DB
:10E5400000000000020000200200002003FFFFE0A6
:10E5500003FFFFE002010020020100200201000091
:10E56000020100000201000002010000020380001D
:10E57000030FE0000300000003C000000060000083
:10E58000000000000000000000000000000000008B
:10E59000000000000000000000000000000000007B
:10E5A000000000000000000000000000000000006B
:10E5B000000000000000000000000000000000005B
:10E5C000000000000007F800003FFE000070078018
:10E5D00001C001C001000040030000200200002033
:10E5E0000200002002000020010020200100204045
:10E5F00003C03F8000303F8000002000000020006A
:10E60000000000000000000000000000000000000A
:10E6100000000000000000000000000000000000FA
:10E6200000000000000000000000000000000000EA
:10E6300000000000000000000000000000000000DA
:10E64000020000200200002003FFFFE003FFFFE0C4
:10E650000200802002008020000080000000800076
:10E6600000008000020080200200802003FFFFE005
:10E6700003FFFFE002000020020000200000000075
:10E68000000000000000000000000000000000008A
:10E69000000000000000000000000000000000007A
:10E6A000000000000000000000000000000000006A
:10E6B000000000000000000000000000000000005A
:10E6C0000000000000000000000000000200002028
:10E6D00002000020020000200200002003FFFFE0F3
:10E6E00003FFFFE0020000200200002002000020E3
:10E6F00002000020000000000000000000000000F8
:10E700000000000000000000000000000000000009
:10E7100000000000000000000000000000000000F9
:10E7200000000000000000000000000000000000E9
:10E7300000000000000000000000000000000000D9
:10E74000000000000000000E0000000F0000000F9D
:10E7500000000001020000010200000102000003AD
:10E760000200000603FFFFFC03FFFFF802000000A9
:10E770000200000002000000020000000000000093
:10E780000000000000000000000000000000000089
:10E790000000000000000000000000000000000079
:10E7A0000000000000000000000000000000000069
:10E7B0000000000000000000000000000000000059
:10E7C00000000000020000200200002003FFFFE024
:10E7D00003FFFFE00200C0200201002000078000CC
:10E7E000000FE0000030F80002603E2003800F20A0
:10E7F000030003E0020000E002000020000000200F
:10E800000000000000000000000000000000000008
:10E8100000000000000000000000000000000000F8
:10E8200000000000000000000000000000000000E8
:10E8300000000000000000000000000000000000D8
:10E8400000000000020000200200002003FFFFE0A3
:10E8500003FFFFE002000020020000200000002073
:10E860000000002000000020000000200000002028
:10E8700000000060000000E0000003000000000055
:10E880000000000000000000000000000000000088
:10E890000000000000000000000000000000000078
:10E8A0000000000000000000000000000000000068
:10E8B0000000000000000000000000000000000058
:10E8C000020000200200002003FFFFE003E0002020
:10E8D00003FF0020001FF0000001FF8000000FE098
:10E8E00000001E000003E000003E002003E00020C6
:10E8F00003FFFFE003FFFFE0020000200200002012
:10E900000000000000000000000000000000000007
:10E9100000000000000000000000000000000000F7
:10E9200000000000000000000000000000000000E7
:10E9300000000000000000000000000000000000D7
:10E94000020000200200002003FFFFE003800020FF
:10E9500003F0002000FC0000001F00000007C000C2
:10E960000001F00000007C0002001F80020007E0B0
:10E9700003FFFFE0020000000200000000000000B2
:10E980000000000000000000000000000000000087
:10E990000000000000000000000000000000000077
:10E9A0000000000000000000000000000000000067
:10E9B0000000000000000000000000000000000057
:10E9C00000000000000FF800003FFE0000F007808C
:10E9D000018000C001000040020000200200002071
:10E9E000020000200200002001000040018000C061
:10E9F00000F00380003FFE00000FF8000000000060
:10EA00000000000000000000000000000000000006
:10EA100000000000000000000000000000000000F6
:10EA200000000000000000000000000000000000E6
:10EA300000000000000000000000000000000000D6
:10EA400000000000020000200200002003FFFFE0A1
:10EA500003FFFFE00200802002008020020080000F
:10EA6000020080000200800002008000030180009C
:10EA70000183000000FE0000007C00000000000098
:10EA80000000000000000000000000000000000086
:10EA90000000000000000000000000000000000076
:10EAA0000000000000000000000000000000000066
:10EAB0000000000000000000000000000000000056
:10EAC00000000000000FF800007FFF0000F003804E
:10EAD000018001C001000640020004200200042061
:10EAE00002000620020003E0010000F80180005C43
:10EAF00000E0038C003FFF0C000FFC18000000003A
:10EB00000000000000000000000000000000000005
:10EB100000000000000000000000000000000000F5
:10EB200000000000000000000000000000000000E5
:10EB300000000000000000000000000000000000D5
:10EB400000000000020000200200002003FFFFE0A0
:10EB500003FFFFE00201002002010020020180000B
:10EB60000201E0000201FC0003033F80018607E090
:10EB700001FC00E000F80020000000200000000080
:10EB80000000000000000000000000000000000085
:10EB90000000000000000000000000000000000075
:10EBA0000000000000000000000000000000000065
:10EBB0000000000000000000000000000000000055
:10EBC00000000000000000000078060000FE01E0E8
:10EBD000018600C0030300400203002002018020E0
:10EBE000020180200201C0200200C0200100E0607C
:10EBF000018070C003E03F8000001F0000000000A3
:10EC00000000000000000000000000000000000004
:10EC100000000000000000000000000000000000F4
:10EC200000000000000000000000000000000000E4
:10EC300000000000000000000000000000000000D4
:10EC400000000000006000000380000003000000DE
:10EC500002000000020000200200002003FFFFE08D
:10EC600003FFFFE00200002002000020020000007D
:10EC7000020000000380000000E00000000000002F
:10EC80000000000000000000000000000000000084
:10EC90000000000000000000000000000000000074
:10ECA0000000000000000000000000000000000064
:10ECB0000000000000000000000000000000000054
:10ECC000020000000200000003FFFF0003FFFFC07E
:10ECD0000200004002000060000000200000002050
:10ECE0000000002000000020020000400200008020
:10ECF00003FFFF000200000002000000000000000F
:10ED00000000000000000000000000000000000003
:10ED100000000000000000000000000000000000F3
:10ED200000000000000000000000000000000000E3
:10ED300000000000000000000000000000000000D3
:10ED400000000000020000000200000003C00000FC
:10ED500003FC0000023FC0000003F80000007F80B9
:10ED6000000007E000000780000078000203C000F8
:10ED7000023C000003C0000002000000020000008E
:10ED80000000000000000000000000000000000083
:10ED90000000000000000000000000000000000073
:10EDA0000000000000000000000000000000000063
:10EDB0000000000000000000000000000000000053
:10EDC0000200000003C0000003FF8000023FFE00BD
:10EDD00002007FE000000F000200F00003EF0000DF
:10EDE00003FF8000020FFE0000003FE000001F0054
:10EDF0000207E00003F8000003000000020000002A
:10EE00000000000000000000000000000000000002
:10EE100000000000000000000000000000000000F2
:10EE200000000000000000000000000000000000E2
:10EE300000000000000000000000000000000000D2
:10EE4000000000000200002002000020038000E01B
:10EE500003F0032002FC0C20021F30000007C0005A
:10EE60000007F00002187C0002601F20038003E00E
:10EE7000020000E00200002000000020000000006E
:10EE80000000000000000000000000000000000082
:10EE90000000000000000000000000000000000072
:10EEA0000000000000000000000000000000000062
:10EEB0000000000000000000000000000000000052
:10EEC00000000000020000000300000003C000007A
:10EED00003F80000023E0020020FC0200001FFE006
:10EEE00000007FE000038020021C00200270000070
:10EEF000038000000200000002000000000000008B
:10EF00000000000000000000000000000000000001
:10EF100000000000000000000000000000000000F1
:10EF200000000000000000000000000000000000E1
:10EF300000000000000000000000000000000000D1
:10EF40000000000000000020006000E0038003E0FB
:10EF500003000FA002003E200200F8200203E02080
:10EF6000020F8020023E00200278002003E00060B3
:10EF7000038000E002000300000000000000000029
:10EF80000000000000000000000000000000000081
:10EF90000000000000000000000000000000000071
:10EFA0000000000000000000000000000000000061
:10EFB0000000000000000000000000000000000051
:10EFC0000000000000000000000000000000000041
:10EFD00000000000000000001FFFFFFC1000000404
:10EFE00010000004100000041000000410000004D1
:10EFF00010000004100000040000000000000000E9
:10F000000000000000000000000000000000000000
:10F0100000000000000000000000000000000000F0
:10F0200000000000000000000000000000000000E0
:10F0300000000000000000000000000000000000D0
:10F0400000000000000000000000000007000000B9
:10F0500003C0000000780000001E00000003C00094
:10F060000000F00000001E0000000780000000F01B
:10F070000000003C0000000600000000000000004E
:10F080000000000000000000000000000000000080
:10F090000000000000000000000000000000000070
:10F0A0000000000000000000000000000000000060
:10F0B0000000000000000000000000000000000050
:10F0C0000000000000000000100000041000000418
:10F0D00010000004100000041000000410000004E0
:10F0E000100000041FFFFFFC0000000000000000F3
:10F0F0000000000000000000000000000000000010
:10F1000000000000000000000000000000000000FF
:10F1100000000000000000000000000000000000EF
:10F1200000000000000000000000000000000000DF
:10F1300000000000000000000000000000000000CF
:10F1400000000000000000000000000000000000BF
:10F150000200000004000000080000001800000089
:10F16000100000001800000018000000040000005B
:10F17000020000000000000000000000000000008D
:10F18000000000000000000000000000000000007F
:10F19000000000000000000000000000000000006F
:10F1A000000000000000000000000000000000005F
:10F1B000000000000000000000000000000000004F
:10F1C000000000010000000100000001000000013B
:10F1D000000000010000000100000001000000012B
:10F1E000000000010000000100000001000000011B
:10F1F000000000010000000100000001000000010B
:10F2000000000000000000000000000000000000FE
:10F2100000000000000000000000000000000000EE
:10F2200000000000000000000000000000000000DE
:10F2300000000000000000000000000000000000CE
:10F2400000000000000000000000000010000000AE
:10F25000100000001000000018000000080000006E
:10F26000040000000000000000000000000000009A
:10F27000000000000000000000000000000000008E
:10F28000000000000000000000000000000000007E
:10F29000000000000000000000000000000000006E
:10F2A000000000000000000000000000000000005E
:10F2B000000000000000000000000000000000004E
:10F2C000000000000000038000018FC000038C607C
:10F2D0000006182000041020000410200004202044
:10F2E00000042040000620400003FFC00001FFE0B2
:10F2F0000000002000000020000000C0000000000E
:10F3000000000000000000000000000000000000FD
:10F3100000000000000000000000000000000000ED
:10F3200000000000000000000000000000000000DD
:10F3300000000000000000000000000000000000CD
:10F3400000000000020000000200000003FFFFE0D8
:10F3500007FFFFC0000180C0000200600002002023
:10F3600000040020000400200004002000060040EB
:10F37000000300C00001FF800000FE00000000004C
:10F38000000000000000000000000000000000007D
:10F39000000000000000000000000000000000006D
:10F3A000000000000000000000000000000000005D
:10F3B000000000000000000000000000000000004D
:10F3C000000000000000000000007E000001FF803F
:10F3D000000381C00002004000060020000400205D
:10F3E0000004002000040020000600200003C040AC
:10F3F0000001C080000003000000000000000000C9
:10F4000000000000000000000000000000000000FC
:10F4100000000000000000000000000000000000EC
:10F4200000000000000000000000000000000000DC
:10F4300000000000000000000000000000000000CC
:10F44000000000000000000000007E000001FF80BE
:10F45000000380C0000600600004002000040020BB
:10F4600000040020020400400202008003FFFFE0CD
:10F4700007FFFFC000000040000000400000000047
:10F48000000000000000000000000000000000007C
:10F49000000000000000000000000000000000006C
:10F4A000000000000000000000000000000000005C
:10F4B000000000000000000000000000000000004C
:10F4C000000000000000000000007E000001FF803E
:10F4D000000311C00002104000041060000410205E
:10F4E000000410200004102000061020000310402B
:10F4F0000001F0C0000071000000000000000000EA
:10F5000000000000000000000000000000000000FB
:10F5100000000000000000000000000000000000EB
:10F5200000000000000000000000000000000000DB
:10F5300000000000000000000000000000000000CB
:10F540000000000000000000000400000004002093
:10F550000004002000040020007FFFE001FFFFE026
:10F560000104002003040020020400200204002003
:10F57000020400000200000001C0000001C0000001
:10F58000000000000000000000000000000000007B
:10F59000000000000000000000000000000000006B
:10F5A000000000000000000000000000000000005B
:10F5B000000000000000000000000000000000004B
:10F5C00000000000000000000000001C0000E33EFE
:10F5D0000003FFC200020CC3000404C1000404C104
:10F5E000000404C1000404C100060CC10003F8C3F8
:10F5F0000005F0620006007E0006003C00000000EE
:10F6000000000000000000000000000000000000FA
:10F6100000000000000000000000000000000000EA
:10F6200000000000000000000000000000000000DA
:10F6300000000000000000000000000000000000CA
:10F6400000000000020000200200002003FFFFE095
:10F6500007FFFFE00001002000020020000600007C
:10F660000004000000040000000400200006002048
:10F670000003FFE00001FFE0000000200000002088
:10F68000000000000000000000000000000000007A
:10F69000000000000000000000000000000000006A
:10F6A000000000000000000000000000000000005A
:10F6B000000000000000000000000000000000004A
:10F6C0000000000000000000000000000004002016
:10F6D0000004002000040020000400200387FFE055
:10F6E000038FFFE0038000200000002000000020C6
:10F6F00000000020000000000000000000000000EA
:10F7000000000000000000000000000000000000F9
:10F7100000000000000000000000000000000000E9
:10F7200000000000000000000000000000000000D9
:10F7300000000000000000000000000000000000C9
:10F7400000000000000000000000000000000006B3
:10F75000000000070000000100000001000400019B
:10F760000004000100040003000400060387FFFCFE
:10F77000038FFFF80380000000000000000000007D
:10F780000000000000000000000000000000000079
:10F790000000000000000000000000000000000069
:10F7A0000000000000000000000000000000000059
:10F7B0000000000000000000000000000000000049
:10F7C00000000000020000200200002003FFFFE014
:10F7D00007FFFFE0000008200000102000003000BC
:10F7E0000000FC0000058E00000707A0000601E0F5
:10F7F000000400E0000400200000002000000000E1
:10F8000000000000000000000000000000000000F8
:10F8100000000000000000000000000000000000E8
:10F8200000000000000000000000000000000000D8
:10F8300000000000000000000000000000000000C8
:10F840000000000000000000000000000200002096
:10F8500002000020020000200200002003FFFFE061
:10F8600007FFFFE000000020000000200000002053
:10F870000000002000000000000000000000000068
:10F880000000000000000000000000000000000078
:10F890000000000000000000000000000000000068
:10F8A0000000000000000000000000000000000058
:10F8B0000000000000000000000000000000000048
:10F8C00000000000000400200007FFE0000FFFE040
:10F8D0000002002000040000000400200007FFE0F8
:10F8E0000003FFE0000200200004000000040020EC
:10F8F0000007FFE00003FFE0000000200000000020
:10F9000000000000000000000000000000000000F7
:10F9100000000000000000000000000000000000E7
:10F9200000000000000000000000000000000000D7
:10F9300000000000000000000000000000000000C7
:10F940000000000000040020000400200007FFE089
:10F95000000FFFE000010020000200200002000074
:10F960000004000000040000000400200006002045
:10F970000003FFE00001FFE0000000200000002085
:10F980000000000000000000000000000000000077
:10F990000000000000000000000000000000000067
:10F9A0000000000000000000000000000000000057
:10F9B0000000000000000000000000000000000047
:10F9C000000000000000000000007E000000FF803A
:10F9D000000381C000020040000600200004002057
:10F9E0000004002000040020000600200002004067
:10F9F000000381C00001FF8000007E0000000000C5
:10FA000000000000000000000000000000000000F6
:10FA100000000000000000000000000000000000E6
:10FA200000000000000000000000000000000000D6
:10FA300000000000000000000000000000000000C6
:10FA40000000000000040001000400010007FFFFA7
:10FA5000000FFFFF000100C1000200410004002070
:10FA600000040020000400200004002000060040E4
:10FA7000000301C00001FF8000007E0000000000C4
:10FA80000000000000000000000000000000000076
:10FA90000000000000000000000000000000000066
:10FAA0000000000000000000000000000000000056
:10FAB0000000000000000000000000000000000046
:10FAC000000000000000000000007E000001FF8038
:10FAD000000380C000020060000400200004002039
:10FAE000000400200004002000020041000300C1C7
:10FAF0000003FFFF0007FFFF0000000100000001FE
:10FB000000000000000000000000000000000000F5
:10FB100000000000000000000000000000000000E5
:10FB200000000000000000000000000000000000D5
:10FB300000000000000000000000000000000000C5
:10FB40000000000000040020000400200004002049
:10FB500000040020000FFFE0000FFFE00000C020C5
:10FB60000001002000020020000600200004000028
:10FB70000004000000070000000300000000000077
:10FB80000000000000000000000000000000000075
:10FB90000000000000000000000000000000000065
:10FBA0000000000000000000000000000000000055
:10FBB0000000000000000000000000000000000045
:10FBC0000000000000000000000003E00001C0E0B1
:10FBD0000003E0400006302000043020000418201C
:10FBE000000418200004182000040C2000020C60FF
:10FBF000000307C000078380000000000000000031
:10FC000000000000000000000000000000000000F4
:10FC100000000000000000000000000000000000E4
:10FC200000000000000000000000000000000000D4
:10FC300000000000000000000000000000000000C4
:10FC400000000000000000000004000000040000AC
:10FC500000040000000C0000001FFF8000FFFFC038
:10FC600000040060000400200004002000040020C4
:10FC700000040040000001800000000000000000BF
:10FC80000000000000000000000000000000000074
:10FC90000000000000000000000000000000000064
:10FCA0000000000000000000000000000000000054
:10FCB0000000000000000000000000000000000044
:10FCC0000000000000040000000400000007FF80A6
:10FCD000000FFFC0000000600000002000000020B6
:10FCE000000000200000002000040040000400800C
:10FCF0000007FFE0000FFFC00000004000000040D0
:10FD000000000000000000000000000000000000F3
:10FD100000000000000000000000000000000000E3
:10FD200000000000000000000000000000000000D3
:10FD300000000000000000000000000000000000C3
:10FD40000000000000040000000400000007800024
:10FD50000007F0000004FE0000041FC0000003E0E4
:10FD60000000038000001C00000460000007800009
:10FD70000006000000040000000000000000000079
:10FD80000000000000000000000000000000000073
:10FD90000000000000000000000000000000000063
:10FDA0000000000000000000000000000000000053
:10FDB0000000000000000000000000000000000043
:10FDC00000040000000600000007C0000007FC005F
:10FDD00000043F80000003E000040F800006F000F4
:10FDE0000007F0000007FF8000040FE00000038020
:10FDF00000043C000007C0000006000000040000F2
:10FE000000000000000000000000000000000000F2
:10FE100000000000000000000000000000000000E2
:10FE200000000000000000000000000000000000D2
:10FE300000000000000000000000000000000000C2
:10FE4000000000000000002000040020000400600A
:10FE5000000700E0000783200007E6000004F80028
:10FE600000003C0000045E20000587A0000601E0C1
:10FE700000040060000400200000002000000000DA
:10FE80000000000000000000000000000000000072
:10FE90000000000000000000000000000000000062
:10FEA0000000000000000000000000000000000052
:10FEB0000000000000000000000000000000000042
:10FEC000000000000004000000040003000700031D
:10FED0000007E0010004F80100041F02000007FC15
:10FEE000000000E000000700000438000007C00028
:10FEF00000060000000400000004000000000000F4
:10FF000000000000000000000000000000000000F1
:10FF100000000000000000000000000000000000E1
:10FF200000000000000000000000000000000000D1
:10FF300000000000000000000000000000000000C1
:10FF4000000000000000000000078060000600E0E4
:10FF5000000403E0000407A000040E2000043C207D
:10FF6000000470200005E0200007802000070060EA
:10FF7000000400E00000038000000000000000001A
:10FF80000000000000000000000000000000000071
:10FF90000000000000000000000000000000000061
:10FFA0000000000000000000000000000000000051
:10FFB0000000000000000000000000000000000041
:10FFC0000000000000000000000000000000000031
:10FFD00000000000000000000000000000008000A1
:10FFE000000080000001400007FE3FF80800000408
:10FFF00010000002100000020000000000000000DD
:02000004900169
:1000000000000000000000000000000000000000F0
